:020000040800F2
:10000000F8B20120390300085B2B0008C922000860
:10001000592B0008E1070008253100080000000006
:10002000000000000000000000000000790200084D
:100030009508000800000000D50200083D2D0008CA
:100040005303000853030008530300085303000838
:100050005303000853030008530300085303000828
:100060005303000853030008530300085303000818
:10007000530300085303000853030008E507000872
:100080005303000853030008530300080000000056
:100090000000000000000000000000005303000802
:1000A0005303000853030008F92D00085303000808
:1000B00053030008530300085303000853030008C8
:1000C00053030008530300085303000853030008B8
:1000D0005303000853030008530300080000000006
:1000E00053030008530300085303000800000000F6
:1000F00000000000000000000000000053030008A2
:1001000000000000530300085303000853030008D5
:1001100000000000000000000000000000000000DF
:100120005303000853030008530300085303000857
:100130005303000800000000000000000000000061
:100140000000000000000000000000005303000851
:100150005303000853030008530300085303000827
:1001600053030008530300080000000000000000D3
:10017000000000000000000000000000000000007F
:100180000000000053030008000000000000000011
:10019000530300085303000800F002F800F05CF875
:1001A0000AA090E8000C82448344AAF10107DA45D2
:1001B00001D100F051F8AFF2090EBAE80F0013F0C8
:1001C000010F18BFFB1A43F001031847B0F90200F2
:1001D000D0F902000A444FF0000C10F8013B13F074
:1001E000070408BF10F8014B1D1108BF10F8015B90
:1001F000641E05D010F8016B641E01F8016BF9D183
:1002000013F0080F1EBF10F8014BAD1C0C1B09D1D9
:100210006D1E58BF01F801CBFAD505E014F8016B4B
:1002200001F8016B6D1EF9D59142D6D370470000DD
:100230000023002400250026103A28BF78C1FBD8EF
:10024000520728BF30C148BF0B6070471FB527F069
:1002500098F91FBD10B510BD00F0F4F91146FFF775
:10026000F5FF1FF0D3F800F012FA03B4FFF7F2FF26
:1002700003BC00F019FA00002C4B19680868B0E8BC
:10028000F04F80F30988BFF36F8F4FF0000080F3C9
:10029000118870470000000008480068006880F37B
:1002A00008884FF0000080F3148862B661B6BFF38F
:1002B0004F8FBFF36F8F00DF00BF00BF08ED00E07E
:1002C000DFF80C00016841F470010160704700BF65
:1002D00088ED00E0EFF30980BFF36F8F134B1A68CE
:1002E0001EF0100F08BF20ED108A20E9F04F1060BB
:1002F00009B44FF0500080F31188BFF34F8FBFF364
:100300006F8F26F0DBFA4FF0000080F3118809BCF4
:1003100019680868B0E8F04F1EF0100F08BFB0EC85
:10032000108A80F30988BFF36F8F70472000002088
:10033000EFF30580704700000948804709480047EF
:10034000FEE7FEE7FEE7FEE7FEE7FEE7FEE7FEE785
:10035000FEE7FEE704480549054A064B70470000E2
:10036000E92D000899010008F8AC0120F8B201203D
:10037000F8AE0120F8AE012053EA020C00F06980CB
:100380002DE9F04B4FF00006002B1FBFB3FA83F5A9
:1003900003FA05F424FA05F65E4012BF1643B2FADA
:1003A00082F502FA05F4C5F120051EBF22FA05FC0C
:1003B00044EA0C04203556EA044C4FEA144418BFB2
:1003C000641C4FF000084FF00009904271EB030CE1
:1003D00039D3002919BFB1FA81F701FA07F6B0FA4B
:1003E00080F700FA07F6C7F120071EBF20FA07FCC6
:1003F00046EA0C062037B6FBF4FCA7EB0507103FD6
:1004000007F01F0BCBF120060CFA0BFB2CFA06F6BB
:1004100044BFB3460026202FA4BF5E464FF0000B1A
:100420005BEA060C08BF4FF0010B19EB0B09ABFBA5
:10043000027C48EB0608C01B06FB02CC0BFB03CC7E
:1004400071EB0C01C1E70B46024641464846BDE848
:10045000F08B13B54FF000004FF00001AFF30080B8
:10046000BDE81C40704710B54C1084EA530404D515
:100470004042C1F1000138BF491E1B4204D552421F
:10048000C3F1000338BF5B1EFFF776FF14F0804F07
:1004900004D04042C1F1000138BF491E14F0004FA2
:1004A00004D05242C3F1000338BF5B1E10BD032AC3
:1004B00040F2308010F0030C00F0158011F8013B81
:1004C000BCF1020F624498BF11F801CB00F8013B68
:1004D00038BF11F8013BA2F1040298BF00F801CB2C
:1004E00038BF00F8013B11F0030300F02580083A03
:1004F000C0F0088051F8043B083A51F804CBA0E85A
:100500000810F5E7121D5CBF51F8043B40F8043BAE
:10051000AFF30080D20724BF11F8013B11F801CBE3
:1005200048BF11F8012B24BF00F8013B00F801CBB4
:1005300048BF00F8012B704710B5203AC0F00B807F
:10054000B1E81850203AA0E81850B1E81850A0E8D7
:100550001850BFF4F5AF5FEA027C24BFB1E8185031
:10056000A0E8185044BF18C918C0BDE810405FEAA1
:10057000827C24BF51F8043B40F8043B08BF70471D
:10058000D20728BF31F8023B48BF11F8012B28BF22
:1005900020F8023B48BF00F8012B704702F0FF0330
:1005A00043EA032242EA024200F02CB84FF0000274
:1005B00000B5134694469646203922BFA0E80C5059
:1005C000A0E80C50B1F12001BFF4F7AF090728BF34
:1005D000A0E80C5048BF0CC05DF804EB890028BFB0
:1005E00040F8042B08BF704748BF20F8022B11F0D9
:1005F000804F18BF00F8012B704770477047704755
:100600004FF000020429C0F0128010F0030C3FF4F8
:10061000CFAFCCF1040CBCF1020F18BF00F8012BD6
:10062000A8BF20F8022BA1EB0C01FFF7C1BF5FEAC6
:10063000C17C24BF00F8012B00F8012B48BF00F853
:10064000012B7047754600F02BF8AE460500694651
:10065000534620F00700854618B020B5FFF77AFE14
:10066000BDE820404FF000064FF000074FF00008B3
:100670004FF0000B21F00701AC46ACE8C009ACE834
:10068000C009ACE8C009ACE8C0098D46704710B598
:100690000446AFF300802046BDE81040FFF7E5BDFB
:1006A0000048704798AC012001491820ABBEFEE716
:1006B0002600020070470000464910B54A6822F43F
:1006C00040324A604A6843681A434A6001684A688F
:1006D00022F480724A6001684A68036942EA032290
:1006E0004A6001684A6822F040724A6001684A68BC
:1006F00083681A434A6001688A6822F400628A604B
:1007000001688A68C3681A438A60816A6FF0706200
:10071000D14201688A6822F070628A6001688A6842
:100720000CD0836A1A438A6001688A6822F04052BA
:100730008A6001688A68C36A1A4301E022F0405265
:100740008A6001688A6822F002028A6001688A6809
:10075000037E42EA43028A6090F820100029016873
:100760004A680FD042F400624A6001684A6822F485
:1007700060424A6001684A68174C436A04EB43339D
:100780001A4301E022F400624A600168CA6A22F456
:100790007002CA620168CA6A838B104C04EB03536F
:1007A0001A43CA6201688A6822F400728A6001688A
:1007B0008A6890F8303042EA43228A6001688A6889
:1007C00022F480628A6001688A68406942EA802077
:1007D000886010BD0023014000E0FFFF0000F0FF33
:1007E000FEE70000014800F065B90000400200206B
:1007F00001681823CAB2103AB2FBF3F2054B6FF34B
:100800000901032A9B5CC36500D9091D816508465F
:1008100070470000F875020810B5014600208B698A
:100820008A6A4FF0C07453B1B3F5005F15D072B14E
:10083000012A0CD0022A0AD0032A09D104E01AB1F5
:10084000012A06D0022A03D1C96AC90100D50120B4
:1008500010BDC96AA142FAD010BD002AF7D0012A02
:10086000F2D0022AF3D0032AF3D010BD30B50468C9
:10087000256825F480252560046863608368402B23
:10088000036803D099600068C26030BD9A60006858
:10089000C16030BD704772B6FEE7000078B5002435
:1008A000009490F83C20012A19D0012280F83C20C5
:1008B0000A6807230568092A13D9EE680A3A02EB89
:1008C000420293409E43EE600B788A680A3B03EB3A
:1008D00043039A400368DD682A43DA6010E002208F
:1008E00078BD2E6902EB420293409E432E610B7845
:1008F0008A6803EB43039A4003681D692A431A611F
:100900004A681F23072A13D205686E6B521E02EB3A
:10091000820293409E436E630A8893B20A79521E04
:1009200002EB820293400268556B2B43536327E02E
:1009300005680D2A12D22E6BD21F02EB8202934061
:100940009E432E630B790A88DB1F92B203EB83036D
:100950009A4003681D6B2A431A6311E0EE6A0D3A50
:1009600002EB820293409E43EE620B790A880D3BB4
:1009700092B203EB83039A400368DD6A2A43DA628A
:100980001B4B0568194A9D420AD10D68122D07D1EB
:10099000556825F400055560556845F48005556097
:1009A00005689D421DD1134D0B68AB4201D0112B40
:1009B00017D1536823F480035360536843F4000352
:1009C00053600968A9420CD10B490C4A0968B1FB74
:1009D000F2F101EB8101490000E0491E009100297C
:1009E000FBD180F83C40002078BD0000002301408E
:1009F00000200140120000101C00002040420F00A7
:100A000070B504004FF0000503D0206C002610B133
:100A100007E0012070BD204600F01CF8666484F8F1
:100A20003C60206CC00610D4206C20F4885040F04C
:100A3000020020642046FFF73FFE6664206C20F031
:100A4000020040F00100206400E0012584F83C60D1
:100A5000284670BD10B586B0044614216846FFF7DD
:100A6000A5FD1149206888421CD110480021026868
:100A700042F480720260006800F4807005900B48B8
:100A80001438026842F001020260006800F00100C0
:100A90000590E02000900320CDE90101694604485B
:100AA00000F08CF906B010BD00200140443802402F
:100AB000000002402DE9F84304464FF00009CDF84C
:100AC000009063484FF41651A56D0068B0FBF1F734
:100AD0002E6894F85C10082000FA01F131420FD022
:100AE00021680A6852070BD50A6822F004020A60DE
:100AF00094F85C108840A860606D40F0010060656B
:100B000094F85C104FF0010808FA01F0304208D068
:100B100021684969090604D5A860606D40F00200AB
:100B2000606594F85C1004208840304208D0216849
:100B30000968890704D5A860606D40F0040060650D
:100B400094F85C1010208840304218D02168096861
:100B5000090714D5A86020680168490304D5006816
:100B6000000308D5A16C07E00168C90503D401683A
:100B700021F008010160216C09B12046884794F8F2
:100B80005C1020208840304231D021680968C906B5
:100B90002DD5A86094F8350005282068016806D096
:100BA000490347D5006800031DD4616C1CE021F0A7
:100BB000160101602068416921F080014161206CCB
:100BC00008B9A06C20B12068016821F0080101601B
:100BD00094F85C103F208840A86084F8358084F841
:100BE0003490216D1FE0E16B09B120468847606DAC
:100BF00000282BD0606DC00714D0052084F8350084
:100C00002068016821F0010101600098401C0090FB
:100C1000B84203D820680068C007F6D184F8358050
:100C200084F83490E16C002910D001B02046BDE872
:100C3000F04308470168C905D5D4016821F01001C7
:100C4000016084F8358084F83490CCE7BDE8F883FF
:100C50001C0000202DE9F041044600F0ADF90646E5
:100C60005CB1022084F83500002584F834502068F7
:100C7000016821F0010101600DE00120BDE8F08173
:100C800000F09AF9801B052805D920206065032013
:100C900084F83500F2E720680068C007F0D12268C8
:100CA000116820480140D4E901031843D4E9033610
:100CB0003343184363691843A3691843E36918432E
:100CC000236A18430843616A042903D1D4E90B134A
:100CD00019430843106020684069666A20F00701E4
:100CE00030460E43012704280CD1A06A0643E06A6F
:100CF00040B12046FFF790FD20B14020606584F8A8
:100D00003570BAE7206846612046FFF771FD94F818
:100D10005C203F2191408160656584F8357000203A
:100D2000ACE700003F8010F02DE9F0410446866DED
:100D300090F83400002501280DD0012084F83400FB
:100D400094F835700020012F07D084F83400022574
:100D50002846BDE8F0810220FBE7022784F83570C1
:100D600060652046FFF782FD94F85C103F208840C4
:100D7000B0602068016841F016010160206C20B16C
:100D80002068016841F0080101602068016841F0B5
:100D900001010160DCE7000070B5044600F00CF9C9
:100DA0000546601C02D004480078044400F004F9B1
:100DB000401BA042FAD370BD100000202DE9F84F6F
:100DC000DFF8B8A10022012403254FF00F090AF132
:100DD000040BAAF1040E00BF0B6804FA02F63340BC
:100DE000B34273D10F7907F00307012F01D0022F0F
:100DF00016D187684FEA420805FA08FC27EA0C0773
:100E0000D1F80CC00CFA08FC4CEA070CC0F808C07A
:100E10004768B7430E79C6F3001696403E434660D6
:100E20000E79F643B6070DD0C768560005FA06FCE2
:100E300027EA0C07D1F808C00CFA06FC4CEA070CAC
:100E4000C0F80CC00E7906F00306022E10D1D608A9
:100E500000EB8608D8F8206057074FEAD76C09FAEC
:100E60000CF7BE430F6907FA0CF73743C8F8207038
:100E700006684FEA420C05FA0CF7BE430F7907F0FB
:100E8000030707FA0CF7374307604E6816F4403F34
:100E90006DD03B4E376847F480473760366822F0A4
:100EA000030706F480460096364E07EB060CDCF886
:100EB000086897073F0F09FA07F826EA0806DFF8DF
:100EC000C880404503D14FF000081EE04FE0DFF836
:100ED000BC80404502D14FF0010816E0DFF8B08039
:100EE000404502D14FF002080FE0DFF8A8804045EE
:100EF00002D14FF0030808E0DFF89C80404502D1A2
:100F00004FF0040801E04FF0070808FA07F848EA34
:100F10000608CCF80888DAF800605746D1F804C013
:100F20009E435FEACC2C00D51E433E60DBF8006098
:100F30005F46D1F804C09E435FEA8C2C00D51E4367
:100F40003E60DEF800607746D1F804C09E435FEA59
:100F50008C3C00D51E433E60084F083F3E68D1F8E8
:100F600004C09E435FEACC3C00D51E433E60521C49
:100F7000102AFFF431AFBDE8F88F0000083C0140B3
:100F800044380240003001400000024000040240AA
:100F900000080240000C024000100240426921EAB1
:100FA00002030A4043EA0241816170470AB181614C
:100FB00070470904FBE700000148806870470000A3
:100FC0001000002070B5040025D094F83D000025E5
:100FD00020B984F83C50204600F0B8F8242084F86A
:100FE0003D002068016821F001010160206801686E
:100FF00041F4004101602068016821F40041016072
:1010000000F056FA4D4A6168914201D84C4900E01F
:101010004C49884201D2012070BD4B492368B0FB86
:10102000F1F15E6826F03F060E435E60636893420E
:1010300006D94FF4967359434FF47A73B1FBF3F129
:101040002368491C1E6A26F03F0631431962616815
:10105000914210D84900401EB0FBF1F2521CC2F37D
:101060000B02042A01D2042022E0B0FBF1F0401C64
:10107000C0F30B001CE0A268F2B301EBC10303EB69
:101080000116431EB3FBF6F35B1C43F480431B05C0
:1010900049D092B301EBC10202EB0111401EB0FB3B
:1010A000F1F0401CC0F30B0040F4804040F40040DD
:1010B0002168CA694CF6FF739A431043C861D4E9AA
:1010C000071001432068026822F0C002114301604A
:1010D000D4E9030101432068826848F2FF339A4350
:1010E00011438160D4E9050108432168CA6822F0F0
:1010F000FF021043C86001E00EE016E020680168BE
:1011000041F0010101602564202084F83D00256341
:1011100084F83E50002070BD01EB4106431EB3FB36
:10112000F6F35B1CB3E70120C2E701EB4101401E6F
:10113000B0FBF1F0401CC0F30B00B7E7A086010044
:1011400080841E0000093D0040420F0010B586B0AB
:10115000044614216846FFF729FA1349206888429B
:1011600020D112480021026842F0020202600068A9
:1011700000F002000590C02000901220CDE901018E
:10118000032003900420049069460948FFF716FEE7
:1011900006481030016841F400110160006800F455
:1011A0000010059006B010BD0054004030380240D9
:1011B000000402400248816802781144816070474F
:1011C000100000200B4810B5016841F40071016067
:1011D000016841F480610160016841F4807101603F
:1011E000032000F099F80F2000F006F800F04AF80C
:1011F000002010BD003C024030B505461C4887B0B9
:101200000024016841F480210160006806A900F40F
:101210008020009001A800F02BF900F059F9154941
:10122000154AB0FBF1F11548491E026040F2E73261
:10123000C0E90324C0E90114846100F077FD0400D3
:1012400012D10E4800F0A0FD04000DD11A2000F0CC
:1012500035F8102D07D2002229461A2000F03CF85C
:101260000748056000E0012407B0204630BD0000BB
:101270004438024040420F000048014078030020FB
:10128000140000200C4882B0016841F480410160E4
:10129000006800F4804000900748001F016841F09A
:1012A000805101600068002200F0805000900F2102
:1012B000901E02B000F010B844380240002809DB4C
:1012C00000F01F02012191404009800000F1E02060
:1012D000C0F8001170470000F0B40E4B1B680C46BC
:1012E000C3F30223C3F10705042D00D90425191DFA
:1012F000072901D2002300E0DB1E012606FA05F1D2
:10130000491E214099409E40761E16403143F0BC54
:1013100001F028BF0CED00E0064900F00702086864
:101320004FF6FF03184040EA0220034A10430860CA
:10133000704700000CED00E00000FA052DE9F047D1
:101340000E46050065D0DFF81481D8F80000F7B22A
:1013500000F00700B04207D288F80070D8F800000B
:1013600000F00700B04254D128683D4C810712D5E7
:10137000400703D5206840F4E0502060287800073B
:1013800003D5206840F4604020602068A96820F000
:10139000F000084320602878C0072DD030496868E5
:1013A0000839012812D0022813D0032811D0096867
:1013B000890700292DDA216821F00301014321600A
:1013C000FFF7FAFD814641F2883A0EE00968890389
:1013D000EFE709688901ECE7FFF7EEFDA0EB0901F3
:1013E000514502D90320BDE8F0872068696800F004
:1013F0000C00B0EB810FEFD1D8F80010404601F09F
:101400000701B14207D90770006800F00700B04239
:1014100001D00120E7E72878400705D52068E96872
:1014200020F4E050084320602878000706D52068A3
:10143000296920F4604040EAC100206000F058F8BB
:101440002168084AC1F30311515CC840064908608D
:1014500006480068FFF7D0FE0020C4E7003C0240C9
:10146000083802401CAF02081C00002014000020B5
:101470000F2202600C4A136803F0030343601368F1
:1014800003F0F0038360136803F4E053C360126851
:101490004FF4E05303EAD20202610448006800F00E
:1014A000070008607047000008380240003C024016
:1014B0000448054900680968044AC1F38221515C67
:1014C000C84070471C000020083802402CAF0208BA
:1014D0000448054900680968044AC1F34231515C77
:1014E000C84070471C000020083802402CAF02089A
:1014F000154810B5006810F00C02144813D01449B8
:10150000042A0FD0082A0ED10F4C241F226823680A
:1015100002F03F025B0207D52068C0F38810A0FBF1
:10152000010106E0084610BD2168C1F38811A1FB46
:1015300000010023FEF720FF2168C1F30141491C8F
:101540004900B0FBF1F010BD083802400024F4005F
:1015500040787D012DE9F84F04006ED02078DFF847
:101560004C93C007A9F104054AD009F104000168B1
:10157000C1F38101012908D00068C0F3810002286D
:101580000AD1D9F80000400206D52868800337D573
:1015900060680028E1D033E06068B0F5803F10D08B
:1015A000B0F5A02F286810D020F48030286028687B
:1015B00020F4802028606068A8B1FFF7FDFC064693
:1015C0000DE0286840F48030F4E740F48020286083
:1015D000F7E700BFFFF7F0FC801B642873D828688A
:1015E0008003F7D50CE0FFF7E7FC064605E000BFF7
:1015F000FFF7E2FC801B6428F0D828688003F7D44A
:101600002078DFF8AC8280074FF0000A3ED5A7486B
:10161000001D016811F00C0F08D00068C0F38100B4
:1016200002280BD1D9F80000400207D428688007AF
:1016300016D5E068012800D112E033E1E068B8B1C6
:101640000120C8F80000FFF7B7FC064605E000BF20
:10165000FFF7B2FC801B0228C0D828688007F7D5A6
:101660002868216920F0F80040EAC10028600DE0F8
:10167000C8F800A0FFF7A0FC064604E0FFF79CFCBA
:10168000801B02281FD828688007F7D4207800071D
:1016900022D5864F87486169703771B10121016099
:1016A000FFF78AFC064604E0FFF786FC801B022851
:1016B00009D838688007F7D50EE0C0F800A0FFF71A
:1016C0007BFC064605E082E0FFF776FC801B0228E3
:1016D0007DD838688007F7D42078400768D5DFF8D0
:1016E000CCB100270BF13C0BDBF80000C0000BD4A1
:1016F000DBF8001041F08051CBF80010DBF800005F
:10170000012700F0805000906B4E3068C00510D467
:10171000306840F480703060FFF74EFC009005E0C8
:10172000FFF74AFC0099401A022850D83068C005DB
:10173000F6D55E4EA0686C3601280FD005283068BB
:1017400010D020F001003060306820F004003060DC
:10175000A068B8B1FFF730FC00900FE0306840F0AF
:101760000100F4E740F004003060F7E7FFF724FCE5
:101770000099411A41F28830814266D8306880076A
:10178000F4D50EE0FFF718FC009007E0FFF714FC1B
:101790000099411A41F28830814256D8306880075A
:1017A000F4D42FB1DBF8001021F08051CBF80010F9
:1017B000A069C8B33D49091D0968C1F38101022927
:1017C0004AD00228504607D0C8F8600000E03CE04C
:1017D000FFF7F2FB04463BE04746C8F86000FFF71E
:1017E000EBFB064605E000BFFFF7E6FB801B022887
:1017F0002BD828688001F7D4D4E907010843A16AEF
:101800002E4A490802EB0141626A41EA821108430B
:1018100094F82C1040EA0161C9F8001001203866E4
:10182000FFF7CAFB044606E03EE000BFFFF7C4FB3B
:10183000001B022809D828688001F7D534E000BFD2
:10184000FFF7BAFB001B022802D90320BDE8F88F7E
:1018500028688001F4D427E00128F7D0D9F80000E7
:10186000E26900F4800191421CD1226A00F03F013C
:10187000914217D147F6C071626A0140B1EB821FF5
:1018800010D1A26A4FF0FF3300F4403103EB520253
:10189000B1EB024F06D194F82C1000F07060B0EB61
:1018A000016F01D00120D1E70020CFE704380240CA
:1018B00000004742800E4742007000400000FFFFDA
:1018C000704770B5040009D0606A002540B12561F9
:1018D0006561A56294F8510040B10CE0012070BD33
:1018E0006068B0F5827FF4D0E561F2E784F850508B
:1018F000204600F045F8022084F851002068016875
:1019000021F040010160A088218900F4827001F477
:1019100004410843A18901F400610843217C01F0DE
:1019200002010843217D01F001010843218B01F4EC
:1019300000710843217F01F03801084394F820101A
:1019400001F080010843218D01F400510843216812
:101950000860A069042101EA104094F8241001F005
:1019600010010843216848602068C16921F40061C2
:10197000C1616565012084F85100002070BD000040
:1019800070B586B0064614216846FEF70FFE1F4963
:101990003068884238D11E480025016841F48041F2
:1019A0000160006800F48040059019481038016813
:1019B00041F0020101600068694600F002000590F4
:1019C0004FF4204000900220CDE901050320039050
:1019D000052004900F48FFF7F1F9104C0E48C4E9B8
:1019E00000054020C4E9020500012061400060615B
:1019F000C4E90605256220466562FFF72BF908B1A8
:101A0000FEF749FFB464A66306B070BD003800401D
:101A10004038024000040240706002404002002052
:101A20002DE9F84F984616468A460446FFF7C4FA51
:101A3000814694F8510001281ED1BAF1000F73D0ED
:101A4000002E71D094F85000012815D0012784F899
:101A50005070032084F8510000256565C4F830A05B
:101A6000A686E686A563A587E58765642564A068E4
:101A7000B0F5004F03D00CE00220BDE8F88F2068DD
:101A8000016821F0400101602068016841F4804153
:101A9000016020680168490603D4016841F04001F3
:101AA0000160E068B0F5006F606803D048B3012EB4
:101AB00027D047E008B1012E1FD1206B2168008894
:101AC000C86006E020688168890709D5216B09880C
:101AD000C160206B801C2063E08E401EE0860CE01D
:101AE000FFF76AFAA0EB0901414503D3B8F1FF3FC4
:101AF00003D035E0B8F1000F32D0E08E0028E1D1FC
:101B000023E0206B21680078087306E02068816874
:101B100089070AD5216B09780173206B401C20636B
:101B2000E08E401EE0860DE02BE0FFF745FAA0EBCB
:101B30000901414503D3B8F1FF3F03D010E0B8F1EC
:101B4000000F0DD0E08E0028E0D14A4641462046E5
:101B500001F052F808B120206065A06830B109E0BA
:101B600084F8517084F85050032086E72068C168DB
:101B70008068009084F8517004F8505F6068002815
:101B8000F3D0012079E7000070B5044690F85100C9
:101B900001281CD1C9B1C2B194F85000012816D057
:101BA000012084F85000032084F851000025656569
:101BB0002163A286E286A56365642564A587E5871F
:101BC000A068B0F5004F04D00DE0012070BD0220E8
:101BD00070BD2068016821F0400101602068016843
:101BE00041F480410160A16C17480864A16C17485A
:101BF000C863A16C1648C864A06C0565E38E2268B2
:101C0000216B0C32A06CFFF78FF830B1606D40F0A3
:101C10001000606584F85050D7E7206801684906D5
:101C200003D4016841F04001016084F850502068FD
:101C3000416841F0200141602068416841F00201A3
:101C40004160002070BD00008B2B0008952B000820
:101C5000692B0008704770477047704710B590F8BF
:101C60003C20012A22D0012280F83C20CA688C68DE
:101C700022F4407222434C6822F4806222430C68B2
:101C800022F4006222430C6922F4805222434C6900
:101C900022F400522243C969002322F480420A43FD
:101CA00001684A6480F83C30002010BD022010BD5D
:101CB00070B590F83C20012A2CD0012480F83C40DB
:101CC000022280F83D2003685A689D6822F0700661
:101CD0000A6832435A60104B02689A420ED0B2F141
:101CE000804F0BD00D4B9A4208D00D4B9A4205D035
:101CF0000C4B9A4202D00C4B9A4204D1496825F011
:101D000080031943916080F83D40002180F83C1029
:101D1000084670BD022070BD000001400004004074
:101D200000080040000C00400040014010B50400D5
:101D300003D094F83D0010B107E0012010BD002051
:101D400084F83C00204600F01EF8022084F83D0094
:101D5000211D206801F05EF8012084F8460084F817
:101D60003E0084F83F0084F8400084F8410084F885
:101D7000420084F8430084F8440084F8450084F865
:101D80003D00002010BD704790F83D10012901D0A2
:101D900001207047022180F83D100168CA6842F0B6
:101DA0000102CA6000680E4988420ED0B0F1804F2F
:101DB0000BD00C49884208D00B49884205D00B490A
:101DC000884202D00A49884204D1816801F00701A3
:101DD000062903D0016841F001010160002070472D
:101DE000000001400004004000080040000C0040DA
:101DF0000040014070472DE9F04104460068C66884
:101E000005694FF00007A90713D5B10711D5F91ED1
:101E1000016101202077206880698007204602D078
:101E2000FFF7E8FF04E000F0C1F8204600F07EF97B
:101E30002777680716D5700714D521686FF004005E
:101E40000861022020772068806910F4407F2046D6
:101E500002D0FFF7CFFF04E000F0A8F8204600F022
:101E600065F92777280715D5300713D521686FF056
:101E700008000861042020772068C0698007204698
:101E800002D0FFF7B7FF04E000F090F8204600F022
:101E90004DF92777E80616D5F00614D521686FF0BE
:101EA00010000861082020772068C06910F4407F86
:101EB000204602D0FFF79EFF04E000F077F82046AE
:101EC00000F034F92777E80708D0F00706D021683A
:101ED0006FF001000861204600F082F9280608D55D
:101EE000300606D521686FF0800008612046FFF7B4
:101EF000B3FE680608D5700606D521686FF040006D
:101F00000861204600F076F9A8060AD5B00608D583
:101F100021686FF0200008612046BDE8F041FFF71E
:101F20009CBEBDE8F081000010B586B004461421C7
:101F30006846FEF73BFB2368174C00211748022236
:101F4000A34211D1036843F001030360006800F06D
:101F50000100059050020090CDE901210120CDE95A
:101F6000031069460E4812E00E4CA34211D10368DB
:101F700043F002030360006800F002000590601562
:101F80000090CDE90121CDE9031269460648FEF72C
:101F900015FF06B010BD00000000014030380240BF
:101FA000000002400008004000040240704770B585
:101FB000044690F83C0000260D4601280FD0012071
:101FC00084F83C006AB1042A1DD0082A2FD00C2ABC
:101FD0003FD00126002084F83C00304670BD02202E
:101FE00070BD206800F076FF2068816941F008012B
:101FF00081612068816921F0040181612068816923
:102000002A69114311E0206800F08CFF2068816983
:1020100041F4006181612068816921F480618161FE
:10202000206881692A6941EA02218161D2E720683A
:1020300000F0A4FF2068C16941F00801C161206877
:10204000C16921F00401C1612068C1692A69114395
:1020500011E0206800F0BEFF2068C16941F4006112
:10206000C1612068C16921F48061C1612068C169D2
:102070002A6941EA0221C161ACE710B5040003D02E
:1020800094F83D0010B107E0012010BD002084F855
:102090003C00204600F01EF8022084F83D00211D7F
:1020A000206800F0B7FE012084F8460084F83E0066
:1020B00084F83F0084F8400084F8410084F842002E
:1020C00084F8430084F8440084F8450084F83D0017
:1020D000002010BD08B500681149884212D111488E
:1020E000016841F0010101600068002200F0010078
:1020F00000900F211A20FFF7EFF8BDE808401A20E2
:10210000FFF7DCB80849884209D10648001F01687A
:1021100041F004010160006800F00400009008BD77
:1021200000000140443802400008004070470000B1
:1021300010B50446022249B104290ED0082913D053
:1021400094F84100012816D0012010BD94F83E00FB
:102150000128F9D184F83E200FE094F83F000128CF
:10216000F2D184F83F2008E094F840000128EBD138
:1021700084F8402001E084F841200122206800F02A
:102180009BFE12492068884203D1426C42F400420F
:102190004264206888420ED0B0F1804F0BD00C49C9
:1021A000884208D00B49884205D00B49884202D0AA
:1021B0000A49884204D1816801F00701062903D049
:1021C000016841F001010160002010BD00000140E4
:1021D0000004004000080040000C004000400140A6
:1021E00000680349884201D1FEF7E4BF7047000050
:1021F00000480140704770B5040004D094F84100D5
:10220000002510B106E0012070BD84F84050204642
:1022100000F024F8242084F841002068C16821F4EB
:102220000051C160204600F0F7FE2068016921F4EA
:10223000904101612068416921F02A0141612068D3
:10224000C16841F40051C1606564202084F84100F8
:1022500084F842006563002070BD000010B586B0B0
:10226000044614216846FEF7A1F914492068884203
:1022700021D113480021026842F020020260006868
:1022800000F0200005900E481438026842F0010268
:102290000260006800F0010005904FF4C05000900B
:1022A0000220CDE901010320039008200490694633
:1022B0000448FEF783FD06B010BD00000014014085
:1022C0004438024000000240FEE700000EB5002442
:1022D00018254FF6FF764FF4FA7700BF24F0E6FAA0
:1022E00008211448FFF724FF00F02CF800F0F6F85E
:1022F000F02300211A460846009400F092F832209C
:1023000000F0C6F9CDE9004533460BA278214820FC
:10231000029400F053FA13F00FF819F079FA23F051
:10232000D3FD25F033F8002024F0F2F938461DF0F3
:10233000CAFAD3E7A002002057656C636F6D652170
:102340000000000000B587B014216846FEF72EF9A2
:1023500009480021026842F001020260006800F0B2
:10236000010005900120CDE9000102906946034873
:10237000FEF724FD07B000BD3038024000000240E7
:102380002DE9F04104461D4616460F462A2000F06E
:1023900043FA204600F030FA304600F02DFA2B20A8
:1023A00000F03AFA384600F027FA284600F024FAFE
:1023B000BDE8F0412C2000F02FBA000070B5141ACF
:1023C0005D1A641C6D1C6C43049EFFF7D9FF0D4D14
:1023D0004FF40060E8602868016841F40061016022
:1023E000A2B231462846FFF7CFFB07480068416894
:1023F0000029FCD10020E8602868016821F4006110
:10240000016070BDE80100204002002010B51446B4
:102410000B460246FFF7B4FF2046BDE8104000F02F
:10242000EBB92DE9F04780461F46581E83B2164689
:10243000501E82B20C464046DDF82090FFF7A0FF08
:102440000AE0454604E0484600F0D6F96D1CADB2FE
:10245000B542F8D3641CA4B2BC42F2D3BDE8F08705
:10246000F0B587B014216846FEF7A0F81848016857
:1024700041F002010160016801F00201059101686B
:1024800041F00201016000684FF4805600F0020044
:10249000059001240F4FCDE900640325694603959B
:1024A0003846FEF78BFC012231463846FEF77EFDAA
:1024B0002E02CDE90064084C694603952046FEF7DC
:1024C0007DFC012231462046FEF770FD07B0F0BDCD
:1024D00030380240000402400000024070B5FFF7AF
:1024E000BFFF00224FF480716748FEF75FFD674D24
:1024F0004FF48054002221462846FEF757FD642001
:10250000FEF74AFC012221462846FEF74FFD6420D3
:10251000FEF742FC112000F07FF97820FEF73CFC2A
:10252000362000F079F9002000F08CF93A2000F014
:1025300073F9052000F086F9B22000F06DF90C2047
:1025400000F080F90C2000F07DF9002000F07AF90D
:10255000332000F077F9332000F074F9B72000F051
:102560005BF9352000F06EF9BB2000F055F9192019
:1025700000F068F9C02000F04FF92C2000F062F95B
:10258000C22000F049F9012000F05CF9C32000F0FE
:1025900043F9122000F056F9C42000F03DF9202044
:1025A00000F050F9C62000F037F90F2000F04AF98A
:1025B000D02000F031F9A42000F044F9A12000F06F
:1025C00041F9E02000F028F9D02000F03BF9042088
:1025D00000F038F90D2000F035F9112000F032F943
:1025E000132000F02FF92B2000F02CF93F2000F0F1
:1025F00029F9542000F026F94C2000F023F9182086
:1026000000F020F90D2000F01DF90B2000F01AF960
:102610001F2000F017F9232000F014F9E12000F04A
:10262000FBF8D02000F00EF9042000F00BF90C208C
:1026300000F008F9112000F005F9132000F002F96C
:102640002C2000F0FFF83F2000F0FCF8442000F0C0
:10265000F9F8512000F0F6F82F2000F0F3F81F20D1
:1026600000F0F0F81F2000F0EDF8202000F0EAF86C
:10267000232000F0E7F8212000F0CEF8BDE87040FC
:10268000292000F0C9B80000000002400004024008
:10269000411F5F2909D84FF4967110FB01F06421A6
:1026A000B0FBF1F001490968C8637047A00200203F
:1026B0002DE9FF4F81B00446DDF83C9000904FEAD1
:1026C00059074FF00008780700D0012000EBD70031
:1026D00000FB09FB203AD0B20390029802994844CB
:1026E000401E83B2E019401E82B22046FFF748FE2A
:1026F000002553E0B9F10C0F2AD0B9F1100F2ED0FC
:10270000B9F1180F2ED0B9F1200F49D127490398FC
:1027100001EB8010002610F805A0109800284FF05B
:10272000010000FA06F000EA0A0022D020B120469B
:10273000049A0299FFF76AFE641C0098A4B2201A5A
:10274000B84225D10298009C401C80B2029023E040
:102750000398174900EB400001EB8000DAE71549C8
:10276000039803E00398144900EB400001EB0010CC
:10277000D0E708B1049800E00E9800F03DF808F1A9
:102780000100C0B2B0FBF7F1804607FB118050B1E9
:10279000761CF6B2082EC0D36D1CADB25D45A9D330
:1027A00005B0BDE8F08F4FF00008F5E7349202085D
:1027B00000760208747A0208648002082DE9FE4F50
:1027C0009946DDE90D6714468A460546DDF83080F6
:1027D0000CE0CDF800804B4651462846CDE9016714
:1027E000FFF766FF05EB560085B2641C2278002ACD
:1027F000EFD1BDE8FE8F000008B5010A8DF800108A
:102800008DF801000123022269460248FFF708F90A
:1028100008BD0000E801002070B5094D06464FF4E0
:102820000074002221462846FEF7C0FB304600F027
:1028300009F821462846BDE870400122FEF7B6BBE4
:102840000000024001B501231A4669460148FFF71E
:10285000E7F808BDE80100201CF044F901201DF054
:1028600032F8F9E77FB500241548009401940294EA
:102870001249039401604FF48031C0E901140461EE
:10288000047680F820400F49C0E90A140125C5618B
:10289000C46080F830404561FEF7B2F808B1FDF73A
:1028A000FAFF0520CDE90005694602940448FDF7CA
:1028B000F5FF002801D0FDF7EEFF7FBD00200140AD
:1028C0004C0100200100000F094808B5016841F4DF
:1028D000001101600068002200F400100090052142
:1028E0000F20FEF7F9FCBDE808400F20FEF7E6BC1C
:1028F0003038024010B500F017FC044A00210448AB
:102900001DF048F80349086010BD00008C750208EE
:102910001D2D00080000002070B586B01421684607
:10292000FDF744FE16480024016841F004010160EF
:10293000016801F004010591016841F001010160A5
:10294000016801F001010591016841F00201016097
:1029500000680C4E00F002004FF400550590002274
:1029600029463046FEF722FB01200095CDE90104FF
:10297000694630460394FEF721FA06B070BD0000A8
:1029800030380240000802400D4810B50B49016084
:102990000C49416000214FF480428160C0E903127C
:1029A00041618161C1610162FEF70CFB002803D027
:1029B000BDE81040FDF76FBF10BD0000005400409F
:1029C00094010020A0860100104810B50E49016056
:1029D0004FF482714160002102228160C0E903123C
:1029E000012242615202C0E9062101624162816214
:1029F0000A21C162FEF765FF002803D0BDE8104040
:102A0000FDF749BF10BD000000380040E80100207C
:102A100010B592B000240F941C2108A81094FDF763
:102A2000C5FD20216846FDF7C1FD20481E49016013
:102A30006321C0E901144FF49671C0E903144461A5
:102A40008461FFF71AFB08B1FDF725FF0F940FA96A
:102A500016481094FFF72CF908B1FDF71CFF602011
:102A6000CDE908040A940B940C940D94082208A94B
:102A70000E480E94FFF79BFA08B1FDF70CFF009487
:102A80004FF40050CDE90440029401940394694648
:102A900006480794FFF7E2F808B1FDF7FCFE03488B
:102AA000FFF742FA12B010BD00000140A002002062
:102AB00010B58AB0002407941C2168460894FDF7DD
:102AC00075FD1648144901606321C0E90114FA211B
:102AD000C0E903148461FFF7D0FA08B1FDF7DBFE0B
:102AE000079407A90D480894FFF7E2F808B1FDF72D
:102AF000D2FE6020CDE9000402940C22694607480A
:102B00000494FFF754FA08B1FDF7C5FE0348FFF738
:102B10000BFA0AB010BD000000080040E8020020D7
:102B20000C4810B50A4901604FF4E13141600021C1
:102B300081600C22C160C0E904128161C161FFF7AC
:102B40005AFB002803D0BDE81040FDF7A4BE10BD1D
:102B50000014014030030020FEE7FEE71821014881
:102B6000FDF724BDC003002010B5806B01684A68E2
:102B700022F003024A60416D41F0100141650121DC
:102B800080F85110FEF79CFE10BD10B5806BFFF76A
:102B900062F810BD38B50546846BFEF70DFA0246A3
:102BA00028680068C00523D42068416821F020010E
:102BB00041602068416821F00201416064212046A3
:102BC00000F01AF818B1606D40F020006065A06850
:102BD000002118B92068C26880680090E186012051
:102BE00084F85100606D18B12046FEF769FE38BDCB
:102BF0002046FFF72FF838BDF8B515460E460B46B0
:102C0000009204460122022100F02CF8A0B91348DA
:102C100013490068B0FBF1F04FF47A71484300901B
:102C20006068B0F5827F0DD13346002280212046B6
:102C3000009500F017F870B1606D40F020006065FD
:102C40000320F8BD009830B1401E009020688068D5
:102C5000C0430006F6D50020F8BD00001C0000208F
:102C600000366E012DE9F8431E469146884604461B
:102C7000089DFEF7A1F9401B351AFEF79DF907469E
:102C800025480068C0F3CB30684338E0701C37D06B
:102C9000FEF792F9C01BA84203D215B1009860B3A9
:102CA0002CE02068416821F0E00141606068B0F5E7
:102CB000827F0BD1A068B0F5004F02D0B0F5806FD5
:102CC00004D12068016821F040010160A06AB0F5DC
:102CD000005F09D12068016821F40051016020687B
:102CE000016841F400510160012084F85100002086
:102CF00084F850000320BDE8F8830025401E0090B2
:102D00002068816838EA010004D000214945BDD11E
:102D10000020F0E70121F9E71C000020064D4FF4E8
:102D200000544FF4FA7621462846FEF737F930462C
:102D30001CF0C9FDF7E700000008024010B54FF095
:102D4000E020006924F02AFA012803D0BDE81040F1
:102D500023F038BF10BD000030B593B03021684675
:102D6000FDF724FC14210CA8FDF720FC1C480024CE
:102D7000016841F080510160006800F080501190BE
:102D80001848016841F4404101600068022500F4E0
:102D9000404011900120039010200490009506956A
:102DA0000820CDE907406420CDE9090504200B90F7
:102DB0006846FEF7CFFB08B172B6FEE70F20CDE9FB
:102DC0000C054FF48050CDE90E4003210CA810945F
:102DD000FEF7B4FA002801D072B6FEE713B030BD9A
:102DE00040380240007000400248016841F4700120
:102DF0000160704788ED00E010B50448FEF7FBFF66
:102E0000BDE810400248FEF7F6BF0000A002002017
:102E100078030020F0B50268204B214C9F03214D20
:102E2000214E984207D0B84205D0A04203D0A84214
:102E300001D0B04204D122F0700C4A6842EA0C0280
:102E4000984210D0B8420ED0A0420CD0A8420AD06E
:102E5000B04208D0154CA04205D0154CA04202D07B
:102E6000144CA04203D122F44074CA6822434C6936
:102E700022F08002224302608A68C2620A6882628B
:102E8000984201D109690163012141610169C907C2
:102E900003D0016921F001010161F0BD0000014092
:102EA0000004004000080040000C004000400140C9
:102EB000004401400048014010B501F01F0301210A
:102EC000046A99408C430462016A9A40114301628A
:102ED00010BD000030B5036A026A22F001020262EE
:102EE0004268846924F073050C682C4323F00205C2
:102EF0008B682B430A4DA8420BD123F00805CB6801
:102F000022F440722B434D6923F0040315438A6970
:102F10002A434260846149684163036230BD000016
:102F20000000014030B5026A036A23F01003036217
:102F3000436884690D6824F4E64444EA05248D68F6
:102F400022F0200242EA05120B4DA8420ED1CD68B4
:102F500022F0800242EA05124D6923F4406343EAFD
:102F600085038D6922F0400243EA85034360846152
:102F700049688163026230BD0000014030B5036AD8
:102F8000026A22F4807202624268C46923F4007308
:102F900024F073050C682C438D6843EA05230C4D1F
:102FA000A8420ED1CD6823F4006343EA05234D699E
:102FB00022F4405242EA05128D6923F4806342EA0A
:102FC00005124260C4614968C163036230BD0000FC
:102FD0000000014030B5046A026A22F480520262A5
:102FE0004268C3690D6823F4E64343EA05238D680C
:102FF00024F4005444EA0534064DA84204D14D6936
:1030000022F4804242EA85124260C3614968016449
:10301000046230BD0000014070B5044600680169DB
:10302000E26821F44051114301612169A068E2691D
:1030300008436169114308432168CA6849F20C6377
:103040009A430243CA6020684169A26921F4407131
:103050001143416131492068884202D03049884299
:1030600002D1FEF735FA01E0FEF722FAE269002309
:10307000192164253226B2F5004F626828D0A0FBE2
:103080000101930F9200FDF777F90146B0FBF5F0CF
:103090006FF01802504301EB800006EB0010B0FB0C
:1030A000F5F000F0F002B1FBF5F002EB0012B1FB1D
:1030B000F5F06FF01803584301EB800006EB0010A9
:1030C000B0FBF5F000F00F0021681044886070BD7F
:1030D000A0FB010192185B41FDF74EF90146B0FBE0
:1030E000F5F00201B1FBF5F06FF01803584301EB66
:1030F000800006EBC000B0FBF5F000F0F80002EB3A
:103100004002B1FBF5F0584301EB800006EBC00034
:10311000B0FBF5F000F00700D6E70000001001401A
:1031200000140140FEE7000010B50121002208460E
:103130001CF004FC074C084A0021A06007481CF062
:1031400029FC054A20602432002105481CF022FC9D
:10315000606010BD04000020B0750208CD22000898
:10316000592800080907090E002804DB00F1E020B7
:1031700080F80014704700F00F0000F1E02080F8A4
:10318000141D704770B5044600256FF02F0608E047
:103190002068411C2160007805EB850106EB4101A8
:1031A00045182068007800F02CF80028F0D1284657
:1031B00070BD70B514460D461BB911460CF088FB66
:1031C000034603FB05F0142C0ED0E11F03290AD897
:1031D000072C0DD0082C0DD0092C0DD00A2C0DD0A9
:1031E000002100EB810070BD590801FB050070BD96
:1031F0000221F6E70421F4E71021F2E74FF4807191
:10320000EFE73038092801D80120704700207047C7
:103210002DE9FC5F9B460CAB8A468146DDE91160D7
:1032200093E81210DDE90F575FEA80784FF0300322
:103230001AD45EB15FEAC07808D000F00C0858EAF2
:103240000C0803D0761E01E00B55641CBC4204D26E
:10325000202CF9D301E00B55641C5FEAC07803D041
:10326000B44201D2202CF6D35FEAC06825D55FEACC
:1032700040580AD44CB1BC4201D0B44205D1641EBE
:1032800003D0102D03D1641E04E0102D02D0022DB6
:103290000AD00EE0850603D4202C1ED2782506E045
:1032A000202C1AD2582502E0202C16D262250D556A
:1032B000641C202C11D20B55641C202C0DD2BCF1A7
:1032C000000F01D02D2306E0430701D52B2302E098
:1032D000030702D520230B55641CCDE900BAC8466C
:1032E000154681468B46AA46800714D1274607E03B
:1032F0002A46DDE900316D1C2020C446E0477F1CD2
:10330000B742F5D307E02A466D1C641EDDE90031A3
:103310001BF80400C047002CF5D15FEA897006D481
:1033200009E02A46DDE900316D1C2020C047A5EBED
:103330000A00B042F5D32846BDE8FC9F2DE9F04FC6
:103340008FB099468B46DDE91818DDE91C63DDE98D
:103350001A4792468646002209B923F01003580501
:1033600007AD00D5C9B1B1FBF4F004FB1010C0B239
:103370000A2801D2303009E05FEA836C02D54FF0B1
:10338000410C01E04FF0610C60440A38B1FBF4F1EC
:10339000A854521C09B1202AE5D3CDF80880CDE904
:1033A0000563CDE90052CDE903474B4652465946E5
:1033B0007046FFF72DFF0FB0BDE8F08F2DE9FF4FEE
:1033C0008FB01CACDDE9239594E8030820AC94E8A9
:1033D000C004002450EA010201D125F010056A055D
:1033E0000DF11C0802D550EA010217D032463B46C7
:1033F000FCF7C2FFD2B20A2A01D2303206E0AB0695
:1034000001D5412300E061231A440A3A08F8042058
:10341000641C50EA010201D0202CE7D3CDE90084DE
:10342000CDF808B0CDE90595CDE9036A0FAF97E86F
:103430000F00FFF7EDFE13B0BDE8F08F9A4200D207
:1034400088547047704770B50D46040011D08DB197
:1034500000F067F800280BD0616800690AF0C0FA34
:103460000646E16B28468847E1680844E06030463C
:1034700070BDFEE7FEE72DE9FF4114460E46054606
:103480000A461F4621466846DDF8288008F0D7FF27
:1034900000281AD0019861682268411A009808FB38
:1034A0000151821A551831683844441A684608F0A8
:1034B000B4FF002107E0625C6B5C1A44FF2A00D96C
:1034C000FF226254491C8142F5D3BDE8FF8110B54B
:1034D00002004FF000000CD04B1E194200D0FEE756
:1034E0000A44521E9A43B2F5803F02D20C2A01D9F7
:1034F000104610BD0C2010BD08444A1E401E9043CB
:10350000114200D0FEE7704710B5402013F076FB63
:10351000040005D04022002113F0A1FC204610BD7C
:10352000FEE72DE9FC410D4604002AD055B304F115
:103530002400804618F0FDF9009008B3076961681F
:1035400038460AF04DFA064629463846626813F0B6
:10355000CBFB04F1300013F076FA019098B104220D
:10356000694613F0C1FB2046009906F025F80422B5
:1035700001A913F0B9FB2146304662680AF040FA0F
:1035800007E0FEE7FEE74046009918F09CF90020AE
:1035900000900098BDE8FC812DE9F0410F46012123
:1035A000002504462E46C16309E01A4919F06CFB58
:1035B00008B16D1C02E0E06B401CE063761C57F81C
:1035C000260010B101780029EFD1A06BA8421FD0CE
:1035D000206B002610B110F037FD2663606B10B130
:1035E00010F032FD6663280113F008FB206338B148
:1035F000680013F003FB606318B1216B11B102E0A6
:10360000FEE7FEE700256A00002113F028FCA56311
:10361000BDE8F0812CD5000810B5044690F85400A0
:10362000E26BC107616C04D121B14B1C18D0491E5B
:103630006164A9B90AB1C10712D02146144813F038
:10364000A7FA00F027F8216909B120468847616987
:1036500009B1204688472046BDE8104010F0F4BC70
:10366000216C49426163002A10D0C10702D1A16BCD
:1036700049426163411C61F3000084F85400E16A2F
:10368000606A6162E062206B2263E06310BD00004B
:103690005851002010B50A4C012084F8A40004F110
:1036A000AC0013F0ABF90028D4F8A80003D0BDE8B3
:1036B00010401BF0B1BABDE810401BF09BBA0000EF
:1036C000AC5000202DE9F0413D4D95F8A50038B1F2
:1036D0005FF0000085F8A5003948AC30074664E08B
:1036E0000120F7E7206D1BF02FF9616B0844606340
:1036F0001BF030F92065002085F8A40094F85400F0
:1037000095F8A510C0F340028A4254D061F34100FD
:1037100084F8540041071ED4616B002941DB000787
:1037200009D4A16939B120468847616A01446162C0
:10373000E16A0844E06220461DF032FFE16809B109
:103740002046884794F8540040F0040084F8540060
:1037500020461DF045FE606B002822DB216B88426D
:1037600000DD6163216A20468847A16A0646B142AE
:103770000DD0A662626812B131462068904795F874
:10378000A40088B9A2682AB131462046904795F82E
:10379000A40048B9D4E90C0181420CDB2046FFF7B4
:1037A0003BFF95F8A40030B1384613F027F9040028
:1037B00098D1BDE8F0812146384613F031F9F6E79B
:1037C000AC50002070B5044640680D4608B1FFF7C4
:1037D000F9FF2268002A04D029462046BDE870403F
:1037E000104770BD70B50D6806460C46286838B1A4
:1037F000296AC90204D5206021463046FFF7F2FF4E
:10380000214630462560BDE87040FFF7DBBF08F079
:10381000D3BB08F017BC000010B5416C96B004464D
:1038200001B3684607F0F4FE2146684607F087FFBB
:103830000F49684607F06DFF6846616C07F061FF4D
:1038400001220021684607F074FF0A49684607F024
:1038500062FF0949684607F04DFF684607F090FF90
:1038600016B010BD16B0BDE810401CF0DDBD000064
:10387000AD040208D5B60008AF04020810B504462E
:10388000406882080AD0496821F00301091D0844F4
:103890006060204600F042F8204610BDFEE7406818
:1038A000103120F00300884201D30120704700202E
:1038B00070472DE9FC47054648680C4620F0030098
:1038C00001AA69461BF0DCFDDDE9007005EBC711BC
:1038D00001EB80098046D9F83C0060B164B1C4E9CD
:1038E000020504F10806C46030460421FFF704FE17
:1038F000864202D0FEE7FEE7FEE7C9F83C40012021
:10390000296900FA07F21143296105EB870100FAE2
:1039100008F04A6902434A61BDE8FC8710B50446D5
:1039200000F087F8046010BD2DE9FC4706464FF013
:1039300000000D0000900746019042D00C46E94679
:103940000DF10408802907D3084621F035FF411FF7
:1039500001208840401E04444246494620461BF050
:103960008FFD009C0A2C2CDA06EB8400019A40693A
:103970004FF0FF3101FA02F210400CD1641C3069A3
:10398000A14008401DD021F00FFF0446009006EB37
:103990008000406978B121F007FF034606EBC411AF
:1039A000019001EB8000C76B5FB1786820F00300E5
:1039B000A84201D2FEE7FEE739463046009A1DF0E4
:1039C0004BFD3846BDE8FC8710B50446FFF7A6FF5F
:1039D000416841F002014160606840F001006060B0
:1039E00010BD10B5044600F024F8416821F0020132
:1039F0004160606820F00100606010BD70B506464F
:103A00000D46084600F015F8040010D02079C007D4
:103A10000BD0686880080BD02146304600F03CF897
:103A200021462846FFF72AFF0546284670BDFEE7D7
:103A3000FEE7426800F1080122F00300001F08447D
:103A4000910800D1FEE7704770B506460C004FF0B4
:103A500000001ED0F2B120791546C0071BD01146D8
:103A60002046FFF71CFF78B12946204600F025F8D4
:103A700005462046FFF752FF6868294640F00200DD
:103A800068603046FFF715FF2046FFF7AAFF04F1F4
:103A9000080070BDFEE7FEE77CB5054648680C46A9
:103AA00020F0030001AA69461BF0EAFCDDE90023CF
:103AB000214628461DF0D0FC7CBD2DE9F0410D4685
:103AC000044600F10801281F0E18606806F1080777
:103AD00020F00300401BA0F1040838460421FFF742
:103AE0000BFD874200D0FEE7606820F0030108EB81
:103AF0000500001D814200D0FEE7307900F0030090
:103B000040EA0800706020F003000C2800D2FEE7B5
:103B1000207900F00300284360603046FFF754FF2F
:103B20003046BDE8F08138B5044611F06DFB05461E
:103B300011F0A5FB0028204605D0616C216416F029
:103B400016F8012038BD0FF0D5FD002820461ED004
:103B50000FF080FCD4E9100181420CD06064206C2D
:103B600000906A462021204617F0B1F80128E9D1DB
:103B7000204615F0FCFF284611F090FB0428E0D108
:103B8000204614F046FC002110F0E5FDD9E70FF0C7
:103B90000FFED6E7002802D0C01C20F003007047BB
:103BA00010F052BAC01C13F029B82DE9F0410446B8
:103BB000006815461346476A0E4600222046B8475D
:103BC00001280FD10020BDE8F0812946204600F0F1
:103BD00013F80028F7D020682B460022476A3146A8
:103BE0002046B8470228F0D020682A4631460369AB
:103BF0002046BDE8F041184770B5044600680E46FF
:103C0000026A20469047050010D0206832462946B7
:103C1000436920469847284609F0DDFEA2693146EF
:103C20009047284609F0CEFE012070BD002070BDEF
:103C30002DE9F04F0C4685B00546002114F00DFB30
:103C400058B32146284600F08DFA2146284600F058
:103C500069F80021284615F0F9F983460021284625
:103C600015F042FA04900021284615F0C6F8012804
:103C70001BD000270021284615F0AAFB8046002112
:103C8000284615F03EF96FF040490646C8450ED16A
:103C9000688D00050BD401200AE005B02046BDE880
:103CA000F04F2022002113F0DAB80127E2E70020CC
:103CB0008046284614F06FFB824628460021822267
:103CC00015F03CFAC2B22369A1682068CDE9003141
:103CD000CDE902075B464146504605F0C3FFA061AF
:103CE0004E4504D1688D400501D4012600E0002630
:103CF000284614F03FFB074628460021832215F092
:103D00001DFAC2B2606900256368E1688DE82B0086
:103D100031463846049B05F0A5FFE06105B0BDE8DB
:103D2000F08F00002DE9F34F81B00C46019805F0AB
:103D300024FA06004FF000081ED1019814F0BEFBD3
:103D400005F01BFA070074D0019805F01AFA8146B5
:103D5000019805F01AFA80468500281D12F04EFFE2
:103D600006462A4607EB890112F0BEFF6FF060415C
:103D700046F828104FF00108019814F00CFB834618
:103D8000304600F01DFF2061800012F037FF2060F8
:103D90002069800012F032FF0025DFF82CA1A0601E
:103DA00038E056F82510DFF82491514531D100272D
:103DB0001FE03946019814F050FA4549009015F07B
:103DC000DEFBA8B9009805F0E0F9012810D10098B1
:103DD00005F0D7F9A8420BD1009815F083FB4946AE
:103DE000484501DA084602E0009815F07BFB814661
:103DF0007F1C019814F070FAB842DAD8B9F1000FBC
:103E000003DBA16841F8259003E0A168002041F898
:103E100025006D1C2069A842C3D8DFF8AC900025AE
:103E200009F10109C9F1000352462F4628469A4676
:103E300014E046E056F82010494503DB6B1803EB0D
:103E40000A050AE0914204D1A16851F820100F44FC
:103E500003E0A3680F4443F82010401C216981420D
:103E6000E8D80021019815F0F1F82169C1F10102AB
:103E700000FB02B0C01B00D50020002114E000BFF1
:103E800056F821204A450EDB02EB0A0300FB03F241
:103E900005EBD57702EB670292FBF5F2A768ED1A06
:103EA000801A47F82120491C22698A4201D9002D35
:103EB000E6D1B8F1000F04D03046BDE8FE4F10F057
:103EC000C3B8BDE8FE8F00009AFFFF1F010000E0AD
:103ED000010006002DE9FC5F054614F03FFC834617
:103EE000A86808B10021C1610021284615F0E3F956
:103EF00001900021284615F051F98246284614F019
:103F00003DFF014601982E4C014401EB0A0728466B
:103F100014F0E2F98046002639E0A868DFF8A090A6
:103F20002849006850F82600009015F028FB68BB6F
:103F3000009815F07DFEE0BB0021009814F042FFD0
:103F4000B8B3012836D0022834D0032832D000215B
:103F5000009815F04CFA60B90098143008F04EFA49
:103F6000019900EB01090021009815F003F848447D
:103F700081460021009814F0E2FF4844A04205DB8E
:103F80000021009814F0DBFF00EB0904761C464585
:103F9000C3D3A86810B1CBF10001C1616FF06040DC
:103FA000C44203D004EB0A00B84200DA3846BDE848
:103FB000FC9FFFE70098A969006A401A401CD7E7F8
:103FC000010000E0010004002DE9FE4F054614F059
:103FD000BFFB0290A86808B100218161002128463A
:103FE00015F03AF900900021284615F006F98346AD
:103FF000284614F0D1FE00EB0B010098DFF85C912D
:1040000001EB00084C46284614F066F907460021EB
:10401000284614F0E6FE01284FF0000645D082E065
:10402000A868CA464E49006850F82600019015F06D
:10403000A6FAC8BB019815F0FBFD20B10198E9690B
:104040004069081A14E00021019814F0BBFE58B131
:10405000032809D0062807D0082805D00021019898
:1040600015F0C2F930B112E00199E8694969401AC6
:10407000401C0BE00198143008F0CFF9009900EBD8
:10408000010A0021019814F063FF50448246002188
:10409000019814F05DFF5044A04205DB0021019817
:1040A00014F056FF00EB0A04761CBE42B8D34C4510
:1040B0003FD05C443DE0A868CA462949006850F8F2
:1040C0002600019015F05BFA60BB019815F0B0FD79
:1040D000E0BB0021019814F075FEB8B3012836D07A
:1040E000042834D0072832D00021019815F07CF93B
:1040F00058B90198143008F090F900EB0B0A002130
:10410000019814F02EFF504482460021019814F0CB
:1041100028FF5044A04205DB0021019814F021FF44
:1041200000EB0A04761CBE42C5D34C4501D0009872
:104130000444A86810B10299494281614C45404647
:1041400002D0444500DD2046BDE8FE8FFFE7019820
:104150006969C069401A401CD6E70000010000E010
:10416000010004002DE9F34F81B00C46019805F0E1
:10417000BCFB06004FF000081ED1019814F09EF918
:1041800005F0B3FB070072D0019805F026FC8146CC
:10419000019805F026FC80468500281D12F02EFDB2
:1041A00006462A4607EB890112F09EFD6FF060413A
:1041B00046F828104FF00108304600F001FD60611C
:1041C000800012F01BFD60606069800012F016FD37
:1041D0000025DFF838A1E0603AE056F82500DFF866
:1041E0003091504533D10027DFF828B11FE0394620
:1041F000019814F032F85946009015F0C0F9A8B9AA
:10420000009805F0EEFB012810D1009805F0E5FBC1
:10421000A8420BD1009814F001F94946484501DA4B
:10422000084602E0009814F0F9F881467F1C0198D6
:1042300014F052F8B842DAD8B9F1000F03DBE168A4
:1042400041F8259003E0E168002041F825006D1C4D
:104250006069A842C1D8DFF8B490002509F10109CE
:10426000C9F1000352462F4628469A4614E04AE018
:1042700056F82010494503DB6B1803EB0A050AE0EA
:10428000914204D1E16851F820100F4403E0E36843
:104290000F4443F82010401C61698142E8D8002196
:1042A000019814F021FF8346019814F063F8014649
:1042B0006069C0F101020BFB0210C01B00D5002099
:1042C000002113E056F821204A450EDB02EB0A03D9
:1042D00000FB03F205EBD57702EB670292FBF5F2E8
:1042E000E768ED1A801A47F82120491C62698A4262
:1042F00001D9002DE6D1B8F1000F04D03046BDE859
:10430000FE4F0FF0A1BEBDE8FE8F00009AFFFF1F19
:10431000010000E00100060070B5044600216E2295
:1043200014F00CFFD8B9204600216C2214F006FFCF
:104330004FF48075A84212D1204600216D2214F05E
:10434000FDFEA8420BD120460021712214F0F6FE9A
:1043500028B920460021722214F0F0FE08B1022094
:1043600070BD20460021602214F0E8FEC0B2FF2894
:104370000DD120460021732214F0E0FE38B920460A
:104380000021672214F0DAFE10F0FF00E8D00120CF
:1043900070BD2DE9F041044606A81D46174690E879
:1043A0004C0002290FD003290BD12946384619F0B9
:1043B00061FC0546304608F030F8401B216808448F
:1043C0002060BDE8F0812946384619F053FC0546C7
:1043D000304608F022F800EBD071491005EBD5709B
:1043E000A1EB6000EAE700002DE9FF4F95B0C87827
:1043F000269CC0070D46002801D0FE4800E0FE487C
:10440000099001D0FD4800E0FD480F9001D1FB4824
:1044100000E0FB48109001D0FA4800E0FA48039011
:1044200001D0FA4800E0FA48069001D1F54800E0D2
:10443000F548059001D1F54800E0F5484FF0140922
:10444000049069E0D4E901124FF0000BA1EB0203E4
:10445000584659464FF00C0E0FE000BF01EB4102E9
:10446000266909EBC20C16F80CC05FEACC7C08D0B8
:104470000EEBC202B2589B1A491C8F42EED80021A3
:1044800044E04FF0100C0CEBC202B2581044F3E7BA
:1044900001EB4106276909EBC60A17F80A20D20783
:1044A00033D1E8B34FF0100C93FBF0F20CEBC60CD9
:1044B000CDF848C057F80C804FF0080C08FB02F804
:1044C00004220CEBC60C02EBC60257F80CC0BA581B
:1044D000CDF820C0C44500DDC446624503DC089A1F
:1044E000424500DD4246424504D04FF0010C47F8FA
:1044F0000AC0E346D4F810C00EEBC6064CF80620FE
:104500002769129EBE59801B9B1A491C62698A4208
:10451000BED8BBF1000F02D06769002F92D100E036
:1045200028E00021159814F06EFC012823D000210A
:10453000002088460D900E900EA90DA8CDE900012F
:104540002878E368626824991BF087FAE87810EA13
:10455000080F05D0159813F01EFF0D9908440D9013
:104560001799159813F079FE0646DFF8A8926FF0B8
:10457000704B3AE1FEE70121DAE7A749304614F033
:10458000FEFF00287AD10021304614F0B1FCE8B3D8
:104590000027384661690FE0226900EB400352F8BA
:1045A0003320B24207D100EB40020C20216900EB1E
:1045B000C2000F5802E0401C8142EDD8E878C007E5
:1045C000708D04D020F4806040F4006003E020F49B
:1045D000006040F48060708506F114000F998246F7
:1045E0008847B84224D0304615F0C1FA706911905E
:1045F000B0691290F0691390306A1490099A3946A4
:104600005046904711AA2E21304600E00CE016F0EB
:104610005EFB304613F052FF3246272116F057FB5F
:10462000304615F0A4FA03E0708D20F440607085E8
:104630006878012823D0022804D0059A002130464A
:10464000904727E0109906F1140088472168059AE1
:10465000491C21F00101081A00EBD0704FEA600AF2
:104660000021304690470746049A00213046904783
:10467000381A00EBD0710AEB61000BE0ADE0109945
:1046800006F1140088472168049A0F1A0021304669
:104690009047381A0790E87810EA080F06D00F996B
:1046A00006F1140088470D99081A0D903046002134
:1046B0006A2214F043FD0746304600216B2214F0B5
:1046C0003DFD8246304614F00DFF0C90304613F04D
:1046D000A5FE0146C7F3417001280DD127F0C04067
:1046E000484509DCB0F1805F01DBABEB00000C9AC0
:1046F0005043642290FBF2F7CAF3417001280CD1B9
:104700002AF0C040484508DCB0F1805F01DBABEB2C
:1047100000004843642190FBF1FA71692298401A25
:104720000744B1692398411A01EB0A000190E87827
:10473000C00706D0039A0021304690470D990844DF
:1047400000E0079800EB070AE878C00701D0079857
:1047500005E0039A0021304690470D9908440199DD
:1047600047185AEA070019D0304615F000FA716967
:1047700001EB0A007061F16901EB0A00F061B069B8
:104780003844B061306A38443062304615F0EFF991
:1047900000233A465146304615F092FAE87810EA7E
:1047A000080F14D10F9906F1140088472599039A30
:1047B00008440E9947180021304690470744069A4E
:1047C0000021304690470D993844084404E00E9982
:1047D000259808440D99081A0D90E87817AAC0F397
:1047E0008001159804F060FF0646002E19D0DDE91F
:1047F000170113E0F7C60008EDC600081BC4000847
:10480000FDC300085D8F0108818F01086F8F0108CB
:104810004B8F0108FEFFFF1F0100060088427FF456
:10482000ACAE19B0BDE8F08F2DE9F04F91B00E009D
:1048300005463AD0AE61286808B10FF005FC06EBDA
:104840004601062000EB410012F0D8F9286018B3A9
:10485000022101EB46010144E960042101EB8601DC
:104860000144C5E9010101210024012E15D03001C8
:10487000103012F0E7F9A346B100CDE9051B8246DE
:10488000C1F1010700EBC600891000F108095C4680
:10489000CDF834B0099196E0FEE7B4220270E868E2
:1048A0000480E8684180A868048011B0BDE8F08FFA
:1048B0004FF00008002F05DC0699032000EB4100B3
:1048C000074408E0DDE905010A1A052101EB420170
:1048D000401E0F4405900698401C069005A800F065
:1048E000DAF870B1059809AB82100DA943F82820B9
:1048F00000F0030041F8280008F10108B8F1040FA6
:10490000D8DBB8F1040F64D10C99099888420AD118
:104910004AF8240049F824B0DDE90D010144DDE93D
:104920000F02104418E00A99884218D04AF824006F
:1049300049F824B069680D98085569680001085560
:104940000998641C401E4AF8240049F824B0DDE9A7
:104950000E0101441098001D084469682CE00B9971
:104960004AF82400884249F824B0DDE90D010844E2
:1049700011D0696808556968000108550998641CD8
:10498000401E4AF8240049F824B0DDE90F0108442C
:104990000830696810E00F9908446968085569682B
:1049A000000108550998641C401E4AF8240049F883
:1049B00024B0109869680C300BF1010B0855696838
:1049C00000010855641C05A800F065F800287FF474
:1049D0006FAF0AEB840140F2D320464351F8041C28
:1049E000B012814205D109EB840151F8041C8142C7
:1049F00019D0A6EB8021B1F5007F03DC494341F3D8
:104A0000CF3106E0C1F58061494341F3CF31C1F1B7
:104A10000F014AF8240049F82400686801556868C5
:104A200009010155641CA01E0DE000BF59F82020AB
:104A30004AF824205AF8202049F8242069680A5CA2
:104A40000A55401E641C0028F0DAEB680021084675
:104A500019801AE0EA6822F81100AB683AF82020C1
:104A600023F811200AE0AB685AF8202033F81160CF
:104A7000964200DA324623F81120401C59F82020D3
:104A80008A4201D1A042EEDB491CA042E2DB504643
:104A90000FF0DAFA09E703C8814201DC0120704710
:104AA00000207047012070477CB504460FF03EF8A7
:104AB000064620460FF036F80546304613F0FEFC59
:104AC0000446302D23D00B2D4DD110F09DFB10B19D
:104AD000007A012847D06946304613F051FD94F81A
:104AE000300010F00C0F30461BD013F054FC05467C
:104AF0000021204614F099F90128009805EBD571A2
:104B00000CD000EB610000BF90FBF5F512E0E16A0C
:104B100002B00022BDE8704018F02EBEC0EB61006C
:104B2000F2E713F027FC019900EBD07201EB620170
:104B300091FBF0F5002D00DA0025E06A0026A8427E
:104B400000D0012610F060FB08B1012200E0002235
:104B50002946204618F010FE002E04D00022202105
:104B6000204616F0B4F87CBD30B5002822DA8B1A46
:104B7000002B00DC531A64225343C0F30901B3FB3A
:104B8000F1F1C0F30953C0F38922C0F3095000EBDF
:104B9000800003EB83034000B1EB430F01D20C46CE
:104BA00000E0044602EB8205B4EB450F03D202EBB2
:104BB0008200400030BDB1EB430FFBD2084630BD50
:104BC000014600206FF0604200E0401C51F82030A8
:104BD0009342FAD170471FB5044690F8640000F084
:104BE0000100884225D094F8640011B140F0010022
:104BF00001E020F0010084F8640004F150016846EF
:104C000007F088FBE06A009942691144009101991C
:104C1000806908440190E06A029940690844029062
:104C2000E06A03998069084403906946204614F0BD
:104C3000B9FF1FBD08B50846114609F064FC009095
:104C4000BDF800009DF8021040EA014008BD0000D8
:104C50002DE9FC5F088C0C46C0F307208F6C09F02F
:104C600073FC8146208D636A81B2CA00B2FBF9F001
:104C7000072202EBC002D6081A0C01FB02FA02FB63
:104C800000F599B20E23364800960AF01BFC060088
:104C900007D0206AD6F81080000C000704D5386AC7
:104CA00018E00020BDE8FC9F207C012801D080B1E5
:104CB00015E001A80090534642460C21386804F0E4
:104CC00074F810B90199514509D030460AF03BFCFF
:104CD000E7E7E06852460169404612F005F8208C8B
:104CE000C0F307200E2837D008EB0A00A0F1010B13
:104CF00008EB0500A0F1010A012000FA09F0401EAE
:104D0000002100F0FF0E0B4624E000BF9BF80000DE
:104D10004A46C84010EA0E000FD080460AE000BFA5
:104D2000C2F1080C00FA0CFC4CEA080C4A440CF0E6
:104D3000FF08D2B2082AF3D340468AF8000001EBFC
:104D40000900C1B2082902D30021ABF1010BAAF17D
:104D5000010A5B1CAB42D9D3FE610120E662A1E7E8
:104D6000A45100202DE9FC478F6C086A0E46D7F845
:104D700000A0C0F307254FF48079072D0DD0082D32
:104D80000DD0092D0DD00A2D0DD0002189008846A7
:104D9000C0F3C04048B1386A28E00221F6E7042198
:104DA000F4E71021F2E74946F0E7307C012801D012
:104DB000D8B115E0084611F021FF040009D001A880
:104DC0000090434622460C21504603F0EEFF20B9E6
:104DD00000E0FEE70199414505D020460FF034F987
:104DE0000020BDE8FC877C6001E0F0680469346362
:104DF000072D09D0082D09D0092D09D00A2D09D079
:104E0000002070630120ECE70220FAE70420F8E7B5
:104E10001020F6E74846F4E72DE9F0430024DDE9E9
:104E20000759D617072808D0082810D0092819D004
:104E30000A2821D00020BDE8F08302EB567405EB70
:104E4000E40502F007020120C2F1070416E002EBBC
:104E50009674022005EBA40502F003020624A4EBDD
:104E600042040BE002EBD274042005EB640502F06F
:104E70000102A0EB820401E00820154401228240D7
:104E8000521E1FFA82FC0026C0F1080211E02F78A2
:104E900009EB8608E74007EA0C0701EB8707241AAD
:104EA0003F6864B2C8F80070002C01DA14466D1C2B
:104EB000761C9E42EBDB0120BDE710B10268D2698F
:104EC0001047FEE770B505460EF02CFE0446284656
:104ED0000EF082FE352C07D1D0F8F802002803D05E
:104EE000BDE8704019F098BE70BD000038B50546A9
:104EF0000948007858B10092888983B2088982B243
:104F0000888884B20888214680B2FDF757FA28467F
:104F1000BDE8384009F030BD480100202DE9F041DE
:104F20000446C0690E4610B10020BDE8F0810122A0
:104F3000002130460AF006FE05004FF0FF3716D07C
:104F400030460BF069FA90B10220A86405F13800F0
:104F5000E561C4E90160204603F0E8FBE169032054
:104F600088640020E0610AF08DFD0120DDE738460D
:104F7000DBE7414302EBA121414303EBA121414384
:104F8000881270477CB5044617F020FC94F8A010F6
:104F900004F12C0541F0010184F8A010F8B10128BA
:104FA0001DD002281DD110F02FF9694610F04AF9E2
:104FB00003226946204616F045FA0021204613F0E8
:104FC00028FF01280ED00026204605F02DFE0146C0
:104FD00094F84C000E40B04206D0012205E0C4F81F
:104FE0009C507CBD0126EFE7002204F1380089B314
:104FF000009902B3D4F884209142F0DBE26F914231
:105000003ADC626FE16F009B891A01EBD17102EB10
:105010006102D11A002900DC991AD4F88460D4F80E
:105020008C20921B02EBD27206EB6206F21A002A67
:105030004ADC9A1B48E0D4F88C209142CFDC626FA6
:10504000914219DBDDE700BF44F89C5F207920F036
:10505000020006E007E000BF44F89C0F207940F012
:10506000020020717CBD01994AB1D4F89020914290
:10507000B5DCA26F91420ADAC4F89C007CBDD4F87A
:1050800088209142ABDBD4F880209142F4DCD4F844
:105090008020A16F521A02EBD27201EB62020199D9
:1050A000511A002901DC0199891AD4F89030D4F8FA
:1050B00088209B1A03EBD37302EB6303019A9A1ABD
:1050C000002A01DC019AD21A8A42C5DABCE72DE92E
:1050D000FF4FB7B0154637981F460C468268DDF87B
:1050E0001081469E1DA807F0AAF900287DD01DA8B2
:1050F00007F093F91C9005A82C22002111F0AFFEB7
:105100001C9811F07BFD03900B90002021902290C1
:10511000239001234246294624A80DF017FD24A818
:105120002190002F07DD00233A4621462DA80DF0DF
:105130000DFD2DA8229010A805900D90BDF814012A
:10514000ADF829009DF816018DF82B008DF8286028
:105150002068C1192868814200DD08461890A068BF
:10516000A968C01B884200DB08461A906068C11914
:105170006868814200DD08461990E068C11BE86854
:10518000814200DA08461B9018A807F046F96168CA
:105190006A68914201DC012100E000218946E16852
:1051A000EA68914201DB012100E000218A46216882
:1051B0002A68914201DC012600E00026A168AA6865
:1051C000914201DB012200E00022904606EA08013C
:1051D00001EA09014FF0010B11EA0A0F03D032284E
:1051E00001DA4FF0000B012000E030E18DF83000D3
:1051F00019EA0B0F0CD0189810901A98129060684A
:105200001190686805A9401E139037980CF0F5F8C6
:105210001AEA0B0F0CD0189810901A981290E868A0
:1052200005A9401C1190E068139037980CF0E5F840
:105230002968A868814205DB96B1B8F1000F02D059
:10524000206812E066B120681090286805A9401E09
:105250001290199811901B98139037980CF0CDF874
:10526000B8F1000F0CD0A868401C1090A0681290F4
:10527000199811901B98139005A937980CF0BDF858
:105280001D98BBF1000F109006D018981F9A411E70
:105290008A423EDA10463DE01F98129068686168C5
:1052A000401AB84200DA3846814600252EE0606890
:1052B0004619E068A0EB05081E98B04202DD20996F
:1052C000414522DBFF211C9A039811F0C8FD1C9870
:1052D0000090334621A8109A03990DF01DFB8DF81C
:1052E00030001E98B04205DC119605A91396379838
:1052F0000CF083F82099414507DBCDF8448005A9DF
:10530000CDF84C8037980CF078F86D1C4D45CEDB0D
:1053100092E0401E129010A807F07FF8051E39DDBC
:1053200056EA090019D01E9C14E011942A46FF2168
:105330001394039811F093FD0095234621A8109A29
:1053400003990DF0E9FA8DF8300005A937980CF0B3
:1053500054F8641C1998A042E7DC56EA0A0619D0F2
:105360001B9C13E011942A46FF211394039811F01B
:1053700076FD0095234621A8109A03990DF0CCFAEA
:105380008DF8300005A937980CF037F82098641C88
:10539000A042E7DA12991D98491C884201DD0146B6
:1053A00001E01299491C10911A99491C884201DCAC
:1053B0001A98401C10901F98129010A807F02DF812
:1053C000051E39DD58EA090019D01E9C14E011941D
:1053D0002A46FF211394039811F041FD00952346BE
:1053E00021A8109A03990DF097FA8DF8300005A9BD
:1053F00037980CF002F8641C1998A042E7DC58EAD0
:105400000A0019D01B9C13E011942A46FF21139423
:10541000039811F024FD0095234621A8109A0399C2
:105420000DF07AFA8DF8300005A937980BF0E5FFFA
:105430002098641CA042E7DA24A80DF0ABFA002FF4
:1054400002DD2DA80DF0A6FA03980EF0FDFD3BB08D
:10545000BDE8F08F2DE9FF4794B015460C46824613
:1054600004A82C220021209E11F0F9FCCDF810D0C8
:10547000BDF85C00ADF825009DF85E008DF82700B2
:105480008DF8246060686968884201DC012700E0CB
:105490000027E068E968884201DB012600E0002679
:1054A00020682968884201DC012100E0002189464A
:1054B000A168AA68914201DB012100E0002100906F
:1054C000A06802906068019068688846401E03905A
:1054D0001FB104A950460BF090FFE868401C0190F2
:1054E000E06803901EB104A950460BF086FF2068C7
:1054F00000902868401E02900FB1686800E0606864
:1055000001900EB1E86800E0E0680390B9F1000F87
:1055100003D004A950460BF070FFA868401C00900F
:10552000A0680290B8F1000F03D004A950460BF018
:1055300064FF18B0BDE8F0872DE9F04F8B46A2F567
:105540007F41A1B091460646FF3942D0F46A208DD2
:105550008046984204D02385608D40F00800608525
:105560004FF4802A5146204613F0EAFE0746514682
:10557000204613F009FF054638460EF05AFD07464F
:10558000304603F080FF80697A1909FB020001466A
:1055900005EBD570A1EB60001D9038446D1E2844CA
:1055A0001F90F06A41691C91C0691E9068460BF01B
:1055B000E5FC6A465146204614F04BF91CAA6946A0
:1055C00058460BF0C5FAA4F82880608D20F008003A
:1055D000608521B0BDE8F08F2DE9F04F0E46A2F5B1
:1055E0007F41A5B090460546FF395CD0EC6A278D17
:1055F0009F4204D02385608D40F00800608503A899
:105600000AF07CFC4FF4802903AA4946204614F096
:1056100062F84946204613F0B7FE1190284603F081
:1056200032FF05003FD00B980EF003FD119AA969D7
:10563000131808FB031119911146199A01EBD17146
:10564000A2EB6101119A19911144401E08441B906C
:1056500060691890E0691A9018AA06F118011FA84D
:1056600006F0EDFED0B118360DF17C0C96E80F0077
:105670008046894692469B469CE80F0086E80F00CC
:105680002846183E10F0F0FA0A9005F1140203A91A
:1056900030460AF002FC183686E8000F2785608D38
:1056A00020F00800608525B0BDE8F08F7FB5044686
:1056B000D0F8A85204E000BF0AF0ECF90AF02EF985
:1056C000A86B0028F8D1204609F0E0F918B1264867
:1056D000006921F0DAF901202063A16BC90702D02B
:1056E000A16B890700D400206063606B08B10126BC
:1056F00000E00026A06A20B3286821696A4605698F
:10570000D4F80003084400906169D4F80403084405
:1057100001902169D4F80803084402906169D4F823
:105720000C03084403903A21204609F051FAA36A79
:105730002A466946204698476A463B21204609F09A
:1057400047FA204609F0A2F900280BD094F8390056
:10575000012801D1002E05D0616AE069814200D1A3
:10576000206A60627FBD0000AC50002038B5406800
:105770000C46010C491E83B20022009111462046BE
:105780005B1E06F0AEFF38BD2DE9F047B8B0054608
:105790000EF0CCF9044628460EF0FFF98246E06A86
:1057A00010F062FA054694F86400C00771D004A8AE
:1057B0000BF0E4FB4FF4C02904AA4946204614F03C
:1057C00048F804F15001684606F0A4FDE06A00992B
:1057D000426911440091019980696A460844019028
:1057E000E06A0299406908440290E06A039980697E
:1057F0000844039004A950460BF0AAF949462046F4
:1058000013F073FB06464946204613F04CFC8719FB
:105810004946204613F08FFC4FF000081E4906440D
:10582000CDF8D480CDF8D880206E09682844884708
:105830000246206E411935A811F056FA00985822F8
:10584000384400900198414630440190E06A13F0DA
:1058500075FC054620A80AF051FB20AA49462046BF
:1058600013F039FF9DF83000022805D829462B98FF
:1058700008F05AFE00280CD135A827909DF8CC00DE
:105880006A4640F040008DF8CC0020A950460AF04E
:1058900004FB38B0BDE8F08760E902082DE9F04F5D
:1058A000EDB0054638300E465E9011F039F900280B
:1058B0007ED105F1140206F1180168A806F0BFFDBB
:1058C000002875D0183668AC96E80F008346209102
:1058D000CDE9642394E80F0086E80F003DA8183E48
:1058E0000AF03DFE4FF4C0243DAA2146284613F09D
:1058F0004CFF21A80BF042FB21AA2146284613F0B9
:10590000A8FF2146284613F069FD00EBD070471030
:105910002146284613F062FD00EBD0704FEA600A82
:105920005E9811F084F890E040223DA94EA811F055
:10593000DBF9702221A9684611F0D6F9A089ADF8EB
:105940006401A07B8DF86601A089ADF82100A07BE1
:105950008DF82300A08AC00502D5D4E900010BE030
:10596000A2686FF0004082426BD066AB2846216986
:1059700008F0B8FADDE966016A6902EB0008A86977
:1059800000EB010927B1BAF1000F01D0012000E0BE
:1059900000206690A8EB07005F9008EB070061907D
:1059A000A9EB0A00609009EB0A006290207D00E0FC
:1059B00056E081071CD0C00701D0686900E040466E
:1059C000CDE95509207D800701D5E86900E0404612
:1059D000CDE957090020519003904EA930460AF0B6
:1059E00082FD669820B15FAA694630460BF0B0F898
:1059F000207D10F00C0F1ED0CDF85481207D400783
:105A000001D5A86900E04846CDE95608207D000789
:105A100001D5286A00E04846589001205190039033
:105A20004EA930460AF05FFD669820B15FAA69462C
:105A300030460BF08DF83F98401C3F902398401C57
:105A4000239021465E9810F0EFFF04007FF46CAFC6
:105A5000DDE964232099C6F818B01C3686E80E00EC
:105A60006DB0BDE8F08F2DE9F04F884601F11802C6
:105A7000A5B0044600F114011AA806F0E0FC0028C5
:105A800072D008F1180114AD91E80D00D8F8241077
:105A9000179185E80D001AAE08F1180096E82E005F
:105AA00080E80E0000212046C8F8245013F011FAB7
:105AB00005460021204613F0E4FA28441E900021F8
:105AC000204613F026FB0544204612F064FC139098
:105AD000204612F04FFC129002A80AF040FD02AAE4
:105AE0000021204613F051FE20460021322213F0FF
:105AF00025FB00F0FF090021204613F0EAF9824659
:105B000020460021342213F019FBC6B2204612F0C1
:105B100057FD2390204612F015FEA16EB9B3A1697E
:105B20002944A1EB000B60690990E0690B90B4F87F
:105B30006800002507B2B9F1020F26D9BAF1000FAB
:105B400023DDB00705D50021204613F0E2FA00B9A5
:105B50000125F00719D020460021112213F0EEFA9A
:105B600098B97F1E3FB210E055E0A16E1298491E11
:105B70006843B0FBF1F058440A900C9002A90495D8
:105B800040460AF0B0FC6D1C2DB2BD42EDDBE06E6C
:105B9000C0B361691E98002701442398B9F1020F30
:105BA000A1EB000BA0690A90206A0C90B4F86C007D
:105BB00005B225D9BAF1000F22DD700705D5002105
:105BC000204613F05EFA00B90127300718D52046A9
:105BD0000021132213F0B2FA90B96D1E2DB20FE01E
:105BE0001398E16E7843491EB0FBF1F058440990D8
:105BF0000B9002A9049740460AF075FC7F1C3FB247
:105C0000AF42EDDB14AD08F1180195E81D0081E805
:105C10000D00C8F8244025B0BDE8F08F2DE9F0470D
:105C2000A0B006460DF07EFF054630460DF07EFF23
:105C30000446172D2DD01A2D28D1206C002825D0F0
:105C4000E06B002822D0A06C00281FD0E06C002858
:105C50001CD030460DF0A1FFA16D054601F00300F8
:105C600001287BD0890779D002280FD168460AF035
:105C700045F96A460021204613F02DFDE06A0790A1
:105C800004F11402694628460AF007F920B0BDE87D
:105C9000F08730460DF092FF054600780228F5D0D7
:105CA000A06D4FF00106C143890755D000F00301F4
:105CB000022951D0C0F3840008F069FCF0BB2046F3
:105CC0000021442213F03AFAC0B2FF2844D1606C9C
:105CD000A0BBA06C3102884207D1E06C884204D19D
:105CE000002204F11401686830E007A920460FF093
:105CF00091F8204612F092FB0746204613F0F2FB83
:105D00000146B4F84820B4F84C0092B2009207ABB8
:105D100080B2CDE9010300233A4603A80EF03DFD11
:105D200003996069084403900499A06908440490A9
:105D30000599606908440590069901E00CE00DE0C2
:105D4000A06900220844069003A9686806F097FB42
:105D500010B1206B002899D02E7097E701A809F0A8
:105D6000ADFF01AA0021204613F05BFCD5E90880B5
:105D7000D5E90667814611A920460FF04BF8A06CC3
:105D80000D90E06C0E90606C0C9094F85800C10976
:105D9000BDF8500061F30C30ADF85000B4F8580075
:105DA000010B9DF8510061F303008DF85100206B49
:105DB0001B90E06A0890A269206C1044401E00907D
:105DC0006169E06B0B1816A882465B1E06F089FC21
:105DD000204600210C2213F0B1F91A90B4F85800B3
:105DE000C0F303220A2A10D2A06B0090514604F19E
:105DF0001400636B06F06CF90DF1580C9CE80F0071
:105E00000DF1700C8CE80F0007E00C2A0ED016ACD8
:105E100094E80F001CAC84E80F001CAA01A92846D6
:105E200009F0F8FE183585E8C0032FE705F11801E1
:105E300004F11402084606F002FBD4E90D125046A4
:105E400006F042FCE8691799411A206C091A491CAE
:105E500091FBF0F24243A8691699411AE06B091AC6
:105E6000491C91FBF0F14143504606F02DFC1835DA
:105E70000DF1700C95E80F008CE80F00BDF8500094
:105E8000183D40F40050ADF85000C6E72DE9F04F42
:105E9000ADF5117D05460DF049FE044628460DF08E
:105EA0007CFE8F9001A9204612F086FA002168221C
:105EB000204613F043F9054600216922204613F0DD
:105EC0003DF90246294601A806F0ACFA01A806F001
:105ED000A4FA099001A806F091FA0790D4E90C10F1
:105EE000401A5FEA000801D14FF0010894F87000F1
:105EF0000027C0F3C200012805D0022806D0079968
:105F00000998884201DB012700E00027204606F0BF
:105F1000ABFD12900021204613F0ADF85D900021FA
:105F2000204613F0C9F85C900021204613F0EBF8EE
:105F30005B900021204613F071F8059004F13C00BD
:105F400001A9009006F0CBF9E16B5D986FF00105B7
:105F50000144E163616C5C98091A6164216C5B988F
:105F600001442164A16C0598091AA164009877B1D5
:105F700006F044FA042818DA0798A16900EBD070FB
:105F800005EB600008442064001DA0640DE006F0ED
:105F900044FA042809DA0998616900EBD07005EB2E
:105FA00060000844E063001D6064009806F035FA64
:105FB0000546009806F022FA2FB1A94604F14405DF
:105FC000C548009E05E08146C44804F1400604F13E
:105FD00048050D90E26E501C14D0616E206BA36ECC
:105FE000091A181A01FB09F100FB09F091FBF8F1FD
:105FF00090FBF8F0401A5043C21700EB126001EB1F
:10600000202006E0A16B206B081A00FB09F090FB32
:10601000F8F0E26D8346501C14D0616D206BA36DC7
:10602000091A181A01FB09F100FB09F091FBF8F1BC
:1060300090FBF8F0401A5043C21700EB126001EBDE
:10604000202006E0D4E90B10081A00FB09F090FBB1
:10605000F8F0824620460021272213F06FF8C0B2E4
:106060000FB1012800D0002094F84C10814208D0D4
:1060700030462E4601210546CAF1000ACBF1000B3D
:1060800000E0002147B1326802EB0A002860326864
:1060900002EB0B00306008E02A68A2EB0A00401C0B
:1060A00030602A68A2EB0B002860129840B3206B86
:1060B000404200FB09F090FBF8F097B129B133683A
:1060C0002A46181A3146401C03E0336832462946F6
:1060D00018442B6811E00B6010601FE0136008602B
:1060E0001CE021B12B682A463146184404E02B6895
:1060F0003246181A2946401C33688342EEDDEAE72F
:106100000D9900988847012808DC00221F212046AD
:1061100014F0DDFD0DF5117DBDE8F08F7AA8009932
:1061200006F0DDF822A80AF029FF22AA4FF4003178
:10613000204613F08EFB204600210C2212F0FEFFB9
:10614000054607990998884200DB0846B5EB600FC1
:1061500000DD4510DDF8A480009806F05EF90446E5
:10616000009806F04BF98442009802DA06F055F9DF
:1061700001E006F043F9B8EB600F01DD4FEA60087B
:106180009DF8B700002400F0070017B1022802D0E4
:1061900002E0012800D101242E9800B101245D986D
:1061A00001264FF00009002810DB5C9800280DDB69
:1061B0005B9800280ADB0598002807DBA84505DA6C
:1061C0002A4601A97AA806F05AF998B34E4694B324
:1061D000702222A95EA8FAF7AFF98DF8C0918DF868
:1061E000B3918DF8D0918DF898917AAA5EA98F9885
:1061F0000AF0AEFC8DF8F490702222A93EA8FAF7BE
:106200009BF98DF850910DF5F47A8DF840918DF849
:1062100064919AE80F000DF5FE7A8AE80F00ECB160
:1062200097B101995D9808447F9003995C98081A8A
:10623000819011E000E04CE054F0010049D08DF86D
:10624000D0908DF8E090D5E702995B980844809053
:10625000DDE90410081A8290CDF814917FAA10216C
:106260008F980AF00FF907467FAA3EA90AF070FC42
:1062700083A80AF069FC4EB101AE96E80F008AAE21
:1062800086E82F0083A938460AF026FC4CB17AAC88
:1062900094E80F008AAC84E80F0183A938460AF01D
:1062A0001BFC07A809F00AFD7FAA07A90E978F9883
:1062B0000AF06CF8702222A93EA8FAF73DF98DF891
:1062C00018918DF833917AAA3EA98F980AF040FC74
:1062D00020E77AAA22A9F8E71BC40008FDC300083A
:1062E0002DE9F043BDB005460DF020FC04462846DC
:1062F0000DF053FC81460021204612F08AFD012852
:106300000BD00025204604F08FFC064694F84C1074
:106310003540A94203D0012502E00125F2E700251E
:10632000204616F05EFA074620467EB112F076F857
:10633000804637B1E06A002803DA1DB104E03890E6
:106340000EE00DB1E06BFAE7606CF8E713F0CAF805
:1063500080460FB3E06A00281EDAF5B11FE03990DD
:1063600068460AF00BFE6A464FF44031204613F0AF
:1063700070FA3346424638A9204619F0A7FB04F1CB
:10638000840038A9074605F0BCFF204616F01EFA27
:10639000022806D03A462AE00DB1A06CDFE7206C57
:1063A000DDE7702269461CA810F09EFC3A4669465B
:1063B00048460AF0CDFB2EB115B1606C389004E070
:1063C000E06BFBE7D5B1206C39903346424638A9E3
:1063D000204619F07BFB04F1740038A9044605F04F
:1063E00090FF70221CA9684610F07EFC2246694688
:1063F00048460AF0ADFB3DB0BDE8F083A06CE3E792
:106400002DE9F04FADB004460DF090FB054612F0BB
:1064100055F806460EA809F071FD0EAA0021304677
:1064200013F059F920460DF0B8FB00F118010446AD
:106430000FC98B46CDE90723824604F1180106F106
:10644000140223A82B9105F0FAFF002860D023AF97
:1064500097E80F0004F1180787E80F0027A93046D6
:1064600003F0C3FA68690190A8690290E869039093
:10647000289801AA049010462B9905F0E0FFC8B1B6
:10648000D4E90881F4E906670DF1040C89469CE81B
:106490000F0084E80F002846183C0FF0E5FB15902C
:1064A00005F114020EA9204609F0F7FC04F11800CA
:1064B00080E8C003686901902A980290E869039017
:1064C000286A01AA049010462B9905F0B8FFC8B1BC
:1064D000D4E90881F4E906670DF1040C89469CE8CB
:1064E0000F0084E80F002846183C0FF0BDFB159004
:1064F00005F114020EA9204609F0CFFC04F11800A2
:1065000080E8C003DDE90723C4E90823C4E906AB3A
:106510002DB0BDE8F08F00002DE9F0438BB00646AA
:10652000DDE912981D4617460C46484617F021FC37
:10653000002872D100234A4601A928460DF0A9FC83
:10654000BDF80C00002868D0BDF80A10002964D0FE
:10655000BDF90E303A681A441144491E0792099158
:10656000D5E90312891A7A681144BDF91020091A75
:10657000891A0844401E0A900891002207A8B168B1
:1065800005F0D4FF30B1B1680022E06805F0CEFF1D
:10659000002842D10198002580B39DF81200002107
:1065A000401E082821D20095BDF80C30BDF80A2005
:1065B000A06909F068F9010017D1A06908B108F0D5
:1065C000C2FFBDF80C20BDF80A1001FB02F0402804
:1065D00000D252000E231248009508F073FF01000C
:1065E0000DD0BDF80C00C880A16101A80DF04CFCD5
:1065F000206008B19DF81200207102E000E0FEE783
:10660000257107A8A06001A8002320611A46214631
:106610003046C04701A80DF00EFD0BB0BDE8F08379
:106620008C510020F0B58FB01D4616460C00074671
:106630004CD02079092849D2DFE800F00519194823
:10664000194848481900684608F0C1FDE07D8DF8FA
:106650002800A08AADF82000A07D8DF8220001203E
:10666000099069463846E2680BF0BBF82EE0A36853
:106670000DF12C0C0FCB8CE80F000BA805F0CDFE14
:106680000E2109F025F90B99401E08440D9068462B
:106690002C22002110F0E3FBA08AADF81500A07DAC
:1066A0008DF81700E07D8DF81400206801690691CF
:1066B0000BA908910089694680B20990A0680090F2
:1066C00002208DF81C0038460AF097FE002E09D0F3
:1066D000002D07D00FB02A4631463846BDE8F040BD
:1066E0000BF0FCBD0FB0F0BD2DE9F34F086B0C466D
:1066F000401E431000F00100C518C969606A8FB0E0
:10670000814201DA0A4600E00246009200DD0846B6
:10671000A0F101000290206A6946A0EB05000190FB
:10672000206A184403900F988268084605F087FE97
:10673000002838D0A06B18B1606B08B1012600E0CA
:1067400000262C2104A810F0CAFBCDF810D0A08D93
:10675000ADF8250094F82E008DF8270094F83C0041
:106760006D468DF82400D6B1684605F056FE064603
:10677000039F01980390D4E90D100844009991FB00
:10678000F0F200FB121A304610F038FA4FF0020B0C
:106790000C958DF82CB081460A90019D35E004A936
:1067A0000F980AF02AFE11B0BDE8F08F3246FF21A3
:1067B000484610F054FB002150460B465A4617E05D
:1067C000D4F834C0844506DBACEB000C0FFA8CFC2B
:1067D0006144604408E0D4F83880C444844501DA58
:1067E000002001E009F80130401C8DF82C20491CE4
:1067F000B142E5DB04A90F980AF0FFFD0198401CA7
:1068000001900398401C6D1C0390BD42CEDD4846AC
:106810000DF01AFCC7E700002DE9F34F8A46096A1C
:10682000DAF82800D9B00AF11C040AF124068142E2
:1068300005DA2146684614F0B1FF314604E03146DE
:10684000684614F0ABFF2146DDE90057684614F0B6
:10685000A5FFDDE90046A4EB0508A6EB0709B8F1A2
:10686000000001DCC8F10000B9F1000101DCC9F150
:106870000001884201DD012000E000200190DAF8EB
:10688000301058B1B9F1000001DCC9F1000042013B
:10689000B8F100000DDCC8F100000AE0B8F100001A
:1068A00001DCC8F100004201B9F1000001DCC9F1CE
:1068B000000092FBF0F0924A105C48433F30C01158
:1068C0004FEA600B00F0010202EB0B010691A542BA
:1068D00001DA294600E02146A1EB00010A9101DD21
:1068E000294600E0214601440C91B74201DA3946BD
:1068F00000E03146A1EB00010B9101DD394600E0DB
:10690000314608440D9059980AA98268084605F056
:1069100096FD00287DD014210EA8F9F747FE1EA889
:106920000E902CA80F9001990020002972D0B8F188
:10693000000F13DDA6EB0B01CDE900102346A7EBFA
:106940000B0229461EA80CF06DF806980121304470
:10695000CDE90001069823463A1812E0069923462D
:106960003144CDE90010069829463A181EA80CF0CB
:1069700059F80121A6EB0B002346A7EB0B02CDE94A
:10698000000129462CA80CF04DF89AF83D004FF074
:10699000020BC0061AD4032107EB0800CDE9000161
:1069A000A5EB09033A4629463AA80CF03BF806EB5A
:1069B0000801CDE9001BA4EB09033246214648A893
:1069C0000CF030F83AA8109048A811900AA805F0E9
:1069D00024FD044615F084F807F0ECFF05460AA8EC
:1069E00005F011FDA84203D20AA805F00CFD0546EA
:1069F000A846284610F002F981460D9F0B980D908D
:106A000000254246FF21484610F029FA2C2113A800
:106A100001E071E014E010F062FA0AA91391BAF8EB
:106A20002C20ADF861209AF82E008DF863009AF8BA
:106A30003C008DF86000CDF864901B910B9E3AE00D
:106A4000CDE9006006983A46231829181EA80BF0D5
:106A5000E9FF0120CDE90060A4EB0B033A46A5EB6A
:106A60000B018FE7009409EB05010A9A33460EA843
:106A700008910BF051FF8DF8680018B9214608986D
:106A800010F02DFA25442919414503D20D98401CD8
:106A90000D900FE08DF868B013A959980AF0ADFC7D
:106AA0000D980025401C0B900D904246FF21484652
:106AB00010F0D5F9761CBE42D4DD0D990B988842B2
:106AC00007D0481E0D908DF868B013A959980AF0A8
:106AD00094FC48460DF0B8FA1EA80BF05BFF2CA8FA
:106AE0000BF058FF9AF83D00C00605D43AA80BF009
:106AF00051FF48A80BF04EFF5BB0BDE8F08F0000DF
:106B0000E4E902082DE9F04F8346086B0C46401E6D
:106B1000411000F001004218E06991B0821A084467
:106B200000920290216AA06A814200DA0846019030
:106B3000216AA06A814200DD0846401E0390694632
:106B40000846DBF8082005F07AFC00283BD0A06B53
:106B500018B1606B08B1012600E000262C2104A8C2
:106B600010F0BDF9CDF810D0A08DADF8250094F847
:106B70002E008DF8270094F83C006D468DF8240017
:106B8000EEB1684605F049FC0F90039F0198039011
:106B90000F9810F033F880460A9002200C958DF87B
:106BA0002C00D4E90D10084401994FF0000991FB25
:106BB000F0F200FB12150E464FF0010A25E004A981
:106BC00058460AF01AFC11B0BDE8F08FFF2140468C
:106BD0000F9A10F044F9606BA84202DA8DF82C90FD
:106BE00001E08DF82CA0D4E90D100844A84200DC87
:106BF000002504A958466D1C0AF0FFFB0198401CB3
:106C000001900398401C761C0390BE42DEDD404696
:106C10000DF01AFAD7E72DE9FF4705460CF086FF7D
:106C2000C46A28460CF0B9FFE26A054600F1180173
:106C30006846143205F003FC002834D0D5E90881F9
:106C4000F5E9066789469DE80F0085E80F0094F88E
:106C50004C00183D800628D5A26C206C824208D1D9
:106C6000212329462046FEF767FC20462123A26CFB
:106C700013E0202329462046FEF75EFC2046202311
:106C80002946A26CFEF7A8FC204601232946226C67
:106C9000FEF752FC226C204601232946FEF79CFC9D
:106CA000183585E8C003BDE8FF8720462023294624
:106CB000A26CFEF741FC20462023A26CEDE7000009
:106CC0002DE9F04FF7B005460CF030FF0446806B1D
:106CD00000287DD028460CF060FF7290608D40F057
:106CE0000801618520466CA911F066FB0025278DFF
:106CF0002585608D2E4640F0080161853BA80AF08D
:106D00003DF957A809F0FAF84FF4A0293BAA4946E3
:106D1000204612F09EFD57AA4946204612F0DBFCA1
:106D2000608D002120F0080060852046278512F044
:106D3000EDF975900021204612F073F9749000214E
:106D4000204612F09BF973900021204612F0B7F90B
:106D500082460DE1761CE06A90A150F8260015F0FD
:106D600093FF0028F6D0606B30F81500C1067CD484
:106D70004FF00008C10501D54FF00108400602D5CB
:106D800048F0800012E0206CA84210D1B80601D56E
:106D900048F02008B80701D548F00208780701D567
:106DA00048F00408380702D548F008008046206BF8
:106DB00000EB051103A805F09BFA03996C98049A5F
:106DC000014403916D99114404910599084400E030
:106DD000D6E005906D990698B8F1000F084406902A
:106DE0007ED0A4F82880608D40F0080161850AA853
:106DF0000AF0C4F826A809F081F80AAA49462046F4
:106E000012F027FD26AA4946204612F064FC278589
:106E1000608D20F0080161859DF871000C95C10618
:106E200036D520F01F000F308DF87100636973991B
:106E3000039A19448A4203D120F004008DF87100AE
:106E4000E2690599A2EB0A00814205D19DF8710023
:106E500020F008008DF87100A2697598049910441B
:106E6000814207D19DF8710000E07FE020F0020030
:106E70008DF87100226A74980699101A814207D120
:106E80009DF871004108490061F304008DF871001C
:106E900003A805F0B3FA07905FEA886008D5606B35
:106EA00030F81500400503D504990798081A049096
:106EB00003AA0AA9729809F04BFE2E987190359892
:106EC000709034990191E06A50F826B06CA805F0F2
:106ED000A4FA9DF8E3200199CDE90010029200E0A8
:106EE00051E0DDE97032594608A816F067FE03A8A4
:106EF00005F093FA0899401A039900EBD07001EB62
:106F00006000039003A805F079FA0999401A0499E2
:106F100000EBD07001EB60000490089903980844DE
:106F2000059009990498084406905FEA88600FD597
:106F3000606B30F8150040050AD50798049900EBFE
:106F4000D070A1EB600104910699A1EB600006905E
:106F50009DF8E400CDF8B4B040F040008DF8E400B6
:106F600003AA26A92895729808F097FF6D1C761C35
:106F7000A06BA8423FF6EFAE608D20F00800608560
:106F800077B0BDE8F08F70223BA90AA80FF0ACFEE5
:106F9000542257A926A80FF0A7FE3DE70A000000DB
:106FA0002DE9F04FF9B005460CF0C0FD0446284627
:106FB0000CF0F3FD71900021204611F08DFF054685
:106FC00000211222204612F0B9F8284477900021BF
:106FD0001322204612F0B2F800EB050B03A808F0CC
:106FE0008DFF03AA4FF40031204612F074FB206B92
:106FF00040B1814694F84C00002700F00F000128B2
:1070000007D007E080222DA920460CF043FB2DA8D5
:10701000EFE7012720460021272212F08FF8C0B2A7
:10702000012800D10127606B4FF0000800285CD0D8
:107030000EF0DAF88246022818D04DA9606B0DF0E8
:107040001BFD012822D04FF0FF363546A069691E8E
:107050007390084475906069711E72900844CDF871
:1070600000807490B7B10722779B16E011989DF8C5
:1070700057206FF060418DE80700129B0B9A50A8D3
:10708000616B16F09BFDDDE95065DFE74E9886B237
:10709000050CDBE7CBF10003082272A904F1140010
:1070A00005F016F8BAF1020F49D04DA808F006FE17
:1070B0004FF4003A4DAA5146204612F0B2FA05EBC1
:1070C000D570421006EBD67041105DA814F06BFB32
:1070D00020466E22514612F031F85890606B549061
:1070E00072AA4DA9719808F095FD18A808F006FF3E
:1070F00018AA0021204612F0EEFA26989DF8AB203F
:107100006FF060418DE8070049466FA8279B209AE1
:1071100016F054FD60696F996B900844401E6D90A5
:10712000A06970996C900844401E6E90606B70B1BD
:10713000CDF8008087B1CBF1000308220EE0606B30
:107140000A9072AA03A9719808F0A7FECDE7002360
:107150000922CDF8008001E0779B07226BA904F19A
:10716000140004F0B5FFCDF87C90206B28B99DF891
:10717000AC0040F040008DF8AC006BAA18A97198E3
:1071800008F08BFE79B0BDE8F08F2DE9F04FABB081
:1071900005460CF0CBFC044628460CF0FEFC0546E8
:1071A0001FA9204611F0C4F8204602F076F90646E1
:1071B00003A808F0A3FEE06A0A90606D1390A06D2A
:1071C000149094F85C0000F00700032808D01FA872
:1071D00005F014F9B0F5806F02DB04F13800179068
:1071E0008DF8576003AA0021204612F074FA9DF82A
:1071F00056004FF0010808B98DF85680606C0C906D
:10720000A06C0D900C994FF6FF70814226D00D991D
:10721000814223D04FF480292746582249462046F0
:1072200011F08CFF02464946384613F044FF0090A7
:10723000BDF80000ADF83B009DF802008DF83D0060
:1072400020461C22494611F079FF0090BDF800004D
:10725000ADF83E009DF802008DF8400094F85C0007
:107260006FF0604B00F00700022801D0032817D10F
:107270009DF85600022801D0032811D11199CDE9BB
:10728000001B0296129B0B9A27A8E16A16F096FC47
:107290001FA805F0C2F82799884201DA8DF85680B8
:1072A00005F118021FA919A805F0C9F800287ED019
:1072B00094F85C00400709D1204611F043FA42429D
:1072C00000211FA805F000FA206A229094F85C00C3
:1072D00000F0070002281BD0032819D01FAA03A919
:1072E000284608F0DAFDD5E907800DF1640C8146E7
:1072F0009CE80F0005F1180CD5F824A0AF698CE8C4
:107300000F0094F85C0000F00700032818D051E04B
:10731000D5E907820DF1640C91469CE80F0005F158
:10732000180CD5F824A0AF698CE80F001FAA03A998
:10733000284608F0B2FD05F1180080E88007D2E782
:107340001199CDE9001B0296129B0B9A29A8E16ABC
:1073500016F034FC1FA805F060F82999884212DA6B
:10736000202211460B980CF032FE616D299A00EB39
:107370004000114408441390A06D14901FAA03A963
:10738000284608F08AFD1FA805F038F82A99884297
:1073900010DA606D13900B980CF04BFEA16D2A9AD9
:1073A0001144084414901FAA03A9284600E004E0F1
:1073B00008F073FD183585E880072BB0BDE8F08F25
:1073C0002DE9F043A7B007460CF0ACFB0546384664
:1073D0000CF0ACFB04464FF480261A2D7DD01D2DF9
:1073E0007CD138460CF0D9FB054603A808F086FD91
:1073F00003AA3146204612F06EF922A9204602F077
:10740000F4FA22AA05F1180118A805F018F80028C6
:1074100064D0204602F03EF88146204612F062F821
:10742000064648460EF020FC01461198CDE90006BC
:107430000122029220A8129B0B9A16F0BFFB204655
:1074400010F0ECFF07460021204611F07FFFC268D4
:10745000D9F8181002EBD27201EB6201A26906465C
:1074600007EBD77802EB68000F1A484610F0D6FFFA
:10747000F168401A002802DDB90391FBF0F70B9880
:10748000A26902EB6801C068219A121A7A4301EBE3
:10749000A23100EBD070A1EB60080021204611F072
:1074A0001EFD074620460021122211F047FE064627
:1074B00020460021132211F041FE6169F2191144A6
:1074C000CDE91C18E169081AC01B21991E9008EB30
:1074D00001001F909DF8570001E020E01CE040F003
:1074E000010018358DF8570095E8D1000DF1600CBA
:1074F00080469CE80F0085E80F004846183D0EF0D6
:10750000B3FB0A901CAA03A9284608F0C6FCC5F8DC
:1075100018801C3585E8D00027B0BDE8F0833846D8
:107520000CF03BFB05461CA9204602F05EFA6846BB
:1075300009F024FD6A463146204612F08AF91CAA59
:107540006946284609F004FBE6E72DE9F043C7B099
:1075500005460CF0EBFA044628460CF01EFB81466B
:1075600042A9204610F0E4FE05A809F007FD05AA8F
:107570004FF40031204612F06CF942AA05A94846A2
:1075800009F0E6FA204610F049FF054604F1140020
:1075900004F043FF461BE06A411C05D07043C1174D
:1075A00000EB1160071208E0204611F003FC10F018
:1075B000010F01D0374600E0002720460021272296
:1075C00011F0BCFDC0B2012800D1F71B606900902A
:1075D000A0690190E0690290206A03900098002D54
:1075E0003844009001DD6D1E00E0002528444FF472
:1075F000403702903946204611F04FFD0646394685
:10760000204611F068FD05463946204611F08DFDF3
:1076100080463946204611F010FD01460098019A37
:10762000801B0090029828440290A2EB0800019071
:1076300003980844039023A809F0A0FC23AA394624
:10764000204612F006F96A4623A9484609F080FA56
:1076500047B0BDE8F0832DE9F04FADF5137D054649
:107660000CF064FA044628460CF097FA814600F1C3
:10767000180204F1140105A804F0E1FE00287ED0F0
:1076800009F1180005AE90E80E00D9F82400CDE904
:107690000A12CDE90C3096E82E0009F1180080E8B6
:1076A0000E00204600213022C9F8245011F046FD7A
:1076B0008B900021204611F03BFD90900021204648
:1076C00011F0BEFC91900021204611F0E9FC8F9052
:1076D0000021204611F002FD8E90208D002514908F
:1076E0002585608D40F0080161852FA809F046FCD2
:1076F0004FF4A0262FAA3146204612F0AAF86BA814
:1077000008F0FCFB6BAA3146204611F0E4FF149808
:107710002085608D002620F008012046618511F04B
:107720001DF80146A26990981044411A8B980E9555
:107730000844401ECDE91050204611F009F88D9004
:107740000021204611F06BFB012800D0002082466A
:10775000002092E1A16B51F8280011998C90491CEE
:10776000401E0844119008980F9181427DDCBAF1C7
:10777000000F0BD0E1698E98091A8D9800E08AE11C
:10778000091A8B98081A401E0E9008E061698F98BC
:1077900001448D98091A8B980844401E10900025CA
:1077A00065E1606B4FF0000B50F8260008B190F8CF
:1077B00000B0BAF1000F0AD00E98401E1090E06B96
:1077C000109950F82500081A401C0E9009E01098F6
:1077D000401C0E90E06B0E9950F825000844401EA6
:1077E0001090002718E0616BF01951F82000C0B12B
:1077F0000078C00715D0E9190422E06B02EB810183
:10780000BAF1000F405803D00E99081A0E9002E00A
:107810001099084410907F1CE06A7919401E81423B
:10782000E1D31199069881427CDB0E982B900F983A
:107830002C901098CDE92D019DF8050141070BD53D
:1078400062698F9B2B991A44914205DD409A02EBA5
:10785000D272A1EB62012B9181070DD5A36990999A
:107860002C9A19448A4207DD00E00BE1409901EBB4
:10787000D171A2EB61012C91010710D5E3698E99BA
:107880002D9A591A491E8A4209DA409901F00102DB
:1078900001EBD17102EB61012D9A11442D91C007CA
:1078A00010D0226A91982E99101A401E814209DA4E
:1078B000409800F0010100EBD07001EB60002E99C0
:1078C00008442E90626C0020424554D1216CA9429C
:1078D00051D1218D4A0602D48A0600D520208A077C
:1078E00001D540F002004A0701D540F00400090725
:1078F00001D540F00800F0B32085608D40F008010C
:1079000061854BA809F03AFB16A808F0F7FA4BAAD4
:107910004FF4A021204611F09CFF16AA4FF4A0219D
:10792000204600E092E011F0D6FE14982085608D8C
:1079300020F008016185CDE94D85CDE918852BAA98
:107940004BA9484609F004F9606B50F8260000285E
:107950007CD04FF4A021204611F0A2FB02904FF4FE
:10796000A021204611F0BAFB85904FF4A0212046BB
:1079700011F0DEFB00E033E084904FF4A0212046BC
:1079800011F05EFB0146002000900E9A0298104410
:107990006790109A8598101A69900F9A84981044ED
:1079A00068901198401A6A90CBF340005FEA000B90
:1079B00001D00120009067A804F02FFD009A2499BF
:1079C000CDE900100292606B259B739A50F8261047
:1079D00087A8083116F0F2F8BBF1000F0BD01CE0BD
:1079E00070222FA94BA80FF07FF954226BA916A87B
:1079F0000FF07AF99FE78C980F9A00EBD070889976
:107A000002EB600201EBD1714010A2EB610200EBCE
:107A100061000F99689208446A900EAA05A980A88F
:107A200004F00DFD90B10DF5007B09F118009BE805
:107A30000E1080E80E00C9F824C0606B67AA16A972
:107A400050F8260008301D90484600E00BE008F092
:107A500024FA0DF1140B09F118009BE80E1080E8D0
:107A60000E00C9F824C03E443D44761C6D1CE06AFB
:107A7000A8423FF696AE08F10100216B80464145D1
:107A80003FF668AE0AAD09F1180495E80F0084E8E6
:107A90000700C9F824300DF5137DBDE8F08F2DE9FE
:107AA000F0479AB005460CF041F8044628460CF021
:107AB00074F88246E06A0EF0D7F8007800284FD1BB
:107AC000206B00284CD00078002849D004A808F08A
:107AD00015FA04AA4FF40021204611F0FCFD94F899
:107AE0007000000705D59DF85B0040F001008DF89F
:107AF0005B000021204611F0D6FA81460021204685
:107B000011F0EFFA80460021204611F014FB0746E1
:107B10000021204611F097FA06460021204611F078
:107B2000E4F9054604F11401684604F0F3FB0098FB
:107B300009EB050108440090029808EB0501401A82
:107B40000290019879190844019003987119401A1C
:107B50000390206B0B906A4604A9504608F09DF9EB
:107B60001AB0BDE8F08730B5A5B00C46054620AA8E
:107B70001CA910F0F9FD1CA804F045FC20B920A8B0
:107B800004F041FC00281CD0694628461BF01EF872
:107B9000012816D11CA804F036FC30B10020029058
:107BA0001CAA6946204608F0D3FF20A804F02BFC4D
:107BB000002806D00120029020AA6946204608F03D
:107BC000C7FF25B030BD2DE9F04F884601F11802FE
:107BD000B9B0044600F1140120A804F030FC0028DC
:107BE0006FD008F1180020AE90E80E00D8F82400FD
:107BF00029910190CDE92B2396E82E0008F1180079
:107C000080E80E0000212046C8F8245011F039FA0F
:107C100006460021204611F07CFA8146204610F0ED
:107C2000BAFB2890204610F0A5FB259004F12C000B
:107C30002A900EF0E7FE05460021204611F00FFACB
:107C4000226F2899C2F1010303FB0010B0FBF2FA86
:107C50004FF4A021204611F002FA8346C5F101023B
:107C600002FB0BA0B0FBF5F7012F00DA0127002182
:107C7000204611F02EF90546204610F0A1FC301ADE
:107C800028443490204610F05DFDA9EB0000284404
:107C9000339002A809F072F902AA4FF4A0212046FD
:107CA00011F0D7FD9DF83700099920F007008DF8F5
:107CB0003700FF208DF82800206A00260844319004
:107CC00069E075E02899401EA1EB0A017143B1FB00
:107CD000F0F134980844616900EB01090020CDE916
:107CE00004062A980EF08AFE52E0287CC0074BD189
:107CF00094F87400000701D4E96800E000217A1EBE
:107D00004A443092CDF8B89007EB0B02484602EB9C
:107D10000009209B309A9A4233DB229A904239DC48
:107D20002889ADF82900A87A8DF82B008819216FD1
:107D3000DDF894C0B0FBF1F201FB1201686850F865
:107D40002120287CC0F3001304EB8303586CDB6C08
:107D5000121A02FB0CF2181A92FBF0F0ACEB0002C4
:107D60003398A369104418442F90686850F8210094
:107D70006FF00041884204D02EAA02A9404608F0C4
:107D8000E7FE0498401C049029462A980EF048FE0D
:107D90000500AAD1761C206FB04293D8DDE92B23D1
:107DA00008F118002999019C80E80E00C8F82440C9
:107DB00039B0BDE8F08F2DE9F04F01F11802884687
:107DC00000F11401CDB0044691460F4644A804F0DA
:107DD00036FB00287DD008F1180144AE91E80D0073
:107DE000D8F824100990CDE938219A4696E82E005B
:107DF00008F1180080E80E00C8F82450206F02280F
:107E000067D30021204611F064F805460021204682
:107E100011F037F946190021204611F07AF905448E
:107E2000204610F0B8FA0890204610F0A3FA069009
:107E3000204610F0C5FB61693144081A3D90204688
:107E400010F080FCA1694A462944081A429039463C
:107E500049A804F0F4FA00283BD028A808F07FFBDA
:107E600028AA4FF4A021204611F08FFC0CA809F09D
:107E700085F84FF400350CAA2946204611F0E9FC9C
:107E80002946204611F0AAFA00EBD0704610294688
:107E9000204611F03CF800EBD07041108946349830
:107EA0004E4500DA314600EBD070B1EB600F05DDD6
:107EB0009DF8DD0040F010008DF8DD0034980128B9
:107EC00005D19DF8DD0040F010008DF8DD00216F38
:107ED00000E033E10898814201DB012000E000204E
:107EE000439004F12C0005460B900EF08BFD401ED4
:107EF0002A900E9028460EF09AFD13E1287CC007C8
:107F000006D02A98401E2A900E98401E0E9005E139
:107F10002889ADF8CC00A87A8DF8CE002889ADF874
:107F20005100A87A8DF8530000202B900F9094F800
:107F30007400000701D4E86800E000203A903D9802
:107F40002F9031903A9848906968834651F8200004
:107F5000297CC1F3001104EB81020699536CC01A0D
:107F60004843D16CC91A90FBF1F00699091A42985E
:107F700000270844329003900590A5E031982F9097
:107F800032983090711C2F9A0AEB010082427EDCFD
:107F90000898216F7843491EB0FBF1F13D98069B8C
:107FA000084431903A98226F3844B0FBF2F102FB5A
:107FB000110B696851F82B00297CC1F3001104EB07
:107FC0008102516CD26C401A5843511A90FBF1F067
:107FD000191A42980844329009983199801B401E22
:107FE00081426EDB002F6CD04398A0B3696848983B
:107FF00051F820206FF00040824262D051F82B10DF
:1080000081425ED032990598814200DB0846059096
:108010000398814200DC0846039031992F988842EA
:108020004FD032983B90481E31902F90039830905B
:108030000598329032993098884201D1481C32908C
:1080400028A9404608F04FFA3198401C31903B98DF
:108050000390059035E0FFE72F983099801B3E9004
:108060002F9830444090A1EB09003F9001EB0900AC
:1080700041906868489950F821206FF000418A4289
:108080000CD050F82B106FF00040814200E01FE050
:1080900004D028A940462B9708F025FA8EB1B9F1F3
:1080A000000F0ED06968489851F820106FF000401A
:1080B000814206D0781E0F903EAA0CA9404608F0D7
:1080C00047FD7F1CCDF820B1206FB8423FF656AF78
:1080D0004398E8B9206FB8421AD169686FF0004040
:1080E00051F82B10814213D031983299801B3E9069
:1080F00031987F1E30444090A1EB09003F9001EB86
:1081000009000F9741903EAA0CA9404608F020FDB7
:108110000E98401E0E902A98401E2A9029460B98D1
:108120000EF082FC05007FF4E9AEDDE9383008F19D
:108130001801099A81E80C04C8F824004DB0BDE884
:10814000F08F00002DE9F04F8A4601F11802C9B006
:10815000054600F114013CA804F071F900287DD017
:108160000AF1180133AC91E80D00DAF824103691C9
:1081700084E80D003CAE0AF1180096E81E0080E885
:108180000E0000212846CAF8244010F0A2FE044642
:108190000021284610F075FF06460021284610F001
:1081A000B8FF0746284610F0F6F84190284610F030
:1081B000E1F84090284610F003FA01466869321948
:1081C0001044401A4290284610F0BCFA0146AA69B1
:1081D00038191044401A43901FA808F0C0F91FAA8C
:1081E0004FF4A021284611F0D0FA03A808F0C6FEEB
:1081F0004FF4003403AA2146284611F02AFB2146F9
:10820000284611F0EBF800EBD0704FEA60092146E8
:10821000284610F07CFE00EBD070401080462B9971
:108220004A46C14500DA104601EBD171B0EB610F4F
:1082300005DD9DF8B90040F010008DF8B9002B98CD
:10824000012805D19DF8B90040F010008DF8B90063
:1082500005F12C0037900EF0EAFBE8E0EAE0207C24
:10826000C0077DD12089ADF8A800A07A8DF8AA00BA
:108270002089ADF82D00A07A8DF82F0095F87400B4
:10828000000701D4E66800E0002642982690449654
:1082900028906068B34650F826000A2826D04198F6
:1082A00000902068002350F82670207CC0F3C000A6
:1082B00005EB8000C26D416D38460EF0D7FC429947
:1082C00000230844289040980090217C6068C1F306
:1082D000001105EB810150F82600CA6C496C0EF0C4
:1082E000C5FC4099081A4399084401E05448289075
:1082F0000026299082E028982690299827902A6FB6
:108300000BEB0600B0FBF2F102FB110760686FF0A7
:10831000004150F8270088427ED040990091217C8E
:108320000023C1F3001105EB8101CA6C496C0EF00A
:108330009DFC40990023091A4398084429904198CC
:108340000090217C2068C1F3C00105EB810150F849
:108350002700CA6D496D0EF089FC4299084400E07F
:1083600061E028905EB32699A1EB0900459001EBEE
:10837000090027994790A1EB0800469001EB0800FF
:1083800048906168449851F820206FF00040824284
:1083900014D051F82710814210D01FA950462296C0
:1083A00008F0A1F8B9F1000F08D0B8F1000F05D01E
:1083B00045AA03A95046069608F0CAFB4497286FC1
:1083C000B0421AD1606850F827106FF00040814227
:1083D00013D0289845AAA0EB09004590289803A936
:1083E000484447902998A0EB0800469029980696A3
:1083F00040444890504608F0ABFB761C286FB042D2
:108400003FF679AF219833AF401C21900598401C6E
:10841000059097E84D0000E00FE00AF1180181E8AF
:108420000D00CAF82460214637980EF0FDFA0400CA
:108430007FF415AF49B0BDE8F08F4497DDE7000049
:10844000010000E02DE9F84304460BF06FFB804685
:1084500020460BF0B3FB0646C06C4068B0F5A02F79
:1084600062D130460AF0E8FF054630460AF0DDFFEB
:10847000044655EA040057D0F06C00278668072EA2
:1084800005DB40223146404605F0D4F828B10DB155
:1084900085F820700CB184F828704FF40042314602
:1084A000404605F0C7F820B354B1404616F030FA04
:1084B0000090BDF8000020849DF8020084F822009E
:1084C00075B1662085F82000404616F021FA00902C
:1084D000BDF80000A5F821009DF8020085F82300F2
:1084E000404605F0A5F8B04203D115B1B22085F899
:1084F00020004FF480423146404605F09BF80028AA
:1085000012D0002C10D0FF2084F8280040462034E0
:1085100016F0FEF90090BDF8000020809DF80200E2
:10852000A0706068401C6060BDE8F8832DE9F041F0
:108530000F46040005D004F1300080460EF05EFACC
:1085400011E0FEE7286861680669304605F048FAE0
:1085500005F04AFA18B9A2693946304690472946CB
:1085600040460EF05DFA0500ECD104F1240013F052
:1085700087F940460EF022FA0020E060BDE8F08165
:108580002DE9F041174604002DD069B304F1240011
:10859000804613F0A3F9050027D02E69A269394659
:1085A00030469047E16B30468847E168091AE16040
:1085B0003046616805F014FA07462869E16A084404
:1085C000294650F8046C404613F006FA384605F088
:1085D000F9F9314604F130000EF0DAFA3046BDE820
:1085E000F0410BF031BDFEE7FEE7BDE8F081087910
:1085F000052801D006281ED1C86C826B2ABBC26B2D
:108600001ABBC26A3AB9036B4FF48072934202D12B
:10861000436B934201D0012300E00023826E02B13C
:1086200001221A4211D1008CC0F307201AB10E2882
:108630000BD0142809D091F85100642805D3642088
:1086400081F85100012081F850000020704710B5DA
:108650000446007E400721D42089282820D02928DC
:108660001ED04FF48041206810F082FF002816D001
:10867000208913381F2813D2DFE800F010121212DD
:1086800010101010101010101012121012121210E0
:10869000101010121212121010121000002010BD33
:1086A000012010BD70B504460CF0AEFD40B1207E37
:1086B000810701D5012070BDC00701D0002070BD29
:1086C0002068856805B108350122214628460BF04F
:1086D000C3FA0128F3D1217E8907F0D42146002076
:1086E0000FF0A5FD0128EAD1217E8907E7D40022F9
:1086F000214628460BF0B0FA0546012814D1207E09
:10870000800711D420680FF0D9FE06000CD0204657
:10871000FFF79DFF40B120462660FFF7C3FF0546E7
:10872000012801D1207E8107284670BDC2691179D8
:108730000B292DD2DFE801F02C060A0E1216241E9A
:108740001A212800D16C083209F0C8BDD16C08325A
:1087500009F047B8D16C083209F0B4B8D16C0832CE
:1087600009F0C2BFD16C083209F09EBFD16C08324B
:1087700008F054BCD16C09F0D6BFD16C0AF086BCAD
:10878000D16C083209F0BABFD16C08320AF07CBA59
:10879000704700002DE9FF4F89B00E46DDE916B4A1
:1087A00017460021099810F016FE05460021099889
:1087B00010F0AAFB0146F07882070BD5C3076FF0D3
:1087C000404202D0954202D006E0914206D120F00C
:1087D0000200F070C00701D0714800E07148814686
:1087E000F078C00712D06F484FF0000AC4F804A018
:1087F000C4F808A0C4F814A0C4F800A0C4F80CA0E1
:10880000C4F810A080463946009798E06448EBE72A
:108810000098B84206D04FF40011284610F0A8FE88
:1088200000287DD16049284610F0A9FE00287BD1A0
:108830000021284610F05CFB0690A8B36069401C3C
:108840006061A26802EB0B01A160217EC9075AD0CA
:1088500000EB4000C100206913F004F9079078B1E3
:10886000606900EB4001079800EBC1004FF0000188
:1088700040F8185CF078C007284602D0042201E0D6
:10888000FEE7062210F05AFC616901EB41020799EC
:1088900001EBC20141F8140CF0784FF00001C00761
:1088A000284602D0052201E01EE0072210F046FC17
:1088B0006169079A01EB410102EBC10141F8100C1B
:1088C0006169079A01EB410102EBC101069841F889
:1088D000080C616901EB4102079901EBC20141F803
:1088E00004AC079820610EE0284649468847F17895
:1088F000890704D5A1680A180C998A4225DCA26868
:1089000058441044A06028464146884701462068E4
:10891000814202DD2846414688472060E06801E048
:1089200013E001E0401CE060F078400702D54FF012
:10893000FF3000E0012000994118009105D409980A
:108940000FF08BFC051E7FF463AFA068002802DDEA
:10895000A0EB0B00A060606908B10C9800E0A06873
:108960006060CDB10098B84216D109996A4689680D
:10897000096851F82050F078C0F38001099800F0A0
:1089800093FE4DB128464146884720602846494617
:10899000884760600120E06000980DB0BDE8F08F6E
:1089A000EB94010823840108010006002DE9F04F33
:1089B00093B0044600217D2210F0C0FB9DF81710F3
:1089C000421C62F30001820862F34101C00860F3B7
:1089D00082018DF81710204600217E2210F0AEFB98
:1089E0008DF81400204600217F2210F0A7FB8DF89F
:1089F000150020460021802210F0A0FB8DF8160003
:108A00000021204610F0FFF9012800D00020804608
:108A10009DF817004FF00001C00720460CD010F061
:108A200066FB81469DF817004FF00001C007204605
:108A300005D010F00EFB04E010F00BFBF1E710F096
:108A400056FB07909DF81700C007204602D00FF094
:108A5000A2FC01E00FF08EFC002106900F4620469C
:108A6000102210F06BFB05463946204610F02BFA19
:108A700006463946204610F011FA800700D53544E5
:108A8000A069054420460FF069FE281A00210890CD
:108A90000E462046122210F051FB05463146204674
:108AA00010F011FA07463146204610F0F7F940075A
:108AB00000D53D446069054420460FF049FE281A60
:108AC00011909DF817009DF81660C00701D008AD01
:108AD00000E011AD0021204610F07DFC1290002135
:108AE000204610F011FA83469DF81700C10708D000
:108AF0006FF04042934502D1618D490509D5C10708
:108B000008D112996FF04042914203D1618D09055D
:108B100000D40026B8F1000F08D0C00706D116B166
:108B2000012E02D002E0012600E000260027BA460E
:108B3000109776B39DF81700400703D5A068028D03
:108B4000521E13E0002211E000200F9009A907989F
:108B5000CDE9000105A92046069BFFF71BFE099AF7
:108B600007EB090157180AF1010A0246A068008DB7
:108B7000904201DD002AE7DABAF1000F01D0A7EB3D
:108B800009079DF81700C007204603D00FF0F2FB3D
:108B900002E00AE00FF0FFFB10A9CDE90051014609
:108BA00053463A46304616F058FF9DF817004107E5
:108BB00003D5A1680E8D761E00E00026B8F1000FE7
:108BC00004D0C00702D128683844286009AFA068E3
:108BD000008DB04243DD002E41DB01200F9007984D
:108BE000CDE90007324605A92046069BFFF7D2FDD6
:108BF0008246B8F1000F07D09DF81700C00703D1D7
:108C000028680999401A286006AB93E8070002AB70
:108C1000019283E88300119800905346324605A9DB
:108C20002046FBF7E1FB56460D980BF00DFA0020AD
:108C30000D90B8F1000F03D09DF81700C00708D0C1
:108C400028680999109A014402EB09000844286039
:108C5000BDE7109A296802EB0900081AF7E7129994
:108C60006FF04040814201D0834502D1204611F08F
:108C700083FB00223021204612F029F813B0BDE812
:108C8000F08F2DE9F74F0546007F93464FF0000A1D
:108C9000C00760D14FF00108EC680026C1467CB9DE
:108CA000287FC0F3C000401E304254D1B9F1000FFC
:108CB00051D00199284688474FF000080446C14624
:108CC0000EB9261E47D0B8F1000F06D0214628461F
:108CD0005A4690470446B0423DD04FF00108002C60
:108CE000DED0206810F066F80006D8D427681FE0B0
:108CF0000121384610F03CFCB0B12FB101213846BB
:108D000010F036FC0028CAD1E868A04223D0B0B1E8
:108D1000284600F00DFB0246E8681121006811F0BA
:108D2000D6FF012817D106E038460FF0C7FB0746EB
:108D3000002FDDD1E8E7E868006810F018FF28464A
:108D4000EC6000F0F5FA0246E8681021006811F0C6
:108D5000BEFF012802D05046BDE8FE8FE8680068DB
:108D600010F005FF296909B1284688470120F3E77B
:108D700070B5846C0546002C16D0206820B10BF02D
:108D800085F920680BF060F9E06908B106F0DBFBBB
:108D9000206A08B106F0D7FB60680BF055F9204651
:108DA0000BF052F90020A86470BD2DE9F0411D467A
:108DB000069C164607460CB100202060002238466B
:108DC0000BF0EAFA002807D123462A4631463846F6
:108DD000BDE8F0410BF0F9B9BDE8F08170B501468E
:108DE000C06ACA6C12F0060F1AD0C2F34102022AFE
:108DF00018D0012A13D1D1E90E54AC4201DA04F59E
:108E0000B4744A6B0E6B1346B24201DA03F5B472C6
:108E1000291901EBD17149108E4206DA304470BD38
:108E2000496B00E0096B084470BD8A4201DD1844BB
:108E300070BD084470BD2DE9F34F93B006466946F6
:108E40000FF0BAFA304610F04DFB099030460FF0A3
:108E5000E5FA08900021304610F010F98346002111
:108E6000304610F02CF904460021304610F04EF93F
:108E700005460021304610F0D4F8804600213046E7
:108E800010F038F907460021304610F0E5F807F0F9
:108E9000010107EBD77201EB620100F0010200EB68
:108EA000D07002EB6000401C491C0D2900DB0D2135
:108EB00089460D2800DB0D2082460D2C00DB0D2499
:108EC00027460D2D00DB0D254046B8F10D0F00DBC8
:108ED0000D208046002457E0306B00EB04110EA8F3
:108EE00003F006FA0E98009A594658450EDCBBF17D
:108EF0000D0F00DB0D21511A08440E900F98A84267
:108F00001ADC01980D2D05DA294604E0A2EB0A01CE
:108F10000844F2E70D21401A0F9908440F90099870
:108F20001099C01B801E81420846009924DB08442A
:108F30000D2F07DA394606E001990246A1EB090038
:108F40001044EBE70D21084410900898119AA0EB0B
:108F500008000199801E8242114411DB4046B8F19D
:108F60000D0F00DB0D200844119000220EA814996B
:108F700003F01BFB58B906E0014401EB0A00E3E7EC
:108F800001EB0900F0E7641CB06BA042A4D8B06B01
:108F9000A04201D14FF6FF7415B02046BDE8F08F16
:108FA00010F00F0000D1012070472DE9F0410E466E
:108FB00004002CD066B304F1300080460DF01EFD95
:108FC00058B1006861680569284604F009FD074644
:108FD0002269314628469047D8B1314604F1240031
:108FE00012F07CFC050017D02969E06A084450F8AB
:108FF000046C40460DF002FD0246314640460DF03D
:1090000098FD61682869BDE8F04104F0E9BCFEE71D
:10901000FEE73846BDE8F0810020FBE72DE9F04788
:109020004FF0000805461C4616460F464046C3F85A
:10903000008006E0E96B226851F82010401C1144C2
:109040002160B042F6D3002128460FF0E8FE012847
:10905000284615D00FF07CFB2168081A20600021FB
:10906000284610F01DF8216808442060E96B51F88B
:1090700026100844401EA0600020C4F804801FE0B1
:109080000FF066FB216808442060284610F02AFA99
:1090900081460021284610F021F822680146A9EBFC
:1090A0000200401AA060E96B51F82610401A2060B7
:1090B000E2E7A96B626851F82010401C114461601E
:1090C000B842F6D30021284610F032F8616808440F
:1090D000606028460FF042FB6168081A6060A96B67
:1090E00051F827100844401EE060BDE8F0872DE9E4
:1090F000F05F89469346824600210FF0B9FF05468E
:10910000002150460FF0D5FF8046002150460FF059
:10911000F7FF0446002150460FF07DFF06465046FB
:1091200010F0E0F9411BA1EB080750460FF076F96B
:10913000001B801B8742504605DA10F0D3F9411B13
:10914000A1EB080003E00FF069F9001B801B00EBA6
:10915000D0704010DAF8141042190A44C9F80020FF
:109160000219DAF81810BBF1000F0A44C9F80420FC
:1091700001D0CBF80000BDE8F09F002185220FF060
:10918000DDBF002186220FF0D9BF002187220FF01A
:10919000D5BF032901D2012300E00023C01A03EB4D
:1091A000430301EB8301891EC1EB41110C23B1FB89
:1091B000F3F111446422B0FBF2F2014401EB90019F
:1091C000891A4FF4C872B0FBF2F008440721B0FBD3
:1091D000F1F201FB1200C0B2704710B50446806C7A
:1091E000002804D144200DF02DFD08B1A06410BD6D
:1091F000FEE700002DE9FC47A9B18569002204279C
:10920000688AC0F308030CE0AE6802EB820456F8EB
:10921000240007EB8404345B081A844206D8521CED
:1092200092B29342F0D80020BDE8FC8702EB8204A2
:109230001221AB6801EB84010026595C0627022944
:109240000BD04FF00C0961B1274A08234FF0100CE6
:1092500003290FD0012926D043E007EB8401595A96
:109260003EE009EB840107EB840259589A5A085CE6
:10927000161836E0ADF804000092A8680CEB8401E3
:1092800003EB8408425A50F80810022301A815F095
:1092900021FE30B3A96851F80820801A07EB840238
:1092A0004010895A1CE0ADF804000092A8680CEB4D
:1092B000840103EB8408425A50F80810022301A8E5
:1092C00015F008FE68B1A96807EB840351F808207F
:1092D000801A09EB840240108A58C95A32F81000EB
:1092E0000E183046A0E70000315F02082DE9F0417A
:1092F0000D46044600F0C7F8071E17D0B8690021D4
:109300002E1A384610F01CF80AF093FE054600218C
:10931000384610F039F800EBD07106EB61012844B3
:1093200091FBF0F0E16B814200D8481EBDE8F0816E
:1093300070B50646002528460BE000BF0BF0AEFFD7
:10934000012820460AD00BF06BFFB04200D1254621
:1093500020460BF06BFF0400F0D1284670BD0000E2
:10936000FEB58369806900255B8AC4689B04A06898
:1093700026D4830F14D00123B3EB907F2CD1174850
:1093800026688DE80700A068042320F0404231469B
:1093900001A815F09FFDF8B1801B801061681AE0EC
:1093A0000F4826688DE80700A068022320F040429D
:1093B000314601A815F08EFD70B1801B4010EDE71D
:1093C0006368805C595C39B130B1637B2268491EA7
:1093D00011FB0321401E0D562846FEBDA1AF00081B
:1093E000B5AF00082DE9FC5F0E461D4617468246C4
:1093F0004FF400310FF0F2FC00EBD07044103F1B33
:109400005046FFF7EBFCBAF85C1001EB000909F1DC
:109410005A0000B215F024FD78434FEAE0380FFA05
:1094200089F015F01DFD7843C7134FF440394946C4
:1094300050460FF01DFE8346494650460FF039FE58
:109440000190494650460FF05BFE00904946504659
:109450000FF0E1FD326820444244A2EB0B01091BEE
:10946000296032680199424421441144A96071681D
:10947000CA190099511A091B696071683944084476
:10948000E860BDE8FC9FC06A002802D000210EF011
:10949000E4BE704700210EF0E0BE70B590F85C109D
:1094A0000024C90600D50124054600210FF099FFCC
:1094B0006FF0404188420CD1002128460FF066FD34
:1094C0006FF06041884204D1688D000501D444F0FA
:1094D0000204204670BDB0F5806F01D201207047B4
:1094E000800A70472DE9F04104460F46618D002047
:1094F0000426C1F305120FE0E36806EBC0055B59D3
:10950000DD0108D523F07F43BB4204D1E16851F867
:109510003000BDE8F081401C8242EDD84FF0806001
:1095200000EBB1204FEAB050608510F47C7F41D051
:10953000C0F30510C100E06812F094FAE060C0B317
:10954000608DC0F305156D1E16D06FF00302530039
:10955000E06802EBC50141585FEAC11C0CD48901E7
:109560000AD403EBC50C00EBC50184446D1EDCE995
:10957000000CC1E9000CEBD1E068082100EBC5004C
:109580000DF099FC0C200DF039FBE16841F8350035
:1095900013F0F3FBE26806EBC500115841F080714F
:1095A0001150E26867F317011150E06850F8350078
:1095B000AFE700E0FEE7FEE70969C06A0844001F64
:1095C000704700007FB516460A4690F83B500446A7
:1095D0002946104606F07CF9072D25D0082D25D008
:1095E000092D25D00A2D25D00021626AD268A2EB70
:1095F0008101B1FBF0F4B44200DD34460020134E8B
:109600000090029025460190681E03906A46322120
:10961000306905F0DDFA684602F0F0FEA0420CDD8C
:109620006D1E002DF0DC0AE00221DEE70421DCE7FC
:109630001021DAE74FF48071D7E7002D02DC00201B
:1096400004B070BD0398401CFAE70000AC50002045
:10965000491E01D5401E0C310C2901DB401C0C3980
:1096600001290DD0072091FBF0F200FB121000EB56
:10967000D07121F00101401AC0F11F00C0B2704743
:1096800081070CD16421B0FBF1F201FB120149B951
:109690004FF4C871B0FBF1F201FB120010B10020D1
:1096A0001C30EBE70120FBE7136821B15B1E136060
:1096B0000BD4806805E05B1C13608068018D8B42D1
:1096C00003DA006850F823007047002070472DE946
:1096D000FC4115460E4604460BF096FD0BF0DEFDF0
:1096E00001280AD0032808D04FF6FF7005B1286082
:1096F00006B130600020BDE8FC810BF085FD6946B5
:109700000BF0A0FD4FF0000855B320460FF020F8F5
:1097100000994718002120460FF081FB01280BD04B
:10972000606900213F1A20460FF0BAFC3A1A002067
:109730004146C5F8008010E0002120460FF0CEFC25
:109740000146E069401AC21BF1E7E36B53F8213090
:109750001844824204DB491C2960E36A9942F4D32D
:10976000DEB120460EF0FAFF01990844A169451ABE
:10977000002120460FF0DCFC2A1A00204146C6F8E2
:10978000008007E0A36B53F821301844824204DBC9
:10979000491C3160236B9942F4D30120ABE72DE9DA
:1097A000FF4F81B00546039880081E2800D91F206E
:1097B000012787401FFA81F86FEA080080B2009005
:1097C00095F82A0001F47F09C0F3C00A4FF0FF3674
:1097D00000244FF0040B1CE0E96801EBC400426870
:1097E00092013DD5BAF1000F12D10BEBC40289589A
:1097F000C1F30741090449450AD103685868384252
:1098000006D0DDE90312184613F093FA01282FD091
:10981000641C688DC0F30510A042DDD820E0E96823
:1098200051F8340042683A4219D00BEBC4028A580E
:10983000C2F307410904494511D11FFA82FA009A7F
:109840001AEA020F0BD1B24509DDDDE9031213F06C
:1098500070FA012803D15046C24508D00646641C60
:10986000688DC0F30510A042D9D8002E03DB01207B
:1098700005B0BDE8F08F0020FAE72DE9F04742F38C
:1098800000061D460F4681465408761C15F0E3FA83
:10989000A7EB040800FB08F0C711484615F0E0FAF2
:1098A00000FB08F0C011002F06DD803F39120A1BB3
:1098B000324421442A6005E0803739120A1B2144D2
:1098C000891B2A60A960002806DD80380012011B70
:1098D00031442044696005E080300012011B2044BF
:1098E000801B6960E860BDE8F087002184220FF0EA
:1098F00025BC2DE9FF4F87B00746DDE917BA0D46B5
:1099000009980AF096FB00EB0B0101EB0A000490AA
:10991000FC6A0BEB0A006C43A1460025039053E060
:109920007B6B53F8241079B3FA6B0092002652F83F
:1099300025E04FF0040C401E0FE0A21953F822203E
:1099400072B11278D2070BD005EB0608009A0CEB27
:109950008808761C52F80880C64472198242ECD3FB
:109960000878800711D509980AF063FB00EB0B011A
:1099700004985144814206DD09980AF05AFB00EB35
:109980000B0101EB0A0004901CE0DDE91501014424
:10999000AEEB01001499CDE9001000220292786B21
:1099A00050F82410DDE9092305A8083114F006F960
:1099B0000699039808440499884200DC0846344418
:1099C00035440490641C6D1CF86A00EB0901A14247
:1099D000A6D804980BB0BDE8F08F002189220FF0C3
:1099E000ADBB00218A220FF0A9BB2DE9FF410C4637
:1099F000064600210FF0AAFC05464FF480213046B0
:109A00000FF0A4FC074628460AF013FB054638462B
:109A10000AF00FFB0746002130460FF0BBFC014661
:109A2000781900EBD07001EB600530460EF0F6FCC3
:109A3000B16900EBD07001EB600005EBD571A0EBD4
:109A4000610060602844E060694630460EF0B4FC76
:109A5000009820600298A060BDE8FF81F0B585B055
:109A60000446FFF717FD06001DD04FF48027394646
:109A700020460FF06BFC0546394620460FF078FC77
:109A8000044630460CF0F0F8014600206FF06042CA
:109A9000CDE90002029023462A4603A814F08EF86E
:109AA000039805B0F0BD0020FBE700002DE9F04170
:109AB0001E461446054601F47F07FFF770FE012895
:109AC00029D08D2C02D21848005D05E01748006BA4
:109AD000A0B1A4F18D01405C10F0010F0ED00FB1C8
:109AE000002700E06D68EDB1298D334639432246E9
:109AF0002846FFF754FE01280DD0F3E797B9012C53
:109B000001D0022C0ED128680AE0012C05D0C169D1
:109B100029B101203160BDE8F0818169F8E7006872
:109B20000028F2D10020F6E7D0E80208AC5000206F
:109B30002DE9F04104460D46638D00200422C3F355
:109B400005110AE0E66802EBC007F659B70103D534
:109B500026F07F46AE4202D0401C8142F2D88142BC
:109B600004D0E16801EBC000BDE8F0814FF08060F7
:109B700000EBB3204FEAB050608510F47C7F2FD00B
:109B8000C0F30510C100E06811F06CFFE060608D6B
:109B9000C0F30510401E0DD06FF00702E16802EB24
:109BA000C00601EBC0030E44401ED6E90016C3E90F
:109BB0000016F3D10821E0680DF07DF90C200DF0BE
:109BC0001DF8E168086013F0D8F8E168486840F0D3
:109BD00000704860E16865F317004860E068C3E71B
:109BE000FEE72DE9F041051E05D005F130000646DF
:109BF0000CF01DFF0DE0FEE720686968006903F0C6
:109C0000EFFE074603F0F0FE38B1214630460CF077
:109C10000BFF0400F0D1BDE8F0813846FBE70000FF
:109C200038B50F480D461446D0F8B0014FF0020188
:109C300090F82400C0074FF0120002D011F070FC21
:109C400001E011F08DFC2246294604F0C9FC009089
:109C5000BDF800009DF8021040EA014038BD000048
:109C6000AC5000202DE9F0474FF0000CDDE909640D
:109C7000089DDDF82CA0E1466F1EF1B9052A03D03E
:109C8000062A01D0042A02D10023012D01D000218F
:109C900007E001225FF000019C4456F82180491C36
:109CA000C444A942F8D3ACEB0301072A21D2DFE870
:109CB00002F004070B201B130D00C4F8009018E0FD
:109CC000411A01EBD1710CE0411A0BE0411A91FBF2
:109CD000F7F3C4F800900CE0411A91FBF5F303EBA5
:109CE000D3714910216004E0421A691C92FBF1F320
:109CF000236000210BE000BF54F8212056F821C05A
:109D0000624404EB810C1A44491CCCF80420B9428B
:109D1000F2D304EB850106EB850251F8041C52F8DE
:109D2000042C114422688A1ABAF1000F0DD00021C8
:109D300009E000BF54F8213056F82170C31ADB1B2C
:109D400044F82130491CA942F4D31046BDE8F087FD
:109D50002DE9F0418CB004466946F9F769FF08A87F
:109D6000102200210DF07BF800210E462046122221
:109D70000FF0E4F90546314620460FF0A1F80746FA
:109D8000314620460FF084F8400700D53D440021BD
:109D90002E460F46204610220FF0D0F905463946D0
:109DA00020460FF08DF88046394620460FF070F8B7
:109DB000800700D5454420460EF0CAFC6169314455
:109DC000081A0A9020460EF0C9FCA1692944081A15
:109DD00000250B9007E0006808AA694650F82500A6
:109DE00000F03AFF6D1CA068018DA942F3D80098DD
:109DF0000AF02AF901980AF027F902980AF024F9E2
:109E000003980AF021F9002120460FF0E1FA0546F7
:109E1000002120460FF075F86FF040418D4201D0CF
:109E2000884202D1204610F0A7FA002230212046B5
:109E300010F04DFF0CB0BDE8F0812DE9F04704466D
:109E4000C06A4FF4404103F038F994F93610A08EFF
:109E50000122FFF79EF90546A06B08B300264FF0DC
:109E600002084FF00309AF1D4FF4004A15E0A06B44
:109E7000A28E30F8261091420ED108EB8601425690
:109E800094F936108A4207D109EB860140565246B2
:109E9000C119E06A03F0DAFB761CE06BB042E6D849
:109EA000A08E218E884210D194F9360094F9321098
:109EB00088420AD194F93300AD1D4119E06ABDE82A
:109EC000F0474FF4804203F0C1BBBDE8F08710B506
:109ED00002464B68127A097A40684FF0FF348A4292
:109EE00015D1012A01D05AB10EE0194612F0CCFE6C
:109EF000002809D002DD4FF0010010BD204610BD42
:109F0000984201D0FAD9F6E74FF0000010BDF5D91C
:109F1000F1E770B5C56804461021284605F0B7FB87
:109F200010B1284605F00FFB207A012804D16068A3
:109F3000BDE870400AF088B870BD00002DE9F04F10
:109F40000C46804687B00C2120460CF0C4FF98F8E0
:109F50001060D8F80C7016B93869002824D00AF0BF
:109F600091FFDFF818A15FEA000908F1140B1ED079
:109F7000012E26D18DF80460009700226946DAF898
:109F8000200103F09DFC050013D003F024FD00F137
:109F900008010EC984E80E00446900222946DAF857
:109FA000200103F048FD204607B0BDE8F08F012EE8
:109FB00007D10222394658460AF0BCF808B1002001
:109FC000F2E72F4800900CF019FD13E0286868B103
:109FD000686858B10022114658460AF0DDF92B682E
:109FE0002246414628469847012808D0294600982D
:109FF0000CF016FD0500E9D1012E16D018E02089DD
:10A000000004000CF8D12088C0F30720142808D0E1
:10A0100004F09AFAA18889B24843C01DC008208183
:10A02000EAE7A0880004C00BF9E758460AF02EF8CA
:10A03000B9F1000F1CD0012E1AD1CDB18DF80460FA
:10A04000384612F037FE0595009094E8070002AB01
:10A05000544683E8070000226946DAF8200103F03D
:10A0600054FC010006D00022D4F8200103F0E3FCE8
:10A07000284699E7009809F0E7FFA0E7AC500020D8
:10A08000BC51002010B502460B68127909790068AE
:10A090004FF0FF348A4215D1012A01D05AB10EE0A7
:10A0A000194612F0F1FD002809D002DD4FF0010041
:10A0B00010BD204610BD984201D0FAD9F6E74FF006
:10A0C000000010BDF5D9F1E70179012902D100683E
:10A0D00009F0BABF704700002DE9F04F95B08346F4
:10A0E0001EA8894690E84005B1F84810ADF8181050
:10A0F00099F84A008DF81A00106B0790506B089081
:10A10000244DD06A1C46174660B114B12068A8429D
:10A1100008D1CDE9006806AB49465846D04715B08E
:10A12000BDE8F08F98E80F000DF1080C8CE80F00E7
:10A13000706842423068414202A802F0C5FA04B990
:10A140000DAC25606560A560E560224602A9384631
:10A150000AF084FC054694E80F000DF1240C8CE80D
:10A160000F00D6E9001209A802F0AEFA012DD6D1EF
:10A1700009AA414611A802F062F90028E5D011A908
:10A1800009A8CDE9000106AB3A4649465846D047F2
:10A19000DBE70000010000E02DE9FF4FADB0C86A29
:10A1A000DDE93A970E4638B9316B4FF48070814241
:10A1B00002D1716B814201D0012000E000201A9091
:10A1C000B06E08B1012500E00025D46A2C220021E0
:10A1D0002069169020891FFA80FA2088C0F3072B87
:10A1E00007A80CF03CFE96F84C008DF8300096F86D
:10A1F0004D00CDF824A000F00F008DF844001A980F
:10A20000284357D1BBF10E0F0ED096F84B00BBF18F
:10A21000140F24D002284DD81698CDF82C90CDE9F3
:10A2200007908DF828B03EE02D9849468268684630
:10A2300002F005F900283AD016980D9000200890F9
:10A24000CDE90F9A36F8480FADF83100B0788DF8A7
:10A25000330002208DF83800CDF81C9023E002284E
:10A2600028D8484602F0CAF80546484602F0D5F814
:10A27000169908910D91CDF82C900AFB00F1A08859
:10A28000CDF81C9080B2B1FBF0F00D9900FB0510E9
:10A290000D904FEA5A00CDE90F9002208DF838005A
:10A2A00012208DF8280007A92D9807F0A6F831B0E4
:10A2B000BDE8F08F1A9885434BD096F84B000228E2
:10A2C00047D8002219A8B16E0AF000FC0746012801
:10A2D0002ED1249860B30088C0F307200E2801D047
:10A2E000062825D1249D28690D90288980B21090D8
:10A2F00006F15400044602F090F8002800DA4C46BB
:10A3000068680022010C491E83B20091114602A820
:10A310005B1E02F0E6F9002003460090092202A924
:10A32000204601F0D5FE02A80F9002208DF83800DB
:10A330001698CDF82C90CDE907908DF828B007A994
:10A340002D9807F05AF8012FB1D119A80AF05EFB39
:10A35000ADE797E80F0020AC84E80F0020A8079035
:10A36000484602F05AF81790484602F047F806901F
:10A3700020A802F052F8054620A802F03FF88046D7
:10A380005C46BBF1060F04D196F84B00022800D9B9
:10A3900010241A9838B10F2C0CD0112C0AD0122C82
:10A3A0000AD0062C25D0204604F0EBF81990142C86
:10A3B00007D023E010241DE01424204604F0E1F827
:10A3C000199005EB4500009011F08AFB04F0F2FAB9
:10A3D000870011F085FB04F0D3FA04F0D2F847436C
:10A3E0000098B7FBF0F74046474500DD0746009868
:10A3F0001DE01524204604F0C4F81990204604F00E
:10A40000C0F86843039011F06BFB04F0D3FA8700A7
:10A4100011F066FB04F0B4FA04F0B3F84743039874
:10A42000B7FBF0F74046474500DD07460398784301
:10A430000CF0E4FB1590A8B108908DF82840239803
:10A440001F90781E219926900844239020A80B90F5
:10A45000142C08D00E2C17D0204604F092F8684334
:10A46000099086E1FEE769000991159A05FB07F15D
:10A4700002EB41010D91CDE90F0502208DF8380066
:10A4800012208DF8280074E108990D91CDE90F058F
:10A4900002208DF83800B6F84800ADF8310096F883
:10A4A0004A008DF833000020089062E12098CDE941
:10A4B0001B0122981D9023981E90D9F80400424257
:10A4C000D9F8000041421BA802F0FEF81A9878B1B2
:10A4D000159A3098CDE904B2CDE902600699CDE92C
:10A4E000001ADDE916231BA92D9808F085FC9EE0D3
:10A4F00096F84B0002287CD31BA801F07FFF07468B
:10A50000BBF1060F16D0142C3DD00E2C3AD01C985F
:10A510001B9A199900FB0AF002FB010116984FF0F3
:10A5200000080844149015981999019005FB01F052
:10A5300003907AE0DDE91B120AFB021116984FF036
:10A54000000E01444FF0FF08159A19E0002010E0BA
:10A5500002EB800311F800C083F802C011F800C0BC
:10A5600083F801C011F800C002F820C083F803800E
:10A57000401CA842ECDB02EB850251440EF1010EB7
:10A58000BE45E3DB53E04FEA5A011C980191484372
:10A5900016991C9A01EB40011B984FF0000801EB43
:10A5A00040010291019901FB02020698414316986D
:10A5B00000EB410010440590159803900D9804900D
:10A5C000680027901EE000BFDDE90210279A0CF01A
:10A5D0008BFBDDE904012A460CF086FBDDE9011066
:10A5E00000EB4100029005990198084405900398FA
:10A5F00000E084E000EB45000390049808F10108B6
:10A6000028440490B845DFDB11E0039A14990198BF
:10A610000CF06AFB0199199808F1010805FB00107C
:10A620001499019001EB0A001490B845EDDB96F8FF
:10A630004B00022863D9B16C8046C0F1FF0701913D
:10A64000142C1ED0122C1CD00E2C7AD020A801F075
:10A65000DAFE01460198C2B212FB08F3C0F30722EA
:10A6600012FB08F003900198C0F3074212FB08F2B6
:10A67000DDF864C0002001FB0CF1DDF854E0059129
:10A680005DE0C1F3C40111FB08F014900198C0F320
:10A690000720810811FB08F005900198C0F30740DE
:10A6A000C10811FB08F001901598009020A801F056
:10A6B000AAFE864600204FF4FC621EE0DDE900138E
:10A6C00031F810804FEAD82111FB07314FF478435D
:10A6D00003EAC10C059BC8F3451111FB073102EADF
:10A6E000D1018C44149B08F01F0111FB0731009B22
:10A6F0000CEB112123F81010401C7045DEDB20E02C
:10A700001EF8001011FB07314FEA112C0EF800C0A3
:10A710000EEB0001DDF80CC091F8018018FB07CCAE
:10A720004FEA1C2C81F801C091F802C01CFB072CD9
:10A730004FEA1C2C81F802C01999084405998142FE
:10A74000DED807A92D9806F058FE2398401C2190CA
:10A75000269908441F99239088420ADD2391142CDE
:10A7600007D120A801F04AFE1599684301EB40008B
:10A770000D9021991F9881427FF798AE159809F0A6
:10A7800063FC94E52DE9F0410446807A0D4640F0E3
:10A790000200A0721E480026016DA14200D146654C
:10A7A0002078012801D002282FD115B1606FA8426E
:10A7B00001D1666715B1A06EA8420DD1A76E57B141
:10A7C000224614213846A66610F081FA3A46142132
:10A7D00020460AF08BFD15B1E06EA84201D1E66675
:10A7E00015B1206FA8420CD1206F48B12246142128
:10A7F000266710F06CFA3246142120460AF076FDE6
:10A8000015B1A06FA84200D1A667BDE8F081000095
:10A81000AC5000202DE9F041044690F83C0000F0D7
:10A82000030001283CD1E16AA06BB1FBF0F0216B81
:10A83000B1FBF0F200FB1211A26B520802FB0011F7
:10A84000B1FBF0F2216300FB1211A26B520802FB74
:10A8500000116163204600210EF078FD05460021BD
:10A8600020460EF097FD0746284609F0E2FB054614
:10A8700020460DF07FFD06462046FEF70BFE024601
:10A88000216BE819414306EBD67305EBD570BDE8A3
:10A89000F0415B10A3EB6000411A104610F0F5BBCD
:10A8A000BDE8F08110B504460069B0B1A069A8B157
:10A8B0006068A0B103F09CF8021D04F12400216936
:10A8C00011F023F8002807D0042104F130000CF027
:10A8D000B2F80348E063012010BDFEE7FEE7FEE7A3
:10A8E000A54A000810B504460069B0B1A069A8B136
:10A8F0006068A0B103F07CF8021D04F12400216916
:10A9000011F003F8002807D0042104F130000CF006
:10A9100092F80348E063012010BDFEE7FEE7FEE782
:10A92000A32F020870B50D4C064600200D460A46BE
:10A9300020602121304610F0CAF9206858B1017812
:10A9400039B1294612F0A0F928B13046216813F038
:10A95000D9FB002070BD012070BD0000A0000020C8
:10A960002DE9F0418CB01F4614460D4606460FF007
:10A9700077F9002839D0A54237D04FF4B47085421A
:10A9800001DDA5F5B475844201DDA4F5B474F16A66
:10A990000D440C44854201DDA5F5B475844201DD0A
:10A9A000A4F5B4740AAA04A93046FEF7A0FB394600
:10A9B00030460EF013FA80463046394651220EF0EA
:10A9C000BDFB06A908B1012200E00022CDE9004844
:10A9D000CDE902210A982B4682B2DDE9040104F098
:10A9E00041FA06A930460FF0DDF80CB0BDE8F08161
:10A9F00010B588B0044606AA04A9FEF778FB6B469A
:10AA000004A92046069AFEF7EDFC204600F0DCFA89
:10AA1000011E03DD0246684601F004FD694620463A
:10AA20000FF0C0F808B010BDF0B50646A1F57F40A4
:10AA30008DB00F46FF384DD0B06BB8424AD9306B5D
:10AA400000EB071102A801F053FC06A930460DF0F7
:10AA5000B3FC002130460EF04DFB04460021304689
:10AA60000EF0FAFA054630460DF0ACFC03F098FF04
:10AA70000A2190FBF1F2A24201DB90FBF1F490FB82
:10AA8000F1F2AA4201DB90FBF1F506980299021B54
:10AA900011440291079A0399521B1144039104999E
:10AAA00008442044049007990598084428440590D8
:10AAB000306CB8420AD1706B30F81700400505D5EC
:10AAC00002A801F09BFC0399081A039002A93046E2
:10AAD0000FF068F80DB0F0BD2DE9FF470446006F98
:10AAE0000D46A84274D920460DF055FC80462046FC
:10AAF0000DF066FD064694F87400010705D500F0D8
:10AB00000700012807D0022863D004B02046BDE822
:10AB1000F0470FF02CB8002120460EF0DAF9074676
:10AB2000002120460EF0ADFA616938440844A0EBDC
:10AB3000060920464FF4A02148220EF0FFFA0646EF
:10AB40004FF4003120460EF049FC07466069009042
:10AB5000A0690190E0690290206A03900199F019C0
:10AB6000091A0191039908440390206F401EA842DE
:10AB700016D908FB05F1B1FBF0F202EB0901891BC4
:10AB8000C91B6A1C009108FB02F1B1FBF0F101EB5B
:10AB90000900304438440290694620460FF002F81C
:10ABA000002D3FD0681E08FB00F1206F401EB1FB56
:10ABB000F0F202EB0901891BC91B009108FB05F1AA
:10ABC000B1FBF0F101EB090030443844029025E07C
:10ABD00028E0002120460EF042FA8146206F08EB63
:10ABE0000901B1FBF0F7002120460EF072F9824610
:10ABF00007FB05F8002120460EF043FA6169504436
:10AC000041444518694620460DF0D6FBA81B00902C
:10AC1000384400990290A1EB090000906946204653
:10AC20000EF0C0FFBDE8FF8770B505460EF05AFC78
:10AC3000044628460DF0F2FB844201DB012070BD82
:10AC4000002070BD28B10A2803D00D2801D00020B3
:10AC500070470120704700002DE9F74F0D4686B080
:10AC60000446CD490EF08BFC00287CD12046FEF72F
:10AC70008CFA82462046FEF7B4FE5FEA000972D0E5
:10AC8000BAF1000F6FD02046FEF77BFA0746204648
:10AC9000FEF7A3FE80462046002188220EF04EFAE1
:10ACA000C6B2204600218B220EF048FAC0B20390B3
:10ACB000296807EB0A006FF0030303EB8000D5F867
:10ACC00008C051F8272009585CF800000844A0EBA0
:10ACD000020B6A6808EB090003EB8000EB6852F88E
:10ACE0002810125818581044401A0290002120468B
:10ACF0000EF083F8012806D116B1022E02D002E030
:10AD0000022600E0002604F11400019001F085FB0A
:10AD10000090019801F072FB8246012E38D0022E7D
:10AD20004FD0032E4FF00001204606D00EF013F94D
:10AD3000296851F82710084451E00EF00CF92968F1
:10AD400051F8271000EB0109002120460EF003F90D
:10AD50000646002120460EF007F93044ABEB000018
:10AD60000090608D00E014E140F40060608503987D
:10AD700001287CD002287BD003284FF00001204618
:10AD800032D00EF0FAF86A6852F828104718B8E086
:10AD900000992046ABEB010900210EF0DCF80646D5
:10ADA000002120460EF0E0F82968301A00EBD07040
:10ADB00051F8272009EBD971491001EB60001044CC
:10ADC0000DE020460EF08EFB296851F8272002EB9B
:10ADD0000B010E1A002120460EF0C6F8301A8146EB
:10ADE000608D20F40060C1E70EF0C7F86A6852F881
:10ADF00028104718002120460EF0BFF80546002114
:10AE000020460EF09FF802992844A1EB000A608DBD
:10AE100040F48060608520460EF064FB0099884213
:10AE200004D120460DF0FAFA504524D06069029012
:10AE3000A0690390E0690490206A059020460EF016
:10AE400096FEDDE9001001F056FC5146019801F034
:10AE50004DFC20460EF08BFE02AA2E2120460FF05C
:10AE600036FF20460DF02AFB2246272101E021E093
:10AE700039E00FF02CFF204600216A220EF05EF927
:10AE80000646204600216B220EF058F90546204662
:10AE90000EF028FB824620460DF0C0FA3F4A0146DC
:10AEA000C6F3417053104FF080584FF0640C0128E6
:10AEB0002BD035E002980021A0EB0A0620460EF0C8
:10AEC0005CF80746002120460EF03CF86A68381A04
:10AED00000EBD07052F8281006EBD672521002EB3D
:10AEE00060000F180DE020460DF098FA6A6802998C
:10AEF00052F8282011440D1A002120460EF022F8A5
:10AF00002F1A608D20F4806084E726F0C0409042C4
:10AF100006DC404500DB181A00FB0AF090FBFCF64B
:10AF2000C5F34170012809D125F0C040904205DCED
:10AF3000404500DB181A484390FBFCF5089A09EBE2
:10AF4000060178199268114462698D1A0899C968D6
:10AF50000844A169461A55EA06001AD020460EF0A8
:10AF600006FE606928446061E0692844E061A069E8
:10AF70003044A061206A3044206220460EF0F7FD84
:10AF800009B0324629462046BDE8F04F00230EF0B6
:10AF900097BE09B0BDE8F08F01000600FEFFFF1F5D
:10AFA0000A880368934201D0981A7047406849881C
:10AFB000401A70470A780368934201D0981A704784
:10AFC00040684978401A70472DE9F0414FF4403607
:10AFD00004463C2231460EF0B1F805462046422296
:10AFE00031460EF0ABF80544314620460EF0C1F86C
:10AFF00000283146204602DD0EF0BBF802E00EF0DC
:10B00000B8F840420544314620460EF0B8F8002812
:10B010003146204602DD0EF0B2F802E00EF0AFF845
:10B02000404205442046382231460EF087F8074654
:10B0300020463B2231460EF081F83844854200DD3F
:10B040002846BDE8F08170B5054608F06BFD044662
:10B05000284608F06BFD06460DF030FA05462F2C09
:10B0600001D02E2C0BD1002130460BF0C3F928461D
:10B0700015F070FC2846BDE8704017F095BF70BD14
:10B080002DE9F0438DB007461D4616468946084611
:10B09000DDF850800DF0B8F90446414648460DF001
:10B0A0008BF922461146404601F0BCF907F118041D
:10B0B000022E05D0012E32D000200DB0BDE8F08365
:10B0C00098E80E00D8F80C0003908DE80E000022DE
:10B0D000694648460EF08EF96A46214604A801F0FA
:10B0E000AEF90028E9D004AC94E80F0008AC84E87D
:10B0F0000F00022208A948460EF07CF908A9424632
:10B10000084601F09CF90028D7D094E80F0085E8A4
:10B110000F0005221146284601F084F90AE0424654
:10B120002146684601F08BF90028C6D09DE80F0043
:10B1300085E80F000120C0E7F8B504460E46001D63
:10B1400001F05CF90546201D01F067F90096024602
:10B15000217D2B46206804F096FB002800D1FEE7F5
:10B16000F8BD70B504460DF0B7F80646002506E0B8
:10B17000A068006850F82500FFF7F3FF6D1CB5428A
:10B18000F6D3608DC1070CD020F001006085204609
:10B190000FF0F2F820460FF01BF816B120460BF026
:10B1A000A7F9608D810708D520F002006085204650
:10B1B000BDE8704000210EF072BE70BD2DE9F04771
:10B1C0008046089D1F46A86A00FB01F39B120028D9
:10B1D00007DD934207DD00BF95F8340080070DD4EA
:10B1E0008BE09342F8DBCB1943439B12002808DD28
:10B1F000934239DA95F8340080077ED40120BDE807
:10B20000F0879342F6DC686A521C504340F3950085
:10B210000312C0B2FF22002828D000BF2E6BC0F15D
:10B22000FF0404FB06F4A2EB242600BFA3EB0104F9
:10B23000A14636D0002C15DBBC4213DAC0F1FF006A
:10B24000C6F1FF014843A2EB6020C1B295F834007B
:10B25000800701D5C1F1FF0118F8040014F026F9A8
:10B2600008F80400641C1CE0686ACEE74FF0FF0693
:10B27000DCE7002C10DBBC420EDAA6EB6000C1B2AA
:10B2800095F83400800701D5C1F1FF0118F80400DA
:10B2900014F00CF908F80400286B641C361ABC4240
:10B2A00002DA286BB042E4DBBC4218DA002C16DB71
:10B2B000686A704380127043C0F34721A86A00286F
:10B2C00001DAC1F1FF0195F83400800701D5C1F121
:10B2D000FF0118F8040014F0E9F808F8040095F8E4
:10B2E0003400800707D54946B94506DC00290DDB47
:10B2F000404609E001E0641C01D500207FE7BC4224
:10B3000004DC391B08EB04000BF0EDFD022076E7AE
:10B310002DE9F05F06460A9F8A461D46786A00FBC3
:10B3200002F18C12002800DD641C97F8343054457B
:10B3300002DA980707D4D5E08C120AEB050CA44575
:10B3400002DA98077ED483E0521C424341F3950110
:10B3500042F395044FEA2129221204F0FF08C9B2F2
:10B36000A9EB0A04914505D0002803DA11B9FF21A1
:10B370009146641E914528D1002C0CDBAC420ADAC0
:10B3800001EB08004108980701D5C1F1FF01305DCC
:10B3900014F08CF8305597F83400641C800706D5FB
:10B3A000A9EB0A01A9424DDA8EE030460AE0AC4230
:10B3B00000DD2C46002C45D006DD00BFA5EB0401C6
:10B3C00006EB04000BF08FFD89E04FF0FF0B002827
:10B3D00044DAB86A404248434FEAA028002C0DDB0B
:10B3E000AC420BDA08FB01F0C0F34721980701D506
:10B3F000C1F1FF01305D14F059F83055796AA8F1B8
:10B40000FF0041438812641E11D4AC420FDAC8F128
:10B41000FF014143ABEB6120C1B297F834008007D4
:10B4200001D5C1F1FF01305D14F040F8305597F8B7
:10B430003400A41C800709D5A9EB0A01491EA942C2
:10B440004DDC00E04EE00029AFDC48E0AC4202DD1C
:10B450000120BDE8F09F002CB0DA40E0C1F1FF0010
:10B46000B96A41434FEAA128002C0EDBAC420CDA4A
:10B4700000FB08F0ABEB6020C1B2980701D5C1F129
:10B48000FF01305D14F012F83055796AC8F1FF0001
:10B4900041438912641C0ED4AC420CDA4843C0F319
:10B4A000472197F83400800701D5C1F1FF01305DD5
:10B4B00013F0FCFF305597F83400641C800707D563
:10B4C000A9EB0A01A9420DDC0029BFF66EAF06E028
:10B4D000AC4200DD2C46002C04D03FF76FAF4FF09C
:10B4E0000200B6E74FF00000B3E7FEB5C46A09F00A
:10B4F0008BFE054609F0D2FE04280CD1216C2046B3
:10B5000061640CF086FF064609F0B0F818B100211E
:10B51000304609F020F9284609F0C0FE012804D081
:10B52000284609F0BBFE032809D16946284609F0E0
:10B5300089FE20460199FDF7D9FE2064606420460B
:10B5400007F088FF206B10B920460EF010FB206C2E
:10B55000029002AA202120460FF0B9FBFEBD000098
:10B5600010B5582109480BF066FA0022212108483D
:10B5700013F03AFA054CAC3CC4F8A800A434F8F730
:10B5800089F800202070607010BD00005851002024
:10B59000C53600082DE9F04105460F480E46002447
:10B5A000074616E00168A94200D01DB94168B142C2
:10B5B00009D046B1014638460BF032FA0028F1D1E5
:10B5C0002046BDE8F08115F0CDFEF8F763F80124C0
:10B5D00038460BF013FAF1E75851002070B50546D4
:10B5E0000A480C4606460BF009FA0BE00168A9422E
:10B5F00004D14168A14207D0002C05D00146304655
:10B600000BF00EFA0028F1D170BD00005851002057
:10B6100010B50446582200210BF021FC4FF4FA70BB
:10B620002063002060626420E062012060640448BE
:10B63000206294F8540040F0080084F8540010BDD3
:10B64000B1B600082DE9F84304464FF48060174670
:10B6500000901E46D4E90C2088460023089D194618
:10B660000BF004FB33463A464146009503F028F8B8
:10B67000626AE16A891A414302EBA120BDE8F883BE
:10B6800008B5B0F94E200092B0F94C30B0F94A201C
:10B69000B0F94810FFF7D6FF08BD08B54FF4806138
:10B6A0000022009140F251231146FFF7CBFF08BD65
:10B6B00038B504464FF480600090D4E90C20002394
:10B6C00019460BF0D3FA626AE16A891A414302EB28
:10B6D000A12038BDD0E90C128A4201DBC06A704754
:10B6E000406A704710B5029C20F8481F8380428052
:10B6F000C48010BD01617047494241637047416198
:10B7000070470163704710F8542F61F3C302027051
:10B710007047416070470162704781637047C16341
:10B7200070474164704701647047C1607047C161F0
:10B73000704741624FF00041C0E90A127047016052
:10B74000704710B542F2107442F2F673A04200D96D
:10B750001846A14200D91946A24200D91A460A2326
:10B76000401D491D521DB2FBF3F2B1FBF3F1B0FBDA
:10B77000F3F0120502EB8121084400F1004010BDF6
:10B7800070B5054620480BF05EF9040028D0582219
:10B7900029460BF0A9FA2868A84200D124601A486B
:10B7A000AC3890F8A51014F8540F61F3410004F878
:10B7B000040913F0CFF801C414F8540900071FD589
:10B7C000A16939B120468847616A01446162E16A32
:10B7D0000844E062204615F0E3FE686818B900E00E
:10B7E000FEE7A86810B1204615F0FAFD626812B1B4
:10B7F000616A20689047A26812B12046616A90474A
:10B80000F7F748FF204670BD5851002010B5D0E929
:10B810000E431B1B02E000BF03F5B473002BFBDBE0
:10B820004FF4B474A34202DBA3F5B473FAE7994270
:10B830000FDC03EBD372B1EB620FC16C02DA41F0A3
:10B84000080101E021F00801C0F84C1041F010019E
:10B8500017E0C3F5B474944203DCC16C41F00801F5
:10B86000F4E7C1F5B474944203DCC16C41F0080103
:10B8700005E01A448A4207DBC16C21F0080121F07F
:10B880001001C164012010BD002010BD10B50C4690
:10B8900087212D22C4E90E120020C4E90B014900C2
:10B8A0006163E16C21F00601E16413492164E16CFC
:10B8B000606441F008016420C4E9120121F0010034
:10B8C000E0641001206513F045F86065606BA065C9
:10B8D000E06C022120F01000E06420460BF039FDFE
:10B8E0004FF4447120460EF037FF2046BDE810406B
:10B8F0000D210FF00BBA00000080FFFF2DE9F0438F
:10B90000BBB0044608F012F90546204608F045F998
:10B91000814614AA31A92846FDF7E9FB14980028AE
:10B920001ADD684603F087FA6A46002128460DF0C2
:10B9300030FEDDE93101CDE90B01A96BE86A08446D
:10B940000990E96BE86A08440A901498ADF834004D
:10B950006946484603F03CFA4FF400384146284611
:10B960000DF086FB0746414628460DF0A2FB064631
:10B97000414628460DF0C4FB0446414628460DF0DA
:10B980004AFBB74201DD394600E03146844201DD21
:10B99000224600E00246914205DDB74201DD38460D
:10B9A00004E0304602E0844200DD204614990C1A7F
:10B9B000002C19DD684603F03EFA6A4641462846E7
:10B9C0000DF0E7FDDDE93101CDE90B01D5E90B0112
:10B9D00008440990696BE86AADF8344008440A905D
:10B9E0006946484603F0F4F936AB31A92846149A63
:10B9F000FDF7F8FC15A805F0C1FA15AA4FF440317F
:10BA000028460DF026FF36AA15A9484605F0A0F8ED
:10BA10003BB0BDE8F08300002DE9F04F89B08A46C5
:10BA2000FE480CF004FC01287DD1504608F07AF85D
:10BA30000546504608F07AF804464FF0640B4FF480
:10BA4000B479022D13D0082D6ED0032DFCD00E2D0D
:10BA50006BD00F2D6AD0132D69D0182D68D01A2DF8
:10BA600061D109B05046BDE8F04FFFF747BF09F07C
:10BA7000CBFB050057D009F011FC012853D101A9D7
:10BA8000284609F0DFFB05AA03A92046FDF72FFB96
:10BA900003990198401A019002990498081A02909B
:10BAA00094F84C00C00731D14FF4003120460DF01E
:10BAB00095F9054605984FF48031401B05902046C6
:10BAC0000DF056FD0028059806D1C11700EB9171C5
:10BAD000B5EBA10F00DA8D10401B0590012801DAAB
:10BAE000012005900198029A404302FB020105984B
:10BAF0004043814206DDE06C40F00101E16412F058
:10BB000029FF606594F84C00C0070CD0019911B969
:10BB10000298002807D0D4E90E06864201DA06F51D
:10BB2000B476029805E0ABE0C0E0D9E0F6E0FBE0D7
:10BB300061E100F075FEE16A401AA16B451A01E06F
:10BB400005F5B475002DFBDB4846854202DBA5F503
:10BB5000B475FAE705984FF41D714843B0FBFBF745
:10BB6000322003F0FFF84FF4B4714843B0FBF7F212
:10BB700094F84C002946C0F3C0072046FFF746FE64
:10BB800000287DD0A06BA26D311AA2EB0008A5EBB6
:10BB90000800002801DD024600E042424FF48C73A9
:10BBA0009A4205DD94F84C20120709D5002508E0DB
:10BBB000E26C5FEAC26C04D4120701D54D4200E08A
:10BBC0000D4677B1E16C0A071ED4CA061CD40028C2
:10BBD00000DC4042984217DD67F3C3010025E164B1
:10BBE00012E08FB9E26C5FEA027C0DD55FEAC26CAD
:10BBF0000AD4002800DC4042C0F5B470984203DD4E
:10BC000067F3C3020D46E264A5EB0805606D12F010
:10BC10009BFE216D41434FF47A70B1FBF0F08542F9
:10BC200002DC4042854200DA0546D4E91132A16BBC
:10BC3000D01A771AFF0097FBF0F0001DC717454494
:10BC400000EB177005EB2010256C0092084432467B
:10BC50000BF00CF8064694F84C00C0F341000228A3
:10BC600003D1A06C811B606C0E18206CB04211D007
:10BC700012F070FE60653146204600F018FA00E0D0
:10BC800011E0AE4206D00022202120460FF01FF81E
:10BC9000012808D1606CB04202D0A06CB04202D141
:10BCA00012F058FE606509B0BDE8F08FE06C20F03E
:10BCB00001012046E1640CF0ACFB054608F0D6FC1F
:10BCC000044609F0A1FA09F0E9FA0428EBD1002CA6
:10BCD000E9D009B02846BDE8F04F002108F03BBD8F
:10BCE000504607F04EFF256C132806D0112804D0CB
:10BCF000142804D0122802D005E0691C00E0691E57
:10BD0000204600F0D4F9206CA842CCD009B02046DF
:10BD1000BDE8F04F002220210EF0D9BF504607F0B9
:10BD20004FFF256C2918EBE7504607F047FF054603
:10BD300003AA01A92046FDF7DAF9A068002600B1A0
:10BD4000066A002120460DF049F8804603993044E8
:10BD5000081A0299029A01440091019903900B1864
:10BD6000121A091A04A800F0BCFC47F6FF7204A8D6
:10BD7000296800F01AFC4FF0000AC0BB2868019A3D
:10BD800001684068891A029A801A00F049FDE16A48
:10BD9000401AA16B471A01E007F5B477002FFBDBCF
:10BDA0004846874202DBA7F5B477FAE703984FF4D9
:10BDB0001D714843B0FBFBF9322002F0D3FF4FF472
:10BDC000B4714843B0FBF9F239462046FFF71EFD37
:10BDD00068B108EB4602114604A800F023FB47F6C1
:10BDE000FF7204A8296800F0E0FB28715BE7FFE719
:10BDF00085F804A057E700210DF03AF90746002125
:10BE000020460DF056F90646002120460DF078F93F
:10BE10000546002120460DF0FEF801E014EA020874
:10BE2000B74201DD394600E03146854201DD2A4650
:10BE300000E00246914205DDB74201DD384604E0EC
:10BE4000304602E0854200DD284680464FF4403906
:10BE5000494620460DF00CF90746494620460DF0AC
:10BE600028F90646494620460DF04AF90546494656
:10BE700020460DF0D0F8B74201DD394600E03146EA
:10BE8000854201DD2A4600E00246914205DDB742C7
:10BE900001DD384604E0304602E0854200DD2846F8
:10BEA000801CA0EB08052046FFF78EF84419504689
:10BEB00007F084FE0168A14200DD0C460460F2E652
:10BEC00070B50C460546114600F076F82146284626
:10BED000BDE8704000F0B6B870B50C460546114696
:10BEE00000F006F821462846BDE8704000F032B860
:10BEF00070B505460C46B1F5B47F01DDA1F5B4740B
:10BF0000D5E90E10421AA4EB010101D502F5B47275
:10BF1000002901DA01F5B4718B1A002B00DC531AE9
:10BF2000B42B03DD28460DF022FE0DE0914203DA2A
:10BF300000230246214604E08A4205DA0023224615
:10BF400001462846FEF70CFD2846EC63BDE870402C
:10BF50001AF042BD70B505460C46B1F5B47F01DD5F
:10BF6000A1F5B474D5E90E010A1AA1EB040101D5BB
:10BF700002F5B472002901DA01F5B4718B1A002BB5
:10BF800000DC531AB42B03DD28460DF0F0FD0DE064
:10BF9000914203DA00232246014604E08A4205DA90
:10BFA0000023024621462846FEF7DAFC2846AC6309
:10BFB000BDE870401AF010BD70B505460C46B1F5ED
:10BFC000B47F01DDA1F5B474D5E90C10421AA4EBDD
:10BFD000010101D502F5B472002901DA01F5B4714D
:10BFE0008B1A002B00DC531AB42B03DD28460DF00E
:10BFF000BEFD0DE04FF40033914202DA02462146C5
:10C0000003E08A4204DA224601462846FEF7A8FCED
:10C010002846FEF7EDFC28466C63BDE87040FEF74D
:10C02000E7BC000002E000BF01F5B4710029FBDBB2
:10C030004FF4B472914202DBA1F5B471FAE7C16228
:10C040000DF095BD70B505460C46B1F5B47F01DD28
:10C05000A1F5B474D5E90C010A1AA1EB040101D5CC
:10C0600002F5B472002901DA01F5B4718B1A002BC4
:10C0700000DC531AB42B03DD28460DF078FD0DE0EB
:10C080004FF40033914202DA2246014603E08A422D
:10C0900004DA024621462846FEF762FC2846FEF7EF
:10C0A000A7FC28462C63BDE87040FEF7A1BC036CDA
:10C0B0008B420CD0826C8A4200DA1146426C8A4272
:10C0C00000DD11468B4202D001641AF085BC704736
:10C0D000F0B50D688C68D1F80CE0641BD0E9006500
:10C0E0004F68DDF814C0AEEB0707162A75D2DFE8FB
:10C0F00002F0C7C71A272D2F454D5D0B6567757B6D
:10C100007D8F97999B9DA1BD8268A2EB060E0EF1D3
:10C11000010E621C0EEBDE7E4FEA6E0E02EBD27257
:10C12000AEEB620233E08068821B601C521C02EBA3
:10C13000D272521000EBD070A2EB600200208AE0B5
:10C140008068621C801B401C821AF7E700220DE009
:10C150008268A2EB060E0EF1010E621C0EEBDE7E73
:10C160004FEA6E0E02EBD272AEEB6202C06807F1CC
:10C17000010E401B401CA0EB0E006CE0826804F135
:10C18000010E921B521CA2EB0E02EFE70022C068C8
:10C19000A0EB050E0EF1010E781C0EEBDE7E4FEAD1
:10C1A0006E0E00EBD070AEEB600054E0826804F1DC
:10C1B000010E921B521CA2EB0E02E8E700220AE0DD
:10C1C0008068821B601C521C02EBD272521000EB82
:10C1D000D070A2EB6002F8433DE051E08068621C41
:10C1E000801B401C821AF6E700220DE08268A2EB59
:10C1F000060E0EF1010E621C0EEBDE7E4FEA6E0E95
:10C2000002EBD272AEEB6202C068401B401C22E01F
:10C21000826804F1010E921B521CA2EB0E02F3E79E
:10C22000E2438BE7E243B2E7E2439FE78068821B89
:10C2300000200FE08268C068921BA0EB050E0EF193
:10C24000010E781C0EEBDE7E4FEA6E0E00EBD07016
:10C25000AEEB6000521C324428441A446044C1E9E9
:10C26000002022443844C1E90220F0BD8268C06841
:10C27000921B401B07F1010E401CA0EB0E00E9E7EA
:10C2800000225BE70A6802604A6842608A6882604E
:10C29000C968C16070470A6802604A6842608A687B
:10C2A0008260C968C16070470A6802604A6842607B
:10C2B0008A688260C968C16070470A6802604A681B
:10C2C00042608A688260C968C16070470A6802601B
:10C2D0004A6842608A688260C968C16070470A68BB
:10C2E00002604A6842608A688260C968C1607047BB
:10C2F0000A6802604A6842608A688260C968C160F0
:10C3000070470A6802604A6842608A688260C96849
:10C31000C16070470A6802604A6842608A68826049
:10C32000C968C16070472DE9F0470C4606461546BE
:10C330001146204600F0E6F800285CD0002229468D
:10C34000204600F09CF800284FF0000051D1E7682B
:10C3500061682368A7EB010C6F68A2687F1AA2EBE3
:10C360000309002F05DD08C60F4486E8860001207A
:10C37000361FE96862688A1AACEB0203002B0CDDF9
:10C38000E268914209DA06EB001C2768A2684CF8C3
:10C39000047B0B448CE80E00401C69686268914283
:10C3A00000DC1146EA68E3689A4200DB1A46531A39
:10C3B0002F682268BF1A002F0BDD002B09DD06EB6A
:10C3C0000018174448F8042B01EB030C88E882108E
:10C3D000401CAA682468151BA9EB0504002C08DD85
:10C3E00006EB00151444C5E900210B44C5E90243DE
:10C3F000401CBDE8F0874FF0FF30FAE7C1684068A5
:10C40000081A401C704702688168891AC26840682F
:10C41000101A401C491C4843704781680068081A7C
:10C42000401C704703685B1A03608368194481608D
:10C430004168891A4160C1681144C160704770B594
:10C440000B681468A34200DC234603604D685468FF
:10C45000A54200DD2C4644608E689568AE4200DA45
:10C4600035468560C968D268914200DB1146C160DB
:10C470000120AB4201DC8C4200DD002070BD7CB5A8
:10C480000D460446006809681646884238DB616834
:10C490006A68914234DBA268AB689A4230DCE26899
:10C4A000EB689A422CDC4EB3CDE900013246694676
:10C4B000284600F07AF8002821D0D4E90110CDE90F
:10C4C000000132466946284600F06FF8002816D071
:10C4D000E1682068CDE9000132466946284600F04F
:10C4E00064F800280BD0D4E90201CDE900013246FE
:10C4F0006946284600F059F8002800D001207CBD8C
:10C5000000207CBD02688B689A420DDC82680B6853
:10C510009A4209DB4268CB689A4205DCC0684968E8
:10C52000884201DB01207047002070477CB50D4632
:10C530000446806809681646884234DBE06869680A
:10C54000884230DB2168A86881422CDC6068EA6898
:10C55000904228DC2EB3CDE90010324669462846C9
:10C5600000F023F8E8B9D4E90110CDE90001324622
:10C570006946284600F019F898B9E1682068CDE9C5
:10C58000000132466946284600F00FF848B9D4E960
:10C590000201CDE9000132466946284600F005F85F
:10C5A00008B100207CBD01207CBD2DE9FF4114466F
:10C5B0000E460A68016805468A422EDBA868824258
:10C5C0002BDC72686B689A4227DBEF68BA4224DC86
:10C5D000002C5DDD401A401C00EBD0704210F81AB0
:10C5E000401C00EBD0704010824200DA10468442BA
:10C5F00000DD04460091286800222044029068680B
:10C60000019068683146204403906846FFF7CDFFEB
:10C6100038B102982044029032E0002004B0BDE816
:10C62000F081E8680022001B0190E8680390314621
:10C630006846FFF7BAFF18B10298204402900DE057
:10C64000A8680022001B0090A86802903146684646
:10C65000FFF7ABFF30B10098001B00900198001B62
:10C66000019010E0686801906868002220440390FF
:10C6700031466846FFF799FF50B10098001B0090C3
:10C68000039820440390314668460FF0A9F8C5E7A7
:10C690000120C3E710B50C6813689C4200DA2346FA
:10C6A00003604C6853689C4200DA234643608C6800
:10C6B00093689C4200DD23468360C968D26891423A
:10C6C00000DC1146C16010BD03680B440360836841
:10C6D00019448160416811444160C1681144C160DE
:10C6E000704710B5029C80E81E0010BD4268491ECC
:10C6F0001144C16070470268491E1144816070474F
:10C7000042688A4201D80020704702681AB1C068A6
:10C7100001FB00207047FEE770B504460068002565
:10C7200010B107F091FC25606560A56070BD002127
:10C73000FFF7E6BF10B50446231D002083E807007D
:10C7400001FB02F00AF05AFA2060002800D1FEE74F
:10C7500010BD70B5044600680D46A0B1D4E90101D2
:10C76000884203D12046091D00F00EF8D4E90001EB
:10C77000E26801FB020029460AF0B6FA6068401C34
:10C780006060012070BDFEE770B50D46C1680446CB
:10C79000694300680FF066F930B1A56020606068F9
:10C7A000A84200D9656070BDFEE740687047000090
:10C7B0002DE9F04781468A46002012F087F90446A9
:10C7C0004FF000080E4F16E0204612F07FF90546A4
:10C7D000A068B8420ED1E668316849450AD171684F
:10C7E000514507D1204612F027F9304607F02CFCBE
:10C7F0004FF001082C46002CE6D14046BDE8F087FA
:10C8000005C8000870B5C568D5E9004612F014F9EE
:10C81000284607F019FC3046A446BDE87040604742
:10C820000022002801DA01224042002901DA4942AF
:10C83000921C884207D9C1EB011101EB4101B1FB08
:10C84000F0F3103205E0C0EB001000EB4000B0FB4D
:10C85000F1F30020D9B216290BD92C2900D80120D8
:10C86000292900D8401C252900D8401C20290BD993
:10C870000BE0022900D30120062900D3401C0A291D
:10C8800000D3401C0F2900D3401C1844D10601D509
:10C89000C0F15A0091074FEAC27105D509B1B43011
:10C8A00005E0C0F1B40002E009B1C0F5B47080B297
:10C8B0007047C16000680DF05AB900684FF0FF3250
:10C8C0000168C26001F15002904202D18268CA62DE
:10C8D00005E001F16002904201D182688A6300683C
:10C8E0000DF045B910B50C4600206421C4E90C01D7
:10C8F000A063E062E06360642064A06494F8701058
:10C9000021F03F0184F8701084F84C0004F15001CC
:10C91000204600F0A2F804F16001204600F09DF8E6
:10C92000082120460DF018FF102120460DF014FFBD
:10C9300020460022BDE81040114600F0CDB810B5E9
:10C940000C46002104F15000FEF724FE04F16000C3
:10C95000BDE810400021FEF71DBE00002DE9F041AA
:10C960000D462F480BF063FC01284FD1284607F0F5
:10C97000D9F80446284607F0D9F88046182C0AD082
:10C98000012C45D0082C43D01A2C3FD12846BDE8B5
:10C99000F041F9F77BBA4FF400310AF0C2FF0446C8
:10C9A000284607F00BF905460068A04200DD044662
:10C9B000002140462C600CF05EFB074600214046FB
:10C9C0000CF07AFB0646002140460CF09CFB044626
:10C9D000002140460CF022FBB74201DA394600E064
:10C9E0003146844201DA224600E00246914205DAED
:10C9F000B74201DA384604E0304602E0844200DA09
:10CA00002046002802DA2968081A2860BDE8F0816B
:10CA100008F13C014046BDE8F0410DF0C3B800000C
:10CA200038EA020890F8700000F00700704790F8AC
:10CA3000701001F00701022901D0006B7047C16E30
:10CA4000491C01D0806E7047806B7047C16D491CD6
:10CA500001D0806D7047C06A704708600020486050
:10CA60008860401EC860704790F8701001F00701A0
:10CA700001290AD1016B002907DA426B002A04DD83
:10CA8000806B884201D1012070470020704738B583
:10CA9000134690F8702002F00702022A1BD1D0E959
:10CAA0000C428A4201DD0D4600E01546AC4201DD34
:10CAB000214602E08A4200DC1146C26A8A4200DA5C
:10CAC0001146826B8A4206D0009300F1600300F1A8
:10CAD000380200F023F838BDF8B5C56A13468D4218
:10CAE0001AD0D0E90C428A4201DD0E4600E016461B
:10CAF000B44201DD214602E08A4200DC1146826B2D
:10CB00008A4200DD11468D4206D0009300F15003A9
:10CB100000F12C0200F002F8F8BD0000F0B597B06B
:10CB200007461C981C4616460D4668B3E068401C34
:10CB300040D0A068C4E90105002118461560FEF741
:10CB400029FD6846FEF764FD21466846FEF7F7FDBD
:10CB500019496846FEF7DDFD4FF4807200216846F2
:10CB6000FEF7E7FD15496846FEF7C4FD384600218B
:10CB700064220CF0E3FA01466846FEF7C2FD6846FF
:10CB8000FEF7FEFD17B0F0BD00211846FEF702FDCE
:10CB90004FF0FF30E060384635600CF0E8FF0021D0
:10CBA0002046FEF7F7FC17B021463846BDE8F040B6
:10CBB000FFF753BF3068BDE7B3C80008BBC8000823
:10CBC00070B58C6C0D462CB1206C18B102F0BBFC1A
:10CBD000002020642846BDE87040FCF7C9B800007A
:10CBE0002DE9FF4F088C85B0C0F30725E81F1E46CE
:10CBF0000C46039003280BD9102D09D0112D07D016
:10CC00000F2D05D0122D03D0132D01D0142D1ED1C0
:10CC1000D4F848805FEA08001AD0D8F800000190E4
:10CC2000284601F091FC81460798FFF7F6FB834602
:10CC3000207C01280FD00020824670686FF0604190
:10CC4000C84231D10398032807D8102006E00020FD
:10CC500009B0BDE8F08F0C20EEE7284602900020D6
:10CC6000009001235A46D8F84000029902F00BFECA
:10CC7000070013D1D8F8400020B102F064FC002076
:10CC8000C8F8400000200090012259465848029BF5
:10CC900002F018FC0700DAD0C8F84070079907C9FD
:10CCA00086E80700F16006E0401C7060F068401CF8
:10CCB000F060D8F8407007997068D7F81080C9689C
:10CCC0008842C4DC0399032946D80822B2FBF9F153
:10CCD0003268B2FBF1F301FB132102910BFB09F166
:10CCE0000123C91D03EBD1010391636B02FB09F220
:10CCF0000AEB8301238D9BB200FB031000EBD209EA
:10CD0000207C012810D0E068016901EB090600BF12
:10CD1000CDE900685B46216B2846029AF8F77CF85B
:10CD2000207C012814D050E0039809F067FF06002A
:10CD30000DD00020009032464946039B0198FCF735
:10CD400034F80028E4D0304607F07EF97FE7FEE7AC
:10CD5000304607F079F938E0102D39D0112D37D051
:10CD60000F2D35D0122D33D0132D31D0142DEDD100
:10CD700039894FF000098DB2218D2B468AB200FB14
:10CD800002A031684246090100EBD101CDF80090C4
:10CD90000198FCF70AF80028D8D1616A0C200A0C27
:10CDA000218D8BB202FB03007268C1F34E0102FBBE
:10CDB0000100316808EB050201445B46CDF80090A4
:10CDC0000198FBF7F2FF0028C0D10120E7623FE79E
:10CDD0000BFB09F1CB08218D8AB200FB02A0316860
:10CDE000424601FB09F100EBD10100200090E7E78A
:10CDF000A451002038B50D46C968287C144620B1DE
:10CE0000012807D0022825D016E00C22204609F080
:10CE10006BFF24E0084607F071F915A10FF034FF0D
:10CE200050B96B460C22214605F1140007F0CDF9EC
:10CE300010B900980C2801D0002038BD207819289E
:10CE400002D06070192020702068202141EA104033
:10CE5000608004E00120A080E0800E2060702068E7
:10CE6000C1B2192902D0400C40006080012038BDB9
:10CE700062696E0010B507F0E3FD040011D00949A6
:10CE800007F0D0FE0849204607F0CEFE07492046AD
:10CE900007F0C6FE0649204607F0C0FE05A0206147
:10CEA00010BDFEE7F5CD0008B9CE0008E1CB0008C3
:10CEB000C1CB000842494E002DE9F04782464FF0B1
:10CEC0000008087C90B00C464546C146012801D0B8
:10CED00088B34FE0E06807F011F95EA10FF0D4FECF
:10CEE00098B92046FCF779F906000ED00C20A6640C
:10CEF00009F084FE070007D00222E16807F01AF962
:10CF000038B1384607F0A0F89FE0002010B0BDE827
:10CF1000F0873760216AC1F30720090C090729D47B
:10CF2000C11F032923D90B3803285ED82146504658
:10CF3000F7F78EFE04E007E021465046F7F712FFB0
:10CF40008046012816D150E0E66830690028DDD01F
:10CF50003088C0F30727206A000C00070AD4F81FA6
:10CF600003280CD80846FCF738F90028CED0E07921
:10CF70000028E1D02046FBF7FBFE4046C6E7A7F1BC
:10CF80000B000328084604D8FCF727F90028BDD079
:10CF9000CCE7FCF722F93168090CC90601D5354602
:10CFA00009E000F1240530890004000C09D0314665
:10CFB000284602F015FBE56228890004000C11D018
:10CFC00012E01822314608A8F3F7B6FA384601F005
:10CFD000BBFA099989B24843C01DC008ADF82800C2
:10CFE00008A9E5E7208D28810125E76A5FB3394666
:10CFF000204607F0BFFD060027D0BE4208D02046DD
:10D00000FBF7B6FE2046FCF7E8F8C661E66201E0F1
:10D01000E062C5B9A079B0B907F08AFC98B1207C6C
:10D020008DF81000E0680390E26A02A9D0680290CF
:10D030005046A36C07F0CAFC38B160642046FCF788
:10D04000CCF8C0F81C90012060E72046FBF790FE6A
:10D050005BE7000062696E0010B50C4610212046A7
:10D060000DF07AFB2046BDE810404FF480610AF0D5
:10D0700070B9000010B5014603480AF0D1FC04461F
:10D080000AF034FD204610BD5CEA020870B5044683
:10D09000806B154688420FD9606B30F81120AA4387
:10D0A00020F811202046FDF7BFFC680504D5204676
:10D0B000BDE870400DF0A6BA70BD70B50E460546CD
:10D0C000002405E0324621462846FFF7DFFF641CB6
:10D0D000A86BA042F6D870BD084600214FF6FF723B
:10D0E0008163C0E90F1201634163C1624164014978
:10D0F00000F0ECBA80EA020810B5014603480AF0D5
:10D100008FFC04460AF0F2FC204610BD9CEA02089F
:10D1100010B50C46086B06F097FF606B06F094FFA5
:10D1200000202063606310BD2DE9FE4F8A46FE4853
:10D130000BF07DF8012833D1504606F0F3FC06468B
:10D14000504606F0F3FC00270446182E02D02F2E7E
:10D1500048D02BE0E06BA146002821D00025D9F86B
:10D160002C800FE0D9F8340030F81500400508D5C0
:10D17000E06BB8B120460BF0FDF8E16BB0FBF1F1CC
:10D1800011E06D1C58F82500002809D0E7A10FF028
:10D190007BFD002804D058F8250000780028E1D154
:10D1A000BDE8FE8F0021504606F089FD2E2E1DD0D1
:10D1B0004FF6FF75012E1BD0022E59D0082E69D0D4
:10D1C000062E7CD0032E7BD0102E7AD0112EE7D0E5
:10D1D000122EE5D00E2E75D01A2EE1D15046F9F759
:10D1E0006FFDDDE7E16A00F071FAD9E72046F9E763
:10D1F000504606F09DFC06462046216CFDF714FCC7
:10D2000008F002F808F04AF8012801D003281AD1E2
:10D210006946304608F016F869462046FBF70BFED3
:10D220002564A842BCD0616B31F81010C1F38012A4
:10D23000002AB5D1C1F300110029B1D10146206403
:10D240002046FDF7F1FB206CA842A9D0616B31F8B4
:10D250001000C0F340210029A2D1C0F3802166E074
:10D26000206C029002AA202120460DF030FD97E7A5
:10D27000206CA84294D0504606F05AFC694607F04C
:10D28000E1FF69462046FBF7D6FD216C814287D03D
:10D29000204659E0216CA9423CD0626B32F8110063
:10D2A000C0F3C013CBB1C0F38013B3B9C30503D52A
:10D2B00094F84430DB0718D040F4807003E02EE08F
:10D2C00040E044E08DE022F8110094F84400C007EB
:10D2D00003D02046216C12F0BAF8216C606B30F854
:10D2E0001100C0F3402131B902E020F48070E5E77D
:10D2F000C0F3802171B1C0F3801159B9C0F300109F
:10D3000040B9206C029002AA202120460DF0DFFCDB
:10D310000128ACD12046216CFDF786FB40E7206C4C
:10D32000A842A4D0616B31F81000C0F3401100296D
:10D330009DD1C0F38011002999D1C0F300100028BD
:10D340008ED02DE72046216CFDF76EFB47E0A06BE9
:10D3500000288CD0504606F0EBFB074607F09EFFF6
:10D3600006462FB9002007F061FF07F097FF064639
:10D3700020460BF04EF807F079F9216CA942CDD187
:10D38000022E02D0042E2AD148B394F84410002073
:10D39000A26BC90701D113E0401C82421DD9616B09
:10D3A00031F81010C1F30013002BF5D1C1F3801335
:10D3B000002BF1D1C1F300210029EDD00DE0401C7C
:10D3C00082420AD9616B31F81010C1F30013002BAF
:10D3D000F5D1C1F380110029F1D12064E0E6256484
:10D3E000DEE62046216CFDF71FFB504606F0C9FB28
:10D3F000132813D0142835D004264FF0080912281A
:10D4000052D0112886D1002120460BF025FE8046FF
:10D41000206CA84274D12764626BA3E0206CA84200
:10D4200002D13846276401E0401C2064A36B984277
:10D4300000D32764666B226C07E0491C2164994283
:10D4400000D32764206C90426DD0216C36F8110017
:10D45000C0F3001CBCF1000FEFD1C0F38010002816
:10D46000EBD157E7206CA84201D1276400E000B956
:10D47000A06B401E20640346626B09E019B1491E8F
:10D480000846216402E0A06B401E2064984267D0E9
:10D49000216C32F81100C0F30016002EEED1C0F35B
:10D4A00080100028EAD135E7002120460BF0D4FD9A
:10D4B0008046206CA84213D12764626B04E0491CAB
:10D4C0002164A06B81424BD2216C32F81100C0F371
:10D4D0000013002BF3D1C0F380100028EFD119E71F
:10D4E000216B01EB0010FEF798FF0346206C216BC7
:10D4F000024601EB00152D6805EB630CA36B25E0DC
:10D500003CE000BF06EB001506EB02174D59CF5962
:10D51000BD421ADD01EB00152D68654515DC09EBF0
:10D5200000154F5904E01BE09CEA02080A000000C5
:10D5300007EB0805654508DB656B35F81050C5F34A
:10D54000801717B9C5F3001515B1401C8342D9D80F
:10D55000834245D8DEE6491C2164A06B814201D399
:10D560002564D7E6216C32F81100C0F30013002BBC
:10D57000F1D1C0F380100028EDD1CBE6216B01EB97
:10D580000010FEF74AFF226C216B01EB02131B68AF
:10D5900003EB600310B21EE006EB001506EB02176A
:10D5A0004D59CF59BD4214DA01EB00152F68A7EB96
:10D5B00008059D420DDC09EB00154D599D4208DB25
:10D5C000656B35F81050C5F3801717B9C5F3001512
:10D5D00025B1401E00B20028DEDA9BE60028B9DB48
:10D5E000206497E62DE9F0410F46A1F57F41FF3910
:10D5F00015D00546806BB84211D30024264609E0B9
:10D60000E86A641C09A150F82400761C0FF03CFB6A
:10D6100000B9641CBE42F3D1A86BB04202D1002015
:10D62000BDE8F081E86A50F82400F9E70A0000003C
:10D63000006C7047836B8B4204D9406B30F811004B
:10D64000824301D0002070470120704770B5044626
:10D65000806B0E461546B0421BD994F84400C007B3
:10D6600006D0E80504D54FF480712046FFF725FD6C
:10D67000606B30F81610294320F81610314620460A
:10D68000FDF7D2F9680504D52046BDE870400CF0DE
:10D69000B9BF70BD70B50E460546002405E03246A0
:10D6A00021462846FFF7D2FF641CA86BA042F6D89B
:10D6B00070BD10B50446806B4200606B09F014FB2E
:10D6C0002046E16ABDE81040AFF300802DE9F04F3D
:10D6D00097B00D0004467DD0F5F75EFF00212722AC
:10D6E0002046E5620BF02AFDC0B2002712903946B1
:10D6F00020460BF0C3FC0646394620460BF0E6FBFD
:10D700008046394620460BF0CFFB400700D5464403
:10D71000002080460146274620460A960BF0F6FC7C
:10D720000646414638460BF0D1FB81464146384615
:10D730000BF0BAFB800700D54E44002120460F961F
:10D740000BF0D8FC0390002120460BF085FC0890DC
:10D7500020460AF020FE069020460AF00BFEE16B00
:10D760000027C1F101020399A94601FB02001090B4
:10D7700038467BE04FF0000B5D4607E0606B79199F
:10D7800030F81100FBF70CFC83446D1C59F82500A0
:10D7900040B13FA10FF078FA20B159F82500007888
:10D7A0000028EBD14DB31098E16B00FB08F0B0FB03
:10D7B000F1F20F981318039A08FB02300E9010989C
:10D7C00008F101025043B0FBF1F0039B0F9908FBF5
:10D7D000031100E058E0401E084414900899069890
:10D7E000C5F1010201FB02000D90002801DA0020C2
:10D7F0000D904FF0000A564630E009F1040032E087
:10D80000606B30F81700FBF7CBFB01460D9800FB6F
:10D810000AF0B0FBFBF208988A4406FB00200D9A40
:10D820000AFB02F1B1FBFBF1089A491E06FB02124A
:10D830001299012904D101460698801A069A521AB3
:10D840000A9901440A98131814980090206B0E9AB4
:10D8500000EB0710FEF745FF761C7F1CAE42CFD3CE
:10D8600009EB8500001D814608F10100E16B80464F
:10D8700041453FF67FAF20460CF0C4FE17B020466E
:10D88000BDE8F04F0CF073B917B0BDE8F08F0000A1
:10D890000A00000070B50446806B0D46A84203D80C
:10D8A000A5F57F40FF380AD12046216CFDF7BCF872
:10D8B000204629462564BDE87040FDF7B5B870BD27
:10D8C0002DE9F04117460E46040017D0BEB104F111
:10D8D0001C00054609F028FDE06888B120683A463A
:10D8E0003146C36820469847040001D000F056F83E
:10D8F000284609F01BFD2046BDE8F081FEE7FEE763
:10D90000284609F013FD0020F6E72DE9F0411746FF
:10D910000E46040016D0B6B104F11C00054609F00D
:10D9200003FDA06880B13A4631462046F6F73DF93E
:10D93000040001D000F032F8284609F0F7FC204638
:10D94000BDE8F081FEE7FEE7284609F0EFFC002085
:10D95000F6E72DE9F0470546DDE9089A00681E461E
:10D96000174688468047040012D004F10C010020BD
:10D97000A76081E84106C4E90058696820468847E5
:10D9800038B104F11C0009F0CDFC2046BDE8F08759
:10D99000FEE7204606F058FB0020F7E700B502003E
:10D9A00006D000F027F810465DF804EB00F013B83D
:10D9B000FEE730B14168491E416001D50021416058
:10D9C0007047FEE710B528B100F005F8BDE810403B
:10D9D00006F03ABBFEE710B18168401A7047FEE7D7
:10D9E00008B108447047FEE708B140687047FEE799
:10D9F0001030704718B14168491C41607047FEE71C
:10DA000030B131B101600021C0E9011201737047EA
:10DA1000FEE7FEE708B1007B7047FEE720B14168F2
:10DA2000002902D0FFF7C5BFFEE7704780680028D5
:10DA300000D0012070472DE9F04116460D00044644
:10DA40000DD004F11C00074609F06EFC3146284653
:10DA5000FFF7E4FF2846FFF7C7FF08B10DE0FEE738
:10DA60002846FFF7D7FF40B12846FFF7B4FFA26969
:10DA7000314690472846FFF7A5FF3846BDE8F041FC
:10DA800009F054BC002800D0016270472DE9F04134
:10DA90000F460C464FF4FD612186012084F83200C8
:10DAA00084F83300A18684F8360084F8370000201B
:10DAB000A063E06304F221104FF45272002109F0D8
:10DAC000CEF900210846324B782506E028B14207FE
:10DAD000B2F1604F08D0072808D253F8202000BFC9
:10DAE00004EB800632640EE02AA2F9E701EB810222
:10DAF00004EB820204EB800682F8215102F221122B
:10DB0000491CC9B23264401CC0B23828DED322A0FE
:10DB1000C4F81C013846FFF7EFFA04F14001E06257
:10DB2000FFF7D4FD54F82C0F4FF40871FFF7B2FD46
:10DB300000231F221949206809F0FAFB64200DF028
:10DB400043FD014620680DF074FA4FF4042120686B
:10DB500009F0FFFB012138460DF0F8F8012120689B
:10DB60000DF000F90022022138460DF04EFA94F92A
:10DB70000A202189384600F015F894F9073094F905
:10DB80000620A1883846BDE8F04100F0ABB800009F
:10DB9000A40000200A0000000000000045840008E6
:10DBA000343070472DE9F05F044688B2A08655B244
:10DBB00084F83650012184F8371082464021E06A0B
:10DBC000FFF77BFA002640223146E06AFFF73EFD70
:10DBD000761C072EF7D3564629463046FBF738FD0C
:10DBE0008346012229463046FBF7D3FA064607460C
:10DBF0004FF001080BEB060910E000BF07EB8701AF
:10DC000004EB8100434636A2142100F221100EF0ED
:10DC1000EFFD08F1010000F0FF087F1CB945EDD8C9
:10DC2000691E5046FBF714FD0025801B401CC7B23F
:10DC300013E000BF05EB850104EB81003B4628A201
:10DC4000142100F221100EF0D3FD4022E91DE06AFC
:10DC5000FFF7FCFC7F1CFFB26D1CB542EAD306EB5C
:10DC60000B05012713E000BF05EB850104EB8100E4
:10DC70003B461BA2142100F221100EF0B9FD4022F8
:10DC8000E91DE06AFFF7E2FC7F1CFFB26D1C2A2D44
:10DC9000EAD32046FCF7D1F8E06AFFF7C9FCA0F50B
:10DCA0007F41FF3903D0F11DE06AFFF7F3FD204605
:10DCB0000BF05DFF20460AF00FFB064600250BE047
:10DCC000294620460AF0C9FAE16A814203D0224679
:10DCD00020210CF0FCFF6D1CB542F1D3BDE8F09F94
:10DCE00025640000018680F8322080F83330FCF78C
:10DCF000A4B810B50C46142104F12C0008F09BFECA
:10DD0000182104F1380008F096FE00206064606578
:10DD1000A064A0656420E064E065206520660320BF
:10DD2000A0660520E0660A2020676FF0004060666C
:10DD300094F8740020F00700401C20F0080084F8DC
:10DD4000740010BD70B50C4601F12C0617E000BF41
:10DD500008F054FE050012D0287C400702D4686801
:10DD600006F072F9287C800702D4286806F06CF966
:10DD70002946304608F00CFF284606F065F9206B6E
:10DD800000283046E4D108F019FE04F1380509E016
:10DD900008F034FE06460146284608F0F9FE3046F3
:10DDA00006F052F9E06B00282846F1D1BDE870403A
:10DDB00008F004BE2DE9FC410E4649480AF037FA46
:10DDC000012864D1304605F0ADFE0546304605F029
:10DDD000ADFE0446012D11D0082D5AD01A2D56D172
:10DDE000304605F0DAFE054601462046F7F73BFED1
:10DDF00004F12C0008F094FE98B36AE007F004FAEE
:10DE0000694607F01FFA009960692546081A0090D4
:10DE100028460AF0D5FB0099471828460AF0BBFAB5
:10DE20000646002128460BF02CF9381A4FF000075F
:10DE30001CD4B04202DD2F6F7F1E17E095F87410DE
:10DE400001F00701012902D002290BD00EE0296F51
:10DE5000491E414306EBD67001EB6000B0FBF6F7BC
:10DE600004E01DE0296F4143B1FBF6F7606EB84254
:10DE70000DD039462046FCF72FFE2046616EFCF798
:10DE80002BFE20460022202167660CF020FFBDE813
:10DE9000FC81616EFCF720FE6FF000406066F6E7E3
:10DEA00094F8740000F00700012804D0022807D07D
:10DEB00003280AD00DE029462046F9F77CFF08E048
:10DEC00029462046F9F77FFE03E029462046FAF767
:10DED00039F929462046BDE8FC41F7F7DFBC0000D0
:10DEE000C0EA02082DE9F04F8BB017460E46050038
:10DEF0001C4609D04EB1286FB84207D800202060D8
:10DF000058600BB0BDE8F08FFEE7FEE728460AF048
:10DF100042FA804628460AF02DFA059095F87400DA
:10DF200000F00700012804D0032809D0022817D0E8
:10DF30005EE0296F08FB07F0491EB0FBF1F056E0E8
:10DF4000CDF80080317C3068C1F3C00205EB82015E
:10DF500050F82700CA6D496D002308F087FE46E09F
:10DF600005F12C000490069008F04CFD82464FF419
:10DF7000A02128460BF073F80890002128460BF0EA
:10DF80006EF801460290286F4FF0000BC0F10103BC
:10DF900003FB0181B1FBF0F9A8EB09017943401EB5
:10DFA000B1FBF0F02060069808F041FD06E0B142B8
:10DFB00006D00BF1010B049808F036FD0100F6D1F4
:10DFC0000299CAF1010308EB0100296F7843B0FB05
:10DFD000F1F009FB0BF1B1FBFAF10144089800FBE9
:10DFE0000392B2FBFAF000EBD07001EB600020600E
:10DFF000002128460AF06DFF8046002128460BF0DC
:10E0000040F8216840440844206028460AF0D8FAC5
:10E010002168081A206095F87400000701D4F068A0
:10E0200000E00020C119286F059BB1FBF0F200FB56
:10E030001210716851F82000317CC1F3001205EB19
:10E0400082014A6CC96C801A5843891A90FBF1F01E
:10E05000181A6060002128460BF05BF861684044A4
:10E060000844606028460AF06DFB6168081A606029
:10E0700047E7000010B50CA0C86201200C460863F9
:10E080000221204609F065F90821204609F061F9CE
:10E090004FF48061204609F05CF92046BDE810404D
:10E0A00010210CF059BB0000436865636B20626F60
:10E0B0007800000010B591F830000C46C00704D17C
:10E0C000E06A05F0C1FF0020E06210BD2DE9F04FCD
:10E0D000CFB0054605F02AFD0446284605F05DFD53
:10E0E0004390002120460BF028F93B9005F0A1FF5A
:10E0F00005462046002127220BF020F8C0B2012857
:10E1000014D000272046002130220BF017F80646D5
:10E11000002120460BF000F800EB06084FF000014C
:10E1200020462FB10AF0CEFF064604E00127E9E7BA
:10E130000AF0AAFF0644002120460AF093FF834616
:10E140004FF4003120460AF09FFF82464FF4003121
:10E1500020460AF0B7FF81464FF4003120460AF00E
:10E16000DBFF40904FF4003120460AF05DFF029043
:10E17000204668224FF400310AF0E0FF019020466B
:10E1800069224FF400310AF0D9FF00901EA802F076
:10E19000F5FE1EAA4FF4003120460BF05AFB57B192
:10E1A000E069801B411BA1EB0A010590A1EB09006E
:10E1B000401C039008E060693044421903900AEB68
:10E1C00009001044401E0590A16901EB08004219A6
:10E1D00004900299409808441044401E0690039809
:10E1E000459004984690059847900698DDE90021EF
:10E1F000489045A8FEF716F945AA1EA9439802F0D3
:10E20000A7FC002120460BF0BCF806460021204662
:10E210000BF0A8F8034600206FF060410096CDE9AE
:10E220000110E16A49A83B9A0FF0C8FC09A801F067
:10E2300065FE09AA002120460BF04DFAE06A109015
:10E2400003A8FEF7DBF8401B00EBD07040103FB195
:10E25000039AA2EB0B01499A3E91891A3C9106E080
:10E26000059A02EB0B01499A3C9111443E91A26937
:10E27000404410444A993D9008443F903CAA09A963
:10E28000439801F00AFE4FB0BDE8F08F2DE9F04F42
:10E2900085B00F463B4809F0CAFF012861D13846D6
:10E2A00005F040FC0546384605F040FC04464FF4B6
:10E2B0000036312D09D0182D56D01A2D51D105B068
:10E2C0003846BDE8F04FFFF701BF384605F076FC51
:10E2D0000546002120460BF030F8814605F0A9FEE6
:10E2E0000746002120460BF04CF8804600212046CE
:10E2F0000BF038F800216FF06042CDF80080CDE9D6
:10E30000012103464A4603A8E16A0FF057FC0021A9
:10E3100020460AF0A7FE8346314620460AF0B4FEA6
:10E320008146314620460AF0CDFE824631462046DF
:10E330000AF0F2FE8046314620460AF075FE01469C
:10E3400007EB0800084407EB0902039902EB0A03F4
:10E350005A1802EB0B0129600499884200DC084638
:10E36000686005B0BDE8F08F384605F027FC05462B
:10E370003146204609F0D5FA2968814200DD084679
:10E380002860EEE7E4EA0208F0B5184D0446C1F350
:10E3900041706E1064274FF0805C012809D121F094
:10E3A000C040A84205DC604500DB301A584390FBB2
:10E3B000F7F1C2F34170012809D122F0C040A84210
:10E3C00005DC604500DB301A584390FBF7F29442BD
:10E3D00001DA204600E01046884201DA0846F0BD26
:10E3E000944201DA2046F0BD1046F0BDFEFFFF1F4B
:10E3F000F0B5184D0446C1F341706E1064274FF01C
:10E40000805C012809D121F0C040A84205DC6045AC
:10E4100000DB301A584390FBF7F1C2F3417001283A
:10E4200009D122F0C040A84205DC604500DB301A6B
:10E43000584390FBF7F2944201DA204600E0104680
:10E44000884201DA0846F0BD944201DA2046F0BD68
:10E450001046F0BDFEFFFF1FFF2916D0B1B10288A4
:10E46000D30A13FB01F31B0A63F3CF22C2F3451354
:10E4700013FB01F31B0A63F34A1202F01F0313FBA1
:10E4800001F1090A61F304020280704702220021AF
:10E4900008F0E5BC10B50346FF2A13D09AB18B42B1
:10E4A00010D041EA0140121D0849D40843EA034252
:10E4B00008400A40121A624300EB5210084040EA3A
:10E4C000104080B210BD084610BD00001FF8E007E4
:10E4D000002208B51146104600F077F80090BDF80C
:10E4E00000009DF8021040EA014008BDC0F307415A
:10E4F000C2B201EB410101EB8201C0F307200844E5
:10E50000C0F3C700704738B50C460546FFF7E0FF7B
:10E510002246294600F064F80090BDF800009DF8FE
:10E52000021040EA014038BD10B50C4600F0A2F8D8
:10E530000346204600F09EF8834201D1012010BD21
:10E54000002010BD01607047801F102817D2DFE83F
:10E5500000F00E080A0C0E080A0C0E121414101209
:10E5600010100120704702207047042070470820D7
:10E5700070471020704718207047202070470020F7
:10E58000704700B5FFF7E0FFC01DC00800BDC01F09
:10E590000F280BD2DFE800F0080808080808080870
:10E5A0000A080A0A0808080001207047002070477E
:10E5B00008B5020A8DF80120C0F307418DF800006C
:10E5C000BDF8000040EA014008BD08B503468DF8DB
:10E5D00001108DF80020BDF8000040EA034008BD9E
:10E5E00078B5C1F30744C2F1FF0314FB03F4C0F391
:10E5F000074515FB024404EBC41505EBC434C4F312
:10E60000C754C1F3072515FB03F5C0F3072616FB16
:10E61000025505EBC51606EBC535ED0D8DF801501D
:10E62000C9B211FB03F1C0B210FB021000EBC01124
:10E6300001EBC030C00D8DF80000BDF8000040EACD
:10E64000044078BDC178FF290FD079B1827812FBE0
:10E6500001F2120A8270427812FB01F2120A427031
:10E66000027812FB01F1090A0170704704220021AF
:10E6700008F0F5BBC0F30721C0F30742090201EB24
:10E680000241C0B208447047010C01F0F8010902D0
:10E69000020A02F0FC0201EBC201C0B201EBD000A1
:10E6A00080B27047FF2208B511461046FFF78DFF74
:10E6B0000090BDF800009DF8021040EA014008BD3E
:10E6C0002DE9FC5F05000C9C74D04FF48067BD42BF
:10E6D00070D001EB4108581A00EB4001A1EB08098A
:10E6E000C8F58061A01AA1EB090B02EB420A00EB0E
:10E6F0004001A1EB0A00CAF580610090081A2C467F
:10E700000026019043464A4659462046F6F731FC1A
:10E71000401B002801DD014600E04142012940DDA7
:10E720000BFB04F101EB4101891201EB490161434B
:10E7300008EBA122002A01DD114600E05142012927
:10E740000CDDC117890241EA90518002D317F1F71D
:10E750008AFE18B1241A761C082ED3DB00262C0062
:10E7600001D534461DE0BC4201DD3C4619E043467C
:10E770004A4659462046F6F7FCFB411B002900DCBF
:10E78000291A01290DDD854201DD264600E02746D4
:10E79000B81B00EBD07006EB6004B44201D0BE425F
:10E7A000E5DBDDE9002102B053462046BDE8F05F1D
:10E7B000F6F7DFBBBDE8FC9F18B100F5387005F037
:10E7C00093B9FEE72DE9F843DFF8788107460E4656
:10E7D00008F1040008F037F904007CD04FF44471CC
:10E7E00008F06DFB4FF0FF302760C4E901600025A1
:10E7F000C4E903056561A06B40F48030A06382200A
:10E80000A061122084F83B004C2008F01BFAC4F8E9
:10E81000A802011E76D0D4F8AC220AB12046904757
:10E82000D4F8A8027F1E761E4560D4F8A802856041
:10E83000D4F8A802C760D4F8A8020661D4F8A812D8
:10E8400094F83B0008750120C4F8600210F082F8CB
:10E85000C4F8FC02102104F5197008F0ECF8D8F89F
:10E8600014604546224621213748C8F8144010F06C
:10E87000BBF8C4F8F80278B310F040F868B30FF0B2
:10E88000B5FF00BFC4F8F402002009F0B9F9C4F8DC
:10E89000C402002004F52E7409F0B2F9A060002033
:10E8A00009F0AEF96060002009F0AAF92060E06884
:10E8B0000CF052F860680CF04FF820680CF04CF83F
:10E8C000022160680BF048FF022120680BF044FF32
:10E8D0000021E06802E014E015E015E00CF035FBE3
:10E8E000002160680CF031FB002120680CF02DFB4A
:10E8F000A068A4F52E740BF03AF96E61A6B114E08D
:10E9000000E0FEE7FEE7FEE700200CF047FE0746CA
:10E9100005200CF043FE01460C48009000233A46C7
:10E9200020460FF06FFFADE76C61002335220849E8
:10E930002046FFF741FFD4F8F80210F062F92046B4
:10E94000BDE8F883AC500020B9EA00089CE4020856
:10E95000C54E000818B907484069002809D0D0F80A
:10E96000602209B1012101E04FF0FF311144C0F8EC
:10E9700060127047AC500020002101637047000016
:10E9800018B903484069002801D090F83B0070474F
:10E99000AC5000200148406970470000AC50002096
:10E9A00010B90348406908B18069704782207047F8
:10E9B000AC50002018B908484069002808D090F8E9
:10E9C000F01201F00701012903D0032901D00068EA
:10E9D0007047406870470000AC50002018B90348E9
:10E9E0004069002801D0D0F8C4027047AC50002024
:10E9F00018B903484069002801D0D0F8B802704720
:10EA0000AC50002018B903484069002801D0D0F864
:10EA1000BC027047AC5000200100034801D007F051
:10EA2000FFBF07F0EBBF0000B050002018B903484B
:10EA30004069002801D0D0F8C0027047AC500020D7
:10EA400018B903484069002801D0D0F8C8027047BF
:10EA5000AC50002008B902484069D0F8F402704771
:10EA6000AC50002018B908484069002808D090F838
:10EA7000F01201F00701012903D0032901D04068F9
:10EA80007047006870470000AC500020006A002802
:10EA900000D001207047000018B9064840690028DE
:10EAA00004D0D0F86002002801DD0120704700206A
:10EAB00070470000AC5000202DE9F041434C28B1D4
:10EAC000C168216110F096F8206902E0FFF762FF4B
:10EAD0002061002878D0416A002975D00A69002A8F
:10EAE00072D0C96800296FD00022362100F070F87A
:10EAF0002069D0F8C0020CF0F3FC2069D0F8C802FD
:10EB000008B10CF0EDFC2069D0F8C4020CF0E8FC70
:10EB10002069D0F8BC020CF0E3FC2069D0F8B80200
:10EB20000CF0DEFC20690026D0F8C012B9B10DF05F
:10EB30001BF812F0A9FA11F0EFFF2069D0F85C126F
:10EB400079B10022392100F043F82069FFF79EFFD8
:10EB500048B3206990F8390001280BD023E0C0F8B1
:10EB60005C6203F0FDFE2069BDE8F0410022372120
:10EB700000F02EB800254FF03C080FE005F50F71AE
:10EB8000415C51B900F5197007F0ACFF226908EB40
:10EB9000051111448EC980E88E006D1C2069D0F8E3
:10EBA0005C12A942EAD820694FF4007200213C307F
:10EBB00008F055F920692022002100F50F7008F0B7
:10EBC0004EF92069CBE7FFE7BDE8F081AC500020AB
:10EBD00070B588B00E46044615461C21684608F0FC
:10EBE0006EF9009404F538700194ADF808600122C4
:10EBF00069460495044605F02FF8012804D1002247
:10EC00006946204605F028F808B070BD2DE9FF5F81
:10EC10001F46DDF838B016465FEA0108814616D077
:10EC20004846FFF7ADFE03904846FFF7C3FE824615
:10EC30004846FFF717FF0546BAF1000F08D03DB16F
:10EC40004046039900F052FB404502D0FEE7FEE744
:10EC5000FEE736B13046039900F048FBB04200D0E1
:10EC6000FEE75046039900F033FE0446BBF1000F67
:10EC700004D004FB05F0B84203D9FEE7B7FBF4F576
:10EC8000B5B1CDE9004809F51C7002972A465146F6
:10EC90008046039B00F002FD8DE8D00009F523704B
:10ECA0002A4651460446039B00F0F8FC16B900E0E2
:10ECB000FEE7002422464146484600F007F804B02B
:10ECC00059464846BDE8F05F00F016B818B9044848
:10ECD0004069002802D0C0E9071241627047000075
:10ECE000AC50002018B903484069002800D0816268
:10ECF00070470000AC50002018B903484069002854
:10ED000001D080F839107047AC50002010B50400D5
:10ED100003D113484469002C21D0C4F8F412D4F86C
:10ED2000D00204281BD1D4F8B402006809F0D4FA48
:10ED3000002814D1D4F8B402406809F0CDFA0028B4
:10ED40000DD1D4F8B402806809F0C6FA002806D1C3
:10ED5000D4F8B4020068BDE810400FF037BD10BD14
:10ED6000AC50002000B501004FF000000ED0FFF7BE
:10ED700017FE48435030B0F5A07F08DB0020FFF7B6
:10ED80000FFE4843A021503090FBF1F000BD012060
:10ED900000BD70B504460D46542007F053FF95E8BA
:10EDA0004E0008304EC02ECD80E82E0004F1180130
:10EDB00020302EC92EC0012140F84819A16B11B98D
:10EDC000A06370BD11460A68002AFBD1086070BDBF
:10EDD0007FB5064691F83C000C4602282AD9206AE5
:10EDE000002827D0D4E90901884223D0A08EE16A07
:10EDF000091A0091216B081A0190A18EE06A08445B
:10EE0000401E0290A18E206B0844401E039069466C
:10EE10003046FFF7BEFF0546402007F0EFFE4022D8
:10EE20002146E86407F060FF082028712946304633
:10EE300000F048FE7FBD38B504464022002108F0AE
:10EE40000EF801202062FF2084F83C00FFF740FB11
:10EE50000090BDF80000A0839DF80200A07740203C
:10EE6000606138BD2DE9FF5F8246DDE910E48B4625
:10EE7000DDE90E800AEB020C03F5B475CDF804C091
:10EE80001E460BEB020C9146AAEB0203ABEB02070A
:10EE9000CDF808C0A84505D1C4E900370198A060A5
:10EEA000029815E14FF4B475AE4201DDA6F5B476D3
:10EEB000A84501DDA8F5B478A9EB000100915FEA4F
:10EEC0000E0104D000EBD07045106D1C00E0002551
:10EED0005A2196FBF1F098FBF1F1C0B2C9B20428B7
:10EEE00000D10320042900D10321884279D146456D
:10EEF00077DC38B301284AD0022874D003286ED1B9
:10EF000006F15A0000B20FF0ABFF009948430AEB3C
:10EF1000E030401B206030B20FF0A2FF00FB09F090
:10EF20000BEBE030401B606008F15A0000B20FF0BC
:10EF300097FF00FB09F00AEBE0302844A0600FFACD
:10EF400088F021E130B20FF08BFF00995A36484328
:10EF50000BEBE030401B606030B20FF081FF00FB34
:10EF600009F00AEBE0302844A0600FFA88F00FF0B7
:10EF700077FF00FB09F00BEBE0302844E06008F17C
:10EF80005A0000B20FF06CFF0099484323E030B202
:10EF90000FF066FF00FB09F00BEBE03028445A3617
:10EFA000E06030B20FF05CFF009948430AEBE030BC
:10EFB0002844A0600FFA88F00FF052FF00994843F0
:10EFC0000BEBE030401B606008F15A0000B20FF01C
:10EFD00047FF00FB09F00AEBE030401B2060BDE872
:10EFE000FF9F2AE0FFE706F15A0000B20FF038FF5A
:10EFF00000FB09F00AEBE030401B206030B20FF05C
:10F000002FFF009948430BEBE0302844E0600FFAF3
:10F0100088F00FF025FF00FB09F00BEBE030401B00
:10F02000606008F15A0000B20FF01AFF00994843DF
:10F030000AEBE0302844A060D1E7C8B1012849D0EC
:10F04000022872D003287FF427AF0029FBD108F1F2
:10F050005A0000B203900FF003FF074606F15A0072
:10F0600000B202900FF0FCFE87427CDA039893E036
:10F070000129E8D108F15A0000B20FF0F1FE00FBBF
:10F0800009F00AEBE030401B20600FFA88F0019095
:10F090000FF0E6FE074630B280460FF0E1FE8742F1
:10F0A00001DA019800E040460FF0DAFE00995A3686
:10F0B00048430BEBE030401B606030B20FF0D0FEF5
:10F0C00000FB09F00AEBE0302844A06002982844D5
:10F0D000E06084E70229B6D1581B20600FFA88F05F
:10F0E0000FF0BEFE00FB09F00BEBE030401B606050
:10F0F00006F15A0000B201900FF0B2FE074608F187
:10F100005A0000B280460FF0ABFE874201DD019845
:10F1100000E040460FF0A4FE009948430AEBE030BF
:10F120002844A06030B24DE0FFE703298BD106F1FF
:10F130005A0000B20FF094FE00FB09F00AEBE03039
:10F14000401B2060781B606008F15A0000B20FF08D
:10F1500087FE00FB09F00AEBE0302844A0600FFABC
:10F1600088F0804600E016E00FF07AFE009900FB80
:10F1700001F730B206460FF073FE0099484387420C
:10F1800001DD404600E030460FF06AFE009948433A
:10F190000BEBE0309BE702980FF062FE00994843CA
:10F1A0000AEBE030401B206030B20FF059FE00FB4C
:10F1B00009F00BEBE030401B606001982844A06030
:10F1C0000FFA88F00FF04CFE00FB09F0E0E710B5F5
:10F1D00004462C2107F07BFEFF2084F828000F2036
:10F1E00084F829002C20606110BD2DE9F0470D4600
:10F1F00004000AD0206948B1606887B2060C206814
:10F20000010C890626D515B107E0FEE7FEE7C0F33D
:10F210000721384600F05CFB0546208980B2A842F1
:10F2200002D10120BDE8F0872088C0F30720FFF756
:10F230008BF97843C01D4FEAD00A55450AD3208880
:10F240002B46C0F3072231463846F3F7B2FFE16898
:10F25000814201D20020E5E72088C0F3072007287B
:10F2600017D0082817D0092817D00A2817D000204F
:10F27000218980008BB2AB4223D2711E2269002704
:10F2800003FB012305FB012103EB00090844804631
:10F2900014E00220ECE70420EAE71020E8E74FF44E
:10F2A0008070E5E75246494607F0B8FD20897F1C8B
:10F2B00081B2A8EB0500A9EB01098046B742F1D362
:10F2C00012E02169002708448146C8460AE05246F8
:10F2D000494607F0A3FDA16819FA81F908EB05007A
:10F2E00080467F1CB742F2D325819AE70A46014641
:10F2F000014800F003B800007451002030B4836866
:10F300000C461BB1204630BC1146184730BC0020CB
:10F310007047F0B589B0040035D0208986B289B332
:10F32000002004900590A0884FF0FF3280B2401E6C
:10F330000690606802EB1040079004AA6846FDF74B
:10F340007EF800282AD06846FDF767F8002825DDFA
:10F350006846FDF753F8002820DDDDE9001220465D
:10F3600000F056F905462088C0F30720FFF7ECF8B7
:10F3700004466846FDF751F800FB04F1C91DCF10A3
:10F38000019C13E000E0FEE700221146204600F059
:10F390003FF96168090C714307F095FD09B0F0BDB4
:10F3A0003946284607F08FFD3544641C0398A04277
:10F3B000F6DAF3E72DE9F05F044600880D46C0F366
:10F3C000072110881F46C0F307209146814200D0D4
:10F3D000FEE72DB12846FDF720F8064617B117E0E5
:10F3E000A08886B22088C0F30720C11F03290ED849
:10F3F000072813D0082813D0092813D00A2813D0BF
:10F4000000208200D9F81010206907F06DFC77B158
:10F410003846FDF702F8B0421ED0FEE70220F0E7C2
:10F420000420EEE71020ECE74FF48070E9E7B9F82C
:10F43000040080B2B042F0D100221146484600F0EC
:10F44000E7F880465DB1D5E90012204600F0E0F80B
:10F450006F688246ED680DE0D7E90012EEE7002202
:10F460001146204600F0D4F8824600276068791ED5
:10F4700001EB104520891FFA80FBB9F808001FFA3C
:10F4800080F92088C0F30720FFF75EF87043C01DA5
:10F49000C41007E022464146504607F025FCDA44F6
:10F4A000C8447F1CAF42F5DDBDE8F09F08B500936E
:10F4B00013460A460146024800F004F808BD000061
:10F4C000745100202DE9F05F81461D4693468A461F
:10F4D0001C20DDF8288007F0B5FB040003D0B8F14C
:10F4E000000001D005E0FEE72946504600F0F0F9A3
:10F4F000804603462A4659465046F3F75AFED9F845
:10F50000002007462946CAB19047060016D0A4F845
:10F5100004A0A4F806B0657030206080A4F80880CC
:10F520001920207029463046FFF7E0FE04F1100153
:10F53000E76081E841022046BDE8F09F204604F0E4
:10F5400083FD0020F8E710B504000FD02068000C00
:10F55000C0060DD5A06950B1616942680AB108467C
:10F5600090472046BDE8104004F06EBDFEE7FEE780
:10F5700010BD38B50C46098989B200912188C1F3C4
:10F58000072361680A0C89B2FFF79CFF051E11D0A2
:10F5900020683021000C6880286841EA10406880AB
:10F5A000E068EA68904200D202462169286907F0C3
:10F5B0009BFB284638BD7FB5050006D0AC692CB151
:10F5C000206900280BD011B106E0FEE7FEE769468E
:10F5D0002846F6F7CBF869462269284690477FBD52
:10F5E0003EB50C460546D4E90301228992B2009249
:10F5F000CDE901102088C0F307236068020C81B2B6
:10F60000284600F04BF82068000C68803EBD0000E2
:10F6100070B50C4603001AD018881969C0F307208A
:10F62000072815D0082815D0092815D00A2815D084
:10F630005FF000051B8901EB85019BB203FB0215FE
:10F640007CB1FEF781FF604305EBD00070BDFEE7A3
:10F650000225EFE70425EDE71025EBE74FF4807571
:10F66000E8E7284670BD2DE9F0470F4608A91D467A
:10F6700091E8000716460446182107F024FC04F11F
:10F68000080181E82007C4E90076BDE8F08700683A
:10F6900011EA104000D00120704700002DE9F0472A
:10F6A000894608A99A4691E860011746040004D0EB
:10F6B0001C2107F008FC0DB105E0FEE75146484665
:10F6C00000F006F9054605FB07F0404502D9002089
:10F6D000BDE8F087A4F80490E78084F801A02581B4
:10F6E0000020608019202070C4E903860448514638
:10F6F000C4E905603046FFF7F9FD0120E8E70000A6
:10F700007451002010B5064800F00CF80448183079
:10F7100000F008F80248BDE81040303000F002B8B0
:10F72000745100200EB5054A00210091CDE9011267
:10F73000034B044A0449FFF796FF0EBDBF6A020857
:10F74000953B0008A13B0008A53B00082DE9FC5FA4
:10F75000040004D02168080CC20703D100E0FEE7D2
:10F76000800602D40020BDE8FC9FC1F30720C11F22
:10F7700003291DD8072809D0082809D0092809D04D
:10F780000A2809D00026002527690EE00226FAE79C
:10F790000426F8E71026F6E74FF48076F3E700BF7B
:10F7A00007EB8500FEF74EFF6D1CB542F8DB63E00A
:10F7B000102804D014281DD0132842D05CE06068C3
:10F7C00000274FEA104A1FFA80F82089D4F81090D9
:10F7D0001FFA80FB0BE04D46002604E02846FEF7AA
:10F7E00031FF2D1D761C4645F8D3D9447F1C574563
:10F7F000F1D341E060684FEA10491FFA80FA20898E
:10F8000080B20090400801902569009800FB095BD8
:10F81000002012E02F46002607E000BF1BF806106C
:10F820003846FEF719FE761CBF1C5645F6D30098E5
:10F8300005440198834408F1010080464845E9D316
:10F840001AE0606800274FEA104A1FFA80F8208902
:10F85000D4F810901FFA80FB0CE04D46002605E01E
:10F86000A9782846FEF7F8FDED1C761C4645F7D32F
:10F87000D9447F1C5745F0D32068012141EA10404C
:10F88000608008466FE72DE9F0419846069D1746CF
:10F890000E46040012D016B92088C0F3072625B9F9
:10F8A0003146104600F014F805462B4632464146D4
:10F8B0003846F3F77EFCE168814202D20020BDE8C1
:10F8C000F0816670A780A4F8068025812046F6E7BF
:10F8D0000A460146014800F003B8000074510020B8
:10F8E00030B443690C461BB1204630BC1146184762
:10F8F00030BC00207047000010B507F0A3F906499E
:10F90000D1F824210260C1F82401D1F82821521C29
:10F91000C1F8282110BD0000AC5000202DE9F041B5
:10F9200000263046FFF778F805460127DFF83080DB
:10F9300012E0D5F8A84206E02146284600F012F869
:10F9400000B10126246C002CF6D10EB9C8F8307134
:10F950002846FFF761F80546002DEAD1BDE8F081A1
:10F96000AC5000202DE9F05F00270E468346DFF8FB
:10F970001091BA468C6B06E02068A16C8046032982
:10F980000ED027464446002CF6D1F06B002520B15E
:10F9900096F8441009B1B16BF1B3D9F8244169E08C
:10F9A0000FB1386001E0C6F83880207906282ED1E2
:10F9B000E06CC569286890B1281DFCF71FFD296817
:10F9C000098989B24843F9F786FDD9F82C21111A23
:10F9D000C9F82C112868FFF7B6FDC5F800A0BBF1E7
:10F9E000000F14D0DBF8A80206E0016CA94202D196
:10F9F000296C016402E008460028F6D1DBF8B02249
:10FA000058460AB129469047284604F01DFB204677
:10FA100003F019FD050000E010E008D095F84C0057
:10FA2000400604D5E86904F00FFBC5F81CA0E06CA3
:10FA300004F00AFB204604F007FBA3E7806B0EE00E
:10FA4000017906290AD1816C41B9C16CC969B142F9
:10FA500004D101218164C9F830110DE0006800284B
:10FA6000EED109E0E268314620469047401C00D0C4
:10FA700001252468002CF5D12846BDE8F09F000040
:10FA8000AC50002002490120C1F83001704700004D
:10FA9000AC5000200448D0F830110029FDD00021DE
:10FAA000C0F8301170470000AC50002010B504467B
:10FAB000302107F00CFAFF2084F82000302060612C
:10FAC00010BD00002DE9F041CE6C1D4D0C4630619B
:10FAD00095F838014FF06408002705F5927520B1BC
:10FAE00084F8518084F8507024E0306860B14FF49D
:10FAF000002109F03DFD38B10120287522461F2163
:10FB000030680BF0E4F82F7584F8518084F8507059
:10FB100004E02A6912B12146284690472D68002D3D
:10FB2000F7D1BDE8F041FFF7F9BE2A6912B12146CD
:10FB3000284690472D68002DF7D1BDE8F0810000E0
:10FB4000AC5000202DE9FF4105462F480C461646D3
:10FB5000D0F82811A86B012915D8032209E0816C7F
:10FB600001290BD190F8501041B1B14206D0826406
:10FB700000680028F3D104B0BDE8F081816C012950
:10FB8000F9D00020F7E7D8B10BF0AAFFFEF712FF7B
:10FB900007460BF0A5FFFEF765FF0146A86B826CD8
:10FBA000012A0DD08268002A0ADC02697F1EBA424F
:10FBB00006DBC268002A03DC4069491E8842E0DA9D
:10FBC0000CB1246800E0AC6B002CDAD0A06C0128EA
:10FBD000F7D194F8500008B1B042F2D104F11808FE
:10FBE000AF6B0BE0B86C032807D0424607F1180151
:10FBF0006846FCF724FC0028E3D13F680FB1A74218
:10FC0000F0D12046B7E70000AC5000201C220021B4
:10FC100007F025B92DE9FE438046C86917460C4612
:10FC2000002849D094F84C00022845D9206B0028C0
:10FC300042DD606B00283FDD6C2006F0DFFF0646EA
:10FC40006C22214607F050F806F12001F06904F01B
:10FC500013FF012804D03046BDE8FE4304F0F4B998
:10FC600039464046FFF795F80546C66405202871D9
:10FC70003846FCF7C3FB06463846FCF7CEFB238E1E
:10FC8000A28E01469BB204F1400092B20093CDE9EE
:10FC9000012005F11800E36A3246044604F07DFDB8
:10FCA000D7E900122046FCF70FFD03B02946404675
:10FCB000BDE8F043FFF706BFBDE8FE8338B5044654
:10FCC0006C22002107F0CBF8FEF702FC0090BDF893
:10FCD0000000A4F848009DF8020084F84A00FF20C4
:10FCE00084F84C00401C44F8300F6060A08B40F456
:10FCF0008050A0830248E0626C2044F81C0C38BDA0
:10FD0000010000E02DE9F0419EB01E000D46804646
:10FD1000144653D02068039060680490A068059052
:10FD2000E0680690E86A38B9296B4FF48070814228
:10FD300002D1696B814225D01046FCF76EFB074665
:10FD40002046FCF75BFB2B8EA98E02469BB205F189
:10FD5000400089B20093CDE90110394603A8EB6A4F
:10FD600004F01BFD0398216808440390049861681F
:10FD70000844049005982168084405900698616835
:10FD80000844069003A91AA8D8F80820FCF757FBE6
:10FD9000002813D0002207A8E96904F097FE012883
:10FDA0000CD11AA8CDE90040002307AA29460296E3
:10FDB0004046FAF791F907A804F028FE1EB0BDE806
:10FDC000F08100002DE9FF4FA3B05FEA030916465A
:10FDD0000C465CD0002207A8E16904F077FE0128F8
:10FDE00055D1606A85B2070C04F15400FCF715FB8D
:10FDF000002803DB04F154000FC801E096E80F006F
:10FE00000DF10C0888E80F00294603A8FCF773FCE5
:10FE1000394603A8FCF76AFC1E480DF1680ADDF8B4
:10FE20000C800FC88AE80F002AE0324603A91EA8FA
:10FE3000FCF705FB48B1CDF800A0CDE901B91AAB3C
:10FE400007AA21462398FAF747F903982844039014
:10FE500005982844059003E00DF10C0A0DF1780B8C
:10FE60000398B1688842E0DD0498CDF80C803844EE
:10FE7000049006983844069008EB0500401E059053
:10FE80000498F1688842E7DD07A804F0BFFD27B0B9
:10FE9000BDE8F08F68AF020870472DE9F0410646D3
:10FEA00091F848000C46022826D9E069002823D0A2
:10FEB0000078002820D0206A00281DD01146304646
:10FEC000FEF767FF0546542006F098FE54222146AF
:10FED000E86406F009FF0420287194F84C004006FD
:10FEE00004D5EF6CE0690CF0E5FEF8612946304678
:10FEF000BDE8F041FFF7E6BDBDE8F08138B5044646
:10FF00005422002106F0ABFFFF2084F8480014348F
:10FF1000FEF7DEFA0090BDF8000020839DF8020095
:10FF2000A0761048E0604FF6FF7020616061FEF738
:10FF3000CFFA0090BDF80000A4F81B009DF8020065
:10FF4000607705200BF02AFB0090BDF80000E083ED
:10FF50009DF8020084F82000002084F83500542029
:10FF6000206038BD9CE402082DE9FF4FB5B0086A57
:10FF7000039035980C46379982682DA8FCF75FFAF4
:10FF800000287DD094F84A70E16907B9012794F8F8
:10FF90004B00C20725D0A26B6FF060430092CDE901
:10FFA00001300AA8E36B226A0DF008FE0A98069059
:10FFB000039804F03EF88046A16B379801EB080BDC
:10FFC000D0E9001204A80BF0EEFB206C1290616CDB
:10FFD0000598002508440590206D6E1E08B321B1D8
:10FFE0001FE03798FCF719FAE1E7379949680029CB
:10FFF00017DA83685A1A002A00DCCA1ACBF100010A
:020000040801F1
:100000004FF4806303EB41018A4200DD0660216DFD
:10001000086831B1002804DB0546059849680844A2
:10002000059094F84B100020CDE90001E069E26BE7
:100030002844069B03990DF0B7FC46192CE000BF3D
:1000400094F84B100020CDE90001E069E26B3044E8
:10005000069B03990DF0A8FC35460599461901EB5E
:100060000B000590206D98B1059911F5806F0FDB9D
:10007000016800290CDA056037980599406800E0AE
:1000800087E0081A216D48603798216D40688860C4
:10009000E069405D00287CD0059800EB08013598A8
:1000A000806840688142CBDB0A97022F02D0032F81
:1000B00012D020E0E069711B2844E36B039A0DF035
:1000C000D9FD07463798FCF7A8F9C01B049900EB47
:1000D000D07001EB60000DE0E069711B2844E36B18
:1000E000039A0DF0C7FD07463798FCF796F9C11B38
:1000F000049808440490D4E909708146874202D9E3
:1001000038464F46814626A8FFF780FD94F8480000
:100110008DF8AF0013A8299034F82C0FADF8AC007F
:10012000A0788DF8AE001AA8FFF7C0FC207F8DF8EC
:10013000880003982C3C90F9160000B90120179014
:1001400015E104991298A6EB050A084404900D9055
:1001500000201990E06928440E90C1E00020009032
:10016000A7F57F40FF380AD0A9F57F41FF3906D0B7
:10017000854A199829181268E0699047009019ABD0
:1001800010AA11A90E980DF0F7FBDDE910210398D4
:1001900000E0F6E003F01BFF8046059814900499F8
:1001A000A8F1010001900844139115900599ABF155
:1001B00001000844199916908A4556D894F84C00C5
:1001C000C00723D00D9831900499019831AB0844B1
:1001D0003390039805991AAAC068014403980069EE
:1001E000091A039890F91500081A17993290491EB8
:1001F00008443490A08DADF8890094F82E008DF855
:100200008B00DDF8E0C000213598E04794F84C0001
:1002100080072AD50D9831900499019831AB084494
:10022000339003990398D1E90321511A4A0003211D
:1002300092FBF1F190F916001AAA00EBD07001EBD5
:10024000600005990844014632901798401E084402
:100250003490A08DADF8890094F82E008DF88B00B5
:10026000DDF8E0C000213598E0474FF6FF70874287
:100270001DD081451BD00098B84218D3484516D2EE
:10028000B4F82F00ADF8AC0094F831008DF8AE0052
:10029000608EADF8890094F834008DF88B00DDF89D
:1002A000E0C013AB1AAA00213598E04706E0A08D04
:1002B000ADF8AC0094F82E008DF8AE003899119886
:1002C000CDE9000104AA26A9039B3598F6F724F985
:1002D000B8F1000F04DD0499E06B08444044049039
:1002E00019998A453FF63AAF94F84B100020CDE9B2
:1002F0000001E069E26B3044069B03990DF054FB6A
:10030000354646193798006804900A98022802D0AA
:10031000032813D022E0E069711B2844E36B039AA1
:100320000DF0A8FC80463798FCF777F8A0EB0800A2
:10033000049900EBD07001EB60000EE0E069711BE6
:100340002844E36B039A0DF095FC80463798FCF740
:1003500064F80499A0EB080008440490059901EBA7
:100360000B00359905908968C968884204DCE0690A
:10037000405D00287FF4E5AE2C98002801D0FFF7FF
:10038000E2F839B0BDE8F08F74E902082DE9FE43C8
:100390008046086B0C46164600283BDD606B002843
:1003A00038DD11464046FEF7F4FC05466C2006F0A9
:1003B00025FC6C222146E86406F096FC0620287194
:1003C0000020A8643046FCF719F807463046FCF7D1
:1003D00024F8238EA28E01469BB204F1400092B213
:1003E0000093CDE901203A4605F118000746E36A7B
:1003F00004F0D3F9D6E900123846FCF765F9E06954
:10040000012180F8441003B029464046BDE8F0437E
:10041000FFF758BBBDE8FE832DE9F04104460068B4
:1004200010B10069BDE8F081201DFBF7F6FF07461B
:10043000201DFBF7E3FF0546217D3846FFF748FA0C
:1004400000FB05F6227D002329463846FFF72EF8EB
:1004500020600028E6D03046F9F73DF8014608480C
:10046000D0F82C211144C0F82C11207DFEF78FF814
:1004700018B100212068FEF74CFF2068D1E700008A
:10048000AC5000202DE9F04114460E4607460BF013
:1004900027FB05464C2006F0D5FBB0B1C76394E8B6
:1004A0008E0000F1180888E88E0094E88E0000F1B4
:1004B000040888E88E001ECC00F1280888E81E0099
:1004C0000675D5F8A81211B907E0FEE711460A6CC7
:1004D000002AFBD10864BDE8F081C5F8A802FAE75C
:1004E0000068FFF795B87FB50B6B0C460546002BEF
:1004F00034D094F83C00022830D9E169606A814226
:1005000001DA0A4600E00246A2EB0302009200DD97
:10051000084618440290216AA06A814200DA08461F
:10052000216B401A0190216AA06A814200DD0846D1
:10053000216B0844039069462846FEF72AFC0646CC
:10054000402006F05BFB40222146F06406F0CCFB25
:100550000720307131462846FFF7B4FA7FBD38B521
:1005600004464022002106F07AFC01202063FF208F
:1005700084F83C00FDF7ACFF0090BDF80000A085BA
:100580009DF8020084F82E004020606138BD2DE9FE
:10059000FF4F81B08B460E9D16461C46E9682869C0
:1005A000571AAA6805F11809ABEB020305F1500AC6
:1005B000B4285CDA6A69B42A7DDA00287BD0002A84
:1005C00079D0904277DDB14259DC696F79434FEAC7
:1005D000A12CE96B7F1C79438912A0F20F15582DCD
:1005E00001D8002909DB451E592D01D8002904DB5B
:1005F0005B38B32802D2002900DD0021A2F20F10DF
:10060000582801D8002909DB501E592801D8002993
:1006100004DB5B3AB32A02D2002900DD0021ACEBF7
:10062000010001EB60000125C71AA74200DD274643
:10063000002F0DDD3B4632465946CDF8009001981B
:1006400000F0CDF8050003D13946019806F04BFCC7
:10065000A74200DD2746002F00DA0027CDF800A0D2
:100660005CE0B54274D1284605B0BDE8F08F66DD88
:100670006A69B42A63DD904261DDB14201DA01208A
:10068000F2E7696F79434FEAA12CE96B7F1C79434C
:100690008912A0F20F15582D01D8002909DB451E3B
:1006A000592D01D8002904DB5B38B32802D2002978
:1006B00000DD002100E042E0A2F20F10582801D82E
:1006C000002909DB501E592801D8002904DB5B3AB8
:1006D000B32A02D2002900DD0021ACEB010001EBBE
:1006E00060000125C71AA74200DD2746002F0DDD57
:1006F0003B4632465946CDF800A0019800F06FF80D
:10070000050003D13946019806F0EDFBA74200DD54
:100710002746002F00DA0027CDF800900198E31B50
:100720000BEB070138441C460746324600F057F8E9
:10073000060096D12146384606F0D5FB91E7012701
:10074000B846B42805D038B109DAB14209DC0AE06C
:1007500043E0B14210DC04E0B14202DC0CE0B14203
:1007600001DC032708E0234632465946CDF80090C5
:10077000019800F034F807466869B42805D050B1F4
:10078000E8680DDAB04203DC0CE0E868B04205DD51
:100790004FF0030802E0E868B042F9DDBFB10EE0B7
:1007A000B042F5DD234632465946CDF800A0019807
:1007B00000F015F8804657B1B8F1000F07D0032FAD
:1007C00002D0012F05D008E0B8F1030F05D10020B9
:1007D0004AE74046B8F1010FFAD0022044E7F8B5E5
:1007E000069C256AE66A521BE569491B94F8345059
:1007F0004FEAC57526B1009485B3FAF7DFFCF8BD62
:1008000085B1207E810727D000F00301012923D084
:10081000022901D1002A1FDBC043800728D1002A0A
:100820001ADC25E0227E02F00304022C14D0D5430A
:10083000AD0711D0012C01D100290DDC920701EB8D
:10084000030207D0002A13DB49420FD50021002BF9
:100850000EDD0FE0002A02DA0120F8BD10E04A4266
:1008600006D49A420ADA991A104405E0994201DB4B
:100870000020F2E7994201DA06F035FB0220ECE7AE
:10088000FAF746FDE9E72DE9F04F8DB08046DDF837
:1008900058900E461C4699F81C00174600F0010AB5
:1008A00007A809F10801D9F81850FBF70FFD0898BF
:1008B000BAF1000F29D0B84249DC0A98B84246DBA9
:1008C00007984119B14204DC099A3119521B91422F
:1008D00007DD08992944B9423DDC0A99491BB94210
:1008E00039DBBAF1000F16D0801B00D50020A042E2
:1008F0002FDC0999891B091A491C4218A24200DD04
:10090000211A002925DB4044E3E0B84211DC0A98B3
:10091000B8420EDBD4E7871BA7420ADC002F03DBBB
:100920003946404606F0DFFA0998851B6D1C002DFC
:1009300003DC00200DB0BDE8F08FA54204DA611B96
:1009400008EB050006F0CFFA1FB9A54201D101203E
:10095000F0E70220EEE7801B019007A8FBF75DFDA2
:10096000069007A8FBF74AFD0899791AA94202DA0E
:10097000681A401E01E0401B081AD9F82010022313
:1009800003EB4003CA684FF00007D35A32F8102037
:100990009E1A8B68496802EB010B069A019933F89D
:1009A00010001144491B01EB0009019929440D1A5B
:1009B0006D1EBAF1000F21D069E0F11B01EB0B00B5
:1009C00010F8010C049009EB07005FEA000A08D454
:1009D000A24506DA18F80A1004980EF067FD08F828
:1009E0000A00B5EB070A08D4A24506DA18F80A107F
:1009F00004980EF05BFD08F80A007F1CB742DCDBB0
:100A000009EB0700A04201DA014600E02146002977
:100A100001DA002002E0A04200DB2046211A404417
:100A200006F061FAA91B481CA04201DA4A1C00E04A
:100A30002246002A01DA002104E0A04201DA491C22
:100A400000E02146404644E0F11B01EB0B0010F8AA
:100A5000010CC0F1FF00049009EB07005FEA000AF7
:100A600008D4A24506DA18F80A1004980EF01EFD04
:100A700008F80A00B5EB070A08D4A24506DA18F808
:100A80000A1004980EF012FD08F80A007F1CB74205
:100A9000DADB681CA04201DA691C00E0214600296B
:100AA00001DA002504E0A04201DA6D1C00E02546D1
:100AB000A9EB0501621B914201DA084600E01046ED
:100AC000002801DA002102E0914200DB114608EB28
:100AD000050006F008FA3CE72DE9F0410546884696
:100AE000007DFDF754FD00282CD0291D2846FEF777
:100AF00050F90446302006F081F830224146E06487
:100B000006F0F2F80A202071E66C3561306898B181
:100B10004FF40027394608F02BFD68B1394630689C
:100B200009F01AFE22461F21D8F800000AF0CFF87B
:100B30003946306806F00DFC21462846BDE8F041F4
:100B4000FEF7C0BFBDE8F0813022002106F087B972
:100B50002DE9F74FC86D8CB00C4698B194F86C1025
:100B600002290FD9012806D1A06E002803DC206ECF
:100B700008B9606E30B1012194F82000022803D832
:100B8000002202E00021F7E70122904694F83B2082
:100B9000022A24D9226B12B30122914694F84820EC
:100BA000022A1ED9626CE2B194F84920930618D447
:100BB000D20616D00122924694F85820022A12D961
:100BC000226D82B1012201279346FF2815D394F8A4
:100BD0002F00400716D0002094F82E2010E00022AD
:100BE000DBE70022E7E70022EDE700BF00EB800330
:100BF000234493F82730FF2B01D0002702E0401C4C
:100C00008242F3D8E9B30E990C98FEF7C2F8064673
:100C1000382005F0F3FFF0640546A16E06F11800D8
:100C20000A460090FBF7FEFBE16D00980A46FBF7D1
:100C3000F9FBD4E918120098FBF746FD1C22214667
:100C40002846EFF779FC38206861E069E861B4F87C
:100C50005900288494F85B0085F82200E06D6862F2
:100C6000A06EA86294F86C0085F83400206EE862EB
:100C7000606E286385F835700320307131460C981A
:100C800000E001E0FEF71EFFB8F1000F55D00E980E
:100C900090E80E00C068CDE90012CDE90230606C2A
:100CA00001281DDD94F84800FD2819D3E069B8B18A
:100CB00094F84900C0F38002114400910199C0F3F7
:100CC00040000844019094F84900C0F3C000181A8D
:100CD000029094F84910039801F00101401A039022
:100CE00069460C98FEF755F80646302005F086FF59
:100CF0000546FEF7DBFE1C2221462846F564EFF789
:100D00001BFC302045F8140FE069A860B4F82100FE
:100D1000A5F80D0094F82300E87304F1240005F110
:100D2000100307C883E8070094F820002873012007
:100D3000307131460C98FEF7C5FEB9F1000F7DD039
:100D4000206B04F051FA06004FF0000508D0012E88
:100D500006D0032872D00C2103A806F0B8F808E0EA
:100D600003A9206B03F088FE012867D1D6B3012EBA
:100D700039D06FF06040CDE900500295D4E90C12F3
:100D800000230AA80CF01AFF0A980695401E089046
:100D90000B980795401E09900023092206A900958B
:100DA0000E98FBF795F906A90C98FDF7F2FF064699
:100DB000542005F023FF0546FFF7A0F81C2221462A
:100DC0002846F564EFF7B8FB54206861208FA885AA
:100DD00094F83A0085F82E00606B2862206BE86179
:100DE00004204EE0FFE794F83D0008B10E9913E0AF
:100DF00004984FF0FF3180B2401E08900498069589
:100E000001EB1040099007950023092206A90095DF
:100E10000E98FBF75DF906A90C98FDF7BAFF064698
:100E20006C2005F0EBFE0546FEF748FF1C2221462C
:100E30002846F564EFF780FB6C2000E026E045F8DB
:100E4000140F206BA86094F83B0085F83800208FC1
:100E5000A88694F83A0085F8360094F83C0085F8A6
:100E6000370094F83D10288F03AB61F34D3028878D
:100E700093E8070005F10C0383E80700E0692865A3
:100E80000520307131460C98FEF71CFE2C264FF0E1
:100E90000208BAF1000F26D00E990C98FDF779FFE1
:100EA00007462C2005F0AAFE05461C222146F864C0
:100EB000EFF742FB45F8146FE069A860E08FA88166
:100EC00094F84000A87394F848002875606C286175
:100ED00094F84900394600F01F00687587F80480CF
:100EE0000C98FEF7EFFDBBF1000F43D00E980FC832
:100EF0008DE80F00D4E91401421811466846FBF74B
:100F000091FA69460C98FDF744FF07462C2005F03E
:100F100075FEF8640546216D07F118000A46814602
:100F2000FBF780FA616D48460A46FBF77BFA1C2204
:100F300021462846EFF700FB6E61E16947F6FF7036
:100F4000814203D0206D0844616D084445F81C0FB0
:100F500034F84A0FA880A078A871A07B2873D4F831
:100F60000600A8600F20687387F8048039460C9843
:100F7000FEF7A8FD0FB0BDE8F08F000038B50446BD
:100F8000702105F0A4FFFDF78DFB0090BDF8000077
:100F900024F8210F9DF80200A070FDF783FB00905C
:100FA000BDF80000A4F803009DF802006071FDF791
:100FB0008FFA0090BDF8000020819DF80200A07219
:100FC000FF25257302206073FDF782FA0090BDF8BB
:100FD0000000A4F81D009DF80200E077FDF778FA04
:100FE0000090BDF8000020879DF8020084F83A00C8
:100FF0000948C4F8130004F8015CA57684F837505A
:1010000084F8275084F84B5014F8280F20F01F0064
:101010000F30207038BD00009CE402082DE9F74F26
:1010200091F83C00ADF5107D0C4602283CD9256AAC
:10103000002D39D0D4E90901884235D0A08EA842CC
:1010400000DA05460FCA69AE86E80F00909869A9D4
:1010500082680CA8FBF7F3F9002825D0A06B47F6AF
:10106000FF7928BB616AA06A01F5B472824203D09D
:1010700000F5B47081421BD180A8FEF7A8F894F85F
:101080003C008DF82802A08BADF82002A07F8DF8DF
:1010900022020F208DF82902CDF81C92899569AAA9
:1010A00080A9909800F09DFB0DF5137DBDE8F08FB1
:1010B000699865906A9866906B9867906C9868904C
:1010C0006599206A0144659166990844669067981D
:1010D000216A401A67906899206A081A6890D4E9D2
:1010E00009764FF4B47001E0A7F5B4778742FBDAD4
:1010F00002E000BFA6F5B4768642FBDA4FF00008A6
:10110000CDF80881CDF80C81CDF81081CDF814818F
:101110000096D4E90B123B4614A801F0A5FB14A8D5
:10112000429000234A4669A96EA801F00FFD6EA8FF
:10113000439000208D9065A8FBF76FF900280EDD25
:1011400065A8FBF75BF9002809DD01234A4665A97C
:1011500077A801F0FBFC77A8449001208D900CA8A3
:10116000FBF74CF908900CA8FBF757F9824605F0FD
:1011700045FD0DF1300B81469BE80F000DF1400B52
:101180008BE80F002C2137A8EFF710FACDF8F49078
:1011900094F83C008DF8F00010A837903F900020A4
:1011A0008E90A16B99B300224AA803F08FFC70B314
:1011B000559860B3CDF818815598CDF81C814FF043
:1011C000FF31808880B2401E48905598406801EBFE
:1011D000104049905598216B8088C0F34E000A1A40
:1011E000E16A091A46A8FBF76FFA46A83B905598A2
:1011F000006938905598008980B2399055980088D8
:10120000C0F307208DF8E800142808D012E0FFE7AB
:10121000A08BADF8F100A07F8DF8F3000AE012205A
:101220008DF8E8003B98FBF7E9F8DDE9381202FB9E
:1012300000108E9000206D9094F83D00C00748D0BB
:1012400005FB05F0834605F0D9FC5A46FF216D9059
:1012500005F005FE681E8B908C9005EBD570421052
:10126000CDF82482CDF82882002389A980A801F036
:101270006DFC80A8CDE909080020DDF8B4B10FE0CD
:1012800003460022594609A8009501F045FB20B904
:1012900058462A46002105F0E2FDAB4408F1010062
:1012A0008046A842ECDBEAB2A18E5DAB38B2F8F71B
:1012B000E4FAD4E90B125DA8FBF706FAEAB2A18EB4
:1012C00061AB30B2F8F7D9FAD4E90B1261A8FBF799
:1012D000FBF9119800260227139071E05246FF2176
:1012E000484605F0BCFDDDE910234946CDF800A0D5
:1012F00042A801F011FB8DF8F80094F83D10C907E1
:101300002DD05E9A1199914211DB609A91420EDCC8
:1013100030B948465246002105F0A1FD8DF8F8701D
:101320004B465DAA10A900956D98F2F7A4F8629952
:101330001198884213DB6499884210DC9DF8F8000C
:1013400030B948465246002105F089FD8DF8F87005
:101350004B4661AA10A900956D98F2F78CF88E980B
:1013600018B39DF8F80000B33B9A11998E98526813
:10137000891A399A520802FB01003B9A10991268A7
:10138000891A0144002008E019F800200B5C12FBC8
:1013900003F2120A09F80020401C5045F4DB9DF8C6
:1013A000F800012801D18DF8F87037A9909800F065
:1013B00024F81198401C11901398401C761C13902F
:1013C000089886428ADB14A801F0E4FA6EA801F0BE
:1013D000E1FA8D9810B177A801F0DCFA484602F0E6
:1013E00033FEA06B10B14AA803F010FB6D980028E3
:1013F0003FF45AAE02F028FE56E6F0B50546087DE9
:1014000095B00C4602287ED9A06910B1207F002833
:1014100079D0AA6868462168FBF711F8002872D0D5
:101420006D6800262868008987B26068E8B369465D
:1014300008462269FBF703F8002864D0226A2AB123
:1014400069460846FAF7FBFF00285CD06846FAF7C1
:10145000E4FF05906846FAF7D1FFCDE90607207D45
:101460008DF8310094F828008DF83200A0680B90B8
:10147000207B8DF83000207B6768FDF765F82269D6
:10148000019953681268C91A0B9B03FB0171009BF9
:101490009A1A424301EBD2000A90A069A0B3217FBF
:1014A00001295AD00890A06900E003E00890606A22
:1014B00058BB54E06846FAF7B0FF05906846FAF763
:1014C0009DFFCDE90607207D8DF82B00B4F81500AF
:1014D000ADF82800E07D8DF82A00A06910B3217FC7
:1014E00001291FD008909DE80F000BAE86E80F0081
:1014F000A8684242686841420BA8FBF7E5F80198EA
:10150000A968421A02E026E027E02BE0009869680B
:10151000411A2846FEF7E4FF04900898A8B1606AD3
:1015200010B104E00896DEE7206AFAF776FF09902A
:10153000206A009902684068891A019A101ADDE948
:10154000082303FB002008440890287D122802D1BC
:1015500004A800F041F815B0F0BD089610E0206A2C
:10156000FAF75BFF0990206A0099026840688A1ABE
:101570000199081ADDE9081303FB001010440890D4
:101580009DE80F000DAE86E80F00A868424268682B
:1015900041420DA8FBF798F8226911AE0FCA86E800
:1015A0000F00A86842426868414211A8FBF78CF816
:1015B0000198A968421A00986968411A2846FEF7FE
:1015C0008FFF0490287D122801D01428C3D104A8CD
:1015D00000F000F9BFE700002DE9F04F054685B0A7
:1015E000D5E901608046A869FDF74EF88146D5E946
:1015F000047095F81BA000902C68E86802902FB149
:10160000BAF1FD0F4FF0000074D2DFE0BAF1FD0F28
:1016100030D3002129E000BF701E20F00F0004EB42
:10162000400304EB4602A00701D024F8029B09EB1B
:1016300009400DE001C401C444F8080B44F8040C4F
:1016400044F8100B44F80C0C44F8080C44F8040C53
:101650009C42EFD302E000BF24F8029B9442FBD3EC
:101660000298491C2044A0EB46044145D4DB05B058
:10167000BDE8F08F2088401C03900020019004906A
:101680004045F4DA0025A00706D021885246484696
:10169000FCF700FF20800125A6F1020B5D4534DA3E
:1016A00004EB450734F81510788881420CD0524677
:1016B0004846FCF7EFFE24F8150079885246484664
:1016C000FCF7E8FE788013E000973A6803988242BE
:1016D00002D1019838600BE03868039052464846C2
:1016E000FCF7D8FE24F81500788000980068019077
:1016F000AD1CD3E750E000BF34F815105246484601
:10170000FCF7C8FE24F815006D1CB542F4DB029806
:1017100004440498401CB2E70025F80706D03A7844
:1017200021884846FCF7B6FE20800125A6F1020A72
:10173000554529DC785BA0F57F41FF3915D090B184
:101740007A5D34F815104846FCF7A4FE24F815001D
:10175000781904EB45014278019149884846FCF725
:1017600099FE01994880AD1CE2E724F8159048469F
:1017700004EB4501F6E77A5D34F815104846FCF7AE
:1017800089FE24F815006D1CB542F4DB0298044470
:10179000009807440BF1010083464045BCDB66E737
:1017A00000250BE0795D11FB0AF0020A34F81510F0
:1017B0004846FCF76FFE24F815006D1CB542F1DBBE
:1017C00002980444009807440BF101008346404509
:1017D000E6DB4CE790F82010122901D10FF0FCBE97
:1017E0007047F0B5074691F8280087B00C461646BA
:1017F00002285AD9606A002857D094F82900C006F8
:1018000053D01046FAF709FE05463046FAF7F6FDC2
:10181000E369854200DB0546B3EB650F00DD6B1025
:101820003068039070680490B0680590F068069086
:1018300094F82910039A4807606A01D4184440427A
:10184000104403900807059A606A01D41844404286
:10185000101A059094F8290004998007606A01D451
:10186000184440420844049094F829000699C0079F
:10187000606A01D118444042081A0690606A181A3A
:1018800000D5002053EA000111D094F828100291ED
:1018900034F8201FADF80410A1788DF806100090E0
:1018A00003AA31463846F3F712FC07B0F0BD94F8AE
:1018B0002800009003AA31463846236AF3F7CAFD90
:1018C000F3E700002DE9F04F0F4683461068C96A20
:1018D00014464218B86ABFB0121A1692A268114490
:1018E000084418906068396B169A0844B96A401A1F
:1018F0001790E068396B0844B96A08441990786A0F
:1019000000EBD071A2EB6100401E09900120189AF3
:1019100000EB610111440B91796A179A01EBD171C7
:10192000A2EB6101491E0A91796A199A01EBD17102
:1019300000EB610010440C9097F834003990FD28BA
:1019400001D9FF20399009A93AA8DBF80820FAF755
:1019500076FD00287DD0214626A8FAF7AEFC4FF090
:10196000FF310A4626A8FAF75DFDF869259026A8FA
:10197000FAF753FD044626A8FAF740FD844226A84C
:1019800002DAFAF74AFD01E0FAF738FD2599B1EBE2
:10199000600F01DD4010259016A8FD69FAF73DFDA6
:1019A000044616A8FAF72AFD844216A802DAFAF7C6
:1019B00034FD01E0FAF722FDB5EB600F00DD4510C4
:1019C000786A441904FB04F0400005F017F92B90E5
:1019D00001462B4616A87A6A11F02AFA97F83500C4
:1019E00010F001064FF000002D902E9007D101233A
:1019F00026A930A8259A01F0A9F830A82D9009A8A9
:101A0000FAF70BFD05F0FAF882461AA82C220021FD
:101A100005F025FA04A81A90CDF880A02290388C01
:101A2000ADF87D0097F822008DF87F0097F834001C
:101A30008DF87C0009A8FAF7F0FC099900EBD0704A
:101A400001EB600909A8FAF7D9FC00EBD0700A99FC
:101A500000E0FCE301EB60050B980690001B401CC6
:101A6000CDE90401601E149008440790049849468B
:101A7000484500DC084604900798A84200DB284649
:101A8000079004A90DA8DBF80820FAF7D8FC80B36A
:101A900026A90DA8259AFAF7F2FC50BB0DA8FAF773
:101AA000BCFC13900A9A0E992B98891A01FB04002A
:101AB0000B9A0D99121B891A0844401E039046B1D7
:101AC00026A90DA8259AFAF731FD10B101202F9013
:101AD00000E02F961398002820DD0D9804900F98B1
:101AE00006900220CDF880A08DF88400DDF83880C3
:101AF00011E013E0CDF81C802F98CDF8148028B3A6
:101B0000039820901AA95846FFF777FC039808F12C
:101B100001082044039010994145EBDA0B98069098
:101B2000001B401C04900C984946001B401C05906B
:101B30000C9807900498484500DC08460490681CFF
:101B400005991390814216DD084615E0224650465D
:101B5000039905F0C9F813980090434651462DA803
:101B60000D9A00F0D9FE8DF884000128CAD1022018
:101B70008DF88400C6E7681C059004A90DA8DBF861
:101B80000820FAF75CFC80B326A90DA8259AFAF77D
:101B900076FC50BB0DA8FAF740FC2A90109A0799E2
:101BA0002B98891A01FB04000B9A0D99121B891AB4
:101BB0000844401E039046B126A90DA8259AFAF7BD
:101BC000B5FC10B101202F9000E02F962A98002834
:101BD00020DD0D9804900F9806900220CDF880A08B
:101BE0008DF88400DDF8408011E013E0CDF81C8012
:101BF0002F98CDF8148058B3039820901AA958460E
